:020000022000DC
:10000000000004205126020061610600D96206004A
:100010006161060061610600616106000000000088
:100020000000000000000000000000006161060008
:100030006161060000000000616106006161060068
:100040005125020061610600CD2802003D28020012
:100050004D28020061610600B921020061610600BD
:1000600061610600AD280200BD28020021260200C1
:100070006161060061610600616106006161060060
:100080001D2D02003126020061610600616106003B
:100090006161060061610600616106006161060040
:1000A0006161060061610600616106006161060030
:1000B00061610600616106000000000000000000B0
:1000C0006161060061610600616106005D28020051
:1000D000412602006161060061610600ED28020010
:1000E000DD280200616106006161060085280200CA
:0800F000000000006161060040
:1010000040190800BC23080040190800C423080048
:1010100040190800CC23080040190800D423080018
:1010200040190800DC23080040190800F4230800D8
:1010300040190800FC23080040190800B0240800EB
:1010400040190800B824080040190800C02408000E
:1010500040190800E824080040190800F02408009E
:10106000401908000825080040190800102508004C
:10107000401908001825080040190800202508001C
:1010800040190800382508004019080040250800CC
:1010900040190800A825080040190800A0260800EB
:1010A00040190800A8260800401908002027080059
:1010B000401908003827080040190800A827080030
:1010C00040190800B027080040190800D827080078
:1010D00040190800E027080040190800E827080028
:1010E00040190800F027080040190800F8270800F8
:1010F00040190800002808004019080008280800C6
:101100004019080010280800401908001828080095
:101110004019080020280800401908002828080065
:101120004019080030280800401908003828080035
:101130004019080040280800401908004828080005
:1011400040190800502808004019080058280800D5
:10115000401908006028080040190800D828080035
:1011600040190800F028080040190800F828080075
:101170004019080000290800401908001829080033
:1011800040190800202908004019080078290800A3
:1011900040190800C029080040190800282A080042
:1011A00040190800502A080040190800982A080031
:1011B00040190800D02A080040190800082B080030
:1011C00040190800102B080040190800782B08006F
:1011D00040190800B02B080040190800082C08002E
:1011E00040190800102C080040190800182C0800AD
:1011F00040190800302C080040190800382C08005D
:1012000040190800402C080040190800502C080024
:1012100040190800582C080040190800702C0800DC
:1012200040190800882C08004019080028280900E7
:1012300040190800B82C0900401908007423080060
:101240006C23080040190800842308007C23080050
:1012500040190800942308008C2308004019080056
:10126000A42308009C23080040190800B4230800A8
:10127000AC230800401908000C24080004240800CE
:1012800040190800D0240800C824080040190800AC
:10129000E0240800D82408004019080000250800B0
:1012A000F824080040190800302508002825080007
:1012B000401908005025080048250800401908007A
:1012C000602508005825080040190800702508000E
:1012D00068250800401908008025080078250800C6
:1012E00040190800902508008825080040190800CA
:1012F000A02508009825080040190800B825080016
:10130000B025080040190800C8250800C0250800BD
:1013100040190800D8250800D02508004019080009
:10132000E8250800E025080040190800F825080015
:10133000F0250800401908000826080000260800CB
:101340004019080018260800102608004019080057
:101350002826080020260800401908003826080022
:1013600030260800401908004826080040260800DA
:1013700040190800582608005026080040190800A7
:101380006826080060260800401908007826080032
:1013900070260800401908008826080080260800EA
:1013A00040190800982608009026080040190800F7
:1013B000B8260800B026080040190800C826080012
:1013C000C026080040190800D8260800D0260800CA
:1013D00040190800E8260800E02608004019080027
:1013E000F8260800F0260800401908000827080021
:1013F00000270800401908001827080010270800D7
:101400004019080030270800282708004019080064
:1014100050270800482708004019080060270800E6
:10142000582708004019080070270800682708009E
:101430004019080080270800782708004019080094
:10144000902708008827080040190800A0270800F6
:101450009827080040190800C0270800B82708008E
:1014600040190800D0270800C827080040190800C4
:101470007028080068280800401908008028080023
:1014800078280800401908009028080088280800DB
:1014900040190800A02808009828080040190800F2
:1014A000B0280800A828080040190800D028080023
:1014B000C828080040190800E8280800E0280800AB
:1014C00040190800102908000829080040190800E0
:1014D0003029080028290800401908004029080080
:1014E0003829080040190800502908004829080038
:1014F0004019080060290800582908004019080010
:101500007029080068290800401908008829080087
:10151000802908004019080098290800902908002F
:1015200040190800A8290800A0290800401908004F
:10153000B8290800B029080040190800D02908007F
:10154000C829080040190800E0290800D829080027
:1015500040190800F0290800E8290800401908008F
:10156000002A0800F829080040190800102A08007D
:10157000082A080040190800202A0800182A080034
:1015800040190800382A0800302A080040190800CD
:10159000482A0800402A080040190800602A08006C
:1015A000582A080040190800702A0800682A080014
:1015B00040190800802A0800782A0800401908000D
:1015C000902A0800882A080040190800A82A080064
:1015D000A02A080040190800B82A0800B02A08000C
:1015E00040190800C82A0800C02A0800401908004D
:1015F000E02A0800D82A080040190800F02A08004C
:10160000E82A080040190800002B0800F82A080002
:1016100040190800202B0800182B0800401908006A
:10162000302B0800282B080040190800402B080028
:10163000382B080040190800502B0800482B0800E0
:1016400040190800602B0800582B080040190800BA
:10165000702B0800682B080040190800882B080030
:10166000802B080040190800982B0800902B0800D8
:1016700040190800A82B0800A02B080040190800FA
:10168000C02B0800B82B080040190800D02B080018
:10169000C82B080040190800E02B0800D82B0800D0
:1016A00040190800F02B0800E82B0800401908003A
:1016B000002C0800F82B080040190800282C08000E
:1016C000202C0800401908000E000000482C0800DB
:1016D00040190800682C0800602C08004019080018
:1016E000802C0800782C080040190800982C08006D
:1016F000902C08004019080000280900F82709006C
:10170000401908001028090008280900401908009D
:10171000202809001828090040F8044B40F8045B11
:1017200040F8046B40F8047B40F8048B40F8049BBD
:1017300040F804AB40F804BB40F804CB40F804DBAD
:101740006846704781F0004102E000BF83F000432B
:1017500030B54FEA41044FEA430594EA050F08BF4C
:1017600090EA020F1FBF54EA000C55EA020C7FEA10
:10177000645C7FEA655C00F0E2804FEA5454D4EB8D
:101780005555B8BF6D420CDD2C4480EA020281EA57
:10179000030382EA000083EA010180EA020281EA8F
:1017A0000303362D88BF30BD11F0004F4FEA0131E1
:1017B0004FF4801C4CEA113102D0404261EB4101F0
:1017C00013F0004F4FEA03334CEA133302D0524276
:1017D00063EB430394EA050F00F0A780A4F1010432
:1017E000D5F1200E0DDB02FA0EFC22FA05F280186C
:1017F00041F1000103FA0EF2801843FA05F3594152
:101800000EE0A5F120050EF1200E012A03FA0EFCD0
:1018100028BF4CF0020C43FA05F3C01851EBE371FA
:1018200001F0004507D54FF0000EDCF1000C7EEB17
:1018300000006EEB0101B1F5801F1BD3B1F5001F55
:101840000CD349085FEA30004FEA3C0C04F1010474
:101850004FEA445212F5800F80F09A80BCF1004F9D
:1018600008BF5FEA500C50F1000041EB045141EA1F
:10187000050130BD5FEA4C0C404141EB0101013CE8
:1018800028BFB1F5801FE9D291F0000F04BF0146D7
:101890000020B1FA81F308BF2033A3F10B03B3F1A9
:1018A00020020CDA0C3208DD02F1140CC2F10C0239
:1018B00001FA0CF021FA02F10CE002F11402D8BF97
:1018C000C2F1200C01FA02F120FA0CFCDCBF41EA63
:1018D0000C019040E41AA2BF01EB0451294330BD32
:1018E0006FEA04041F3C1CDA0C340EDC04F114040F
:1018F000C4F1200220FA04F001FA02F340EA0300E6
:1019000021FA04F345EA030130BDC4F10C04C4F12B
:10191000200220FA02F001FA04F340EA030029460B
:1019200030BD21FA04F0294630BD94F0000F83F455
:10193000801306BF81F480110134013D4EE77FEA38
:10194000645C18BF7FEA655C29D094EA050F08BF84
:1019500090EA020F05D054EA000C04BF1946104665
:1019600030BD91EA030F1EBF0021002030BD5FEAA9
:10197000545C05D14000494128BF41F0004130BDD1
:1019800014F580043CBF01F5801130BD01F0004525
:1019900045F0FE4141F470014FF0000030BD7FEA98
:1019A000645C1ABF194610467FEA655C1CBF0B4693
:1019B000024650EA013406BF52EA033591EA030FAA
:1019C00041F4002130BD00BF90F0000F04BF0021A2
:1019D000704730B54FF4806404F132044FF00005D5
:1019E0004FF0000150E700BF90F0000F04BF00214E
:1019F000704730B54FF4806404F1320410F00045B4
:101A000048BF40424FF000013EE700BF42004FEAAE
:101A1000E2014FEA31014FEA02701FBF12F07F432B
:101A200093F07F4F81F06051704732F07F4208BFE2
:101A3000704793F07F4F04BF41F40021704730B5E9
:101A40004FF4607401F0004521F000411CE700BF35
:101A500050EA010208BF704730B54FF000050AE0B8
:101A600050EA010208BF704730B511F0004502D5B9
:101A7000404261EB41014FF4806404F132045FEABB
:101A8000915C3FF4D8AE4FF003025FEADC0C18BF64
:101A900003325FEADC0C18BF033202EBDC02C2F156
:101AA000200300FA03FC20FA02F001FA03FE40EAE8
:101AB0000E0021FA02F11444BDE600BF4FEA4102D4
:101AC000B2F1E04324BFB3F5001CDCF1FE5C0DD99C
:101AD00001F0004C4FEAC0024CEA5070B2F1004FE6
:101AE00040EB830008BF20F00100704711F0804FE9
:101AF00021D113F13872BCBF01F00040704741F4AE
:101B000080114FEA5252C2F11802C2F1200C10FAB1
:101B10000CF320FA02F018BF40F001004FEAC12395
:101B20004FEAD32303FA0CFC40EA0C0023FA02F339
:101B30004FEA4303CCE77FEA625307D150EA01330F
:101B40001EBF4FF0FE4040F44000704701F00040DF
:101B500040F0FE4040F40000704700BF53B94AB95E
:101B6000002908BF00281CBF4FF0FF314FF0FF30A5
:101B700000F036B9ADF1080C6DE904CE02F05AF967
:101B8000DDF804E0DDE9022304B0704770B54FF0E2
:101B9000FF0C4CF4E06C1CEA11541DBF1CEA1355F9
:101BA00094EA0C0F95EA0C0F00F0DEF82C4481EA61
:101BB000030621EA4C5123EA4C5350EA013518BF81
:101BC00052EA033541F4801143F4801338D0A0FB6E
:101BD00002CE4FF00005E1FB02E506F00042E0FB1B
:101BE00003E54FF00006E1FB03569CF0000F18BF21
:101BF0004EF0010EA4F1FF04B6F5007F64F54074C9
:101C000004D25FEA4E0E6D4146EB060642EAC6215B
:101C100041EA55514FEAC52040EA5E504FEACE2EC8
:101C2000B4F1FD0C88BFBCF5E06F1ED8BEF1004FCB
:101C300008BF5FEA500E50F1000041EB045170BD47
:101C400006F0004646EA010140EA020081EA03018B
:101C5000B4EB5C04C2BFD4EB0C0541EA045170BD87
:101C600041F480114FF0000E013C00F3AB8014F101
:101C7000360FDEBF002001F0004170BDC4F100044A
:101C8000203C35DA0C341BDC04F11404C4F12005CB
:101C900000FA05F320FA04F001FA05F240EA020026
:101CA00001F0004221F0004110EBD37021FA04F65C
:101CB00042EB06015EEA430E08BF20EAD37070BD16
:101CC000C4F10C04C4F1200500FA04F320FA05F075
:101CD00001FA04F240EA020001F0004110EBD37077
:101CE00041F100015EEA430E08BF20EAD37070BDE7
:101CF000C4F1200500FA05F24EEA020E20FA04F3C0
:101D000001FA05F243EA020321FA04F001F000416E
:101D100021FA04F220EA020000EBD3705EEA430EDF
:101D200008BF20EAD37070BD94F0000F0FD101F00E
:101D30000046400041EB010111F4801F08BF013C47
:101D4000F7D041EA060195F0000F18BF704703F085
:101D50000046520043EB030313F4801F08BF013D0C
:101D6000F7D043EA0603704794EA0C0F0CEA1355C8
:101D700018BF95EA0C0F0CD050EA410618BF52EA82
:101D80004306D1D181EA030101F000414FF0000088
:101D900070BD50EA410606BF1046194652EA430696
:101DA00019D094EA0C0F02D150EA013613D195EA0A
:101DB0000C0F05D152EA03361CBF104619460AD152
:101DC00081EA030101F0004141F0FE4141F470015C
:101DD0004FF0000070BD41F0FE4141F4780170BD4C
:101DE000704700BF4A0011D212F5001211D20DD572
:101DF0006FF47873B3EB62520ED44FEAC12343F011
:101E0000004343EA505323FA02F070474FF00000BA
:101E1000704750EA013002D14FF0FF3070474FF069
:101E200000007047182A2DE9F74F054621D0202AD7
:101E300022D00A200423C5F8002185F8040185F882
:101E40000531284600F098FA0022034695F805412E
:101E5000A24214D3DFF8DCC0DFF8DCE000EB84033F
:101E600095F804210132B4EB820F1AD303B0BDE818
:101E7000F08F0C200623DEE70E200823DBE711F8A5
:101E8000044B03F8044B11F8034C03F8034C11F80E
:101E9000024C03F8024C11F8014C03F8014C0132DA
:101EA000D4E795F80521B4FBF2FA02FB1A4913F8BE
:101EB000041C13F8038C13F8027C13F8016C0192D4
:101EC000B9F1000F0BD11CF808B01CF807801CF802
:101ED00006701CF801601EF80A108BEA0101D5F8A3
:101EE0000021202A0CD1B9F1040F09D1DFF8449068
:101EF00019F8011019F8088019F8077019F8066028
:101F0000019AA21A043310F8229000EB820281EAAF
:101F1000090103F8041C517888EA010803F8038CCE
:101F200091784F4003F8027CD278564003F8016C58
:101F3000013495E7173309000C3309002DE9F04F00
:101F4000044685B0084600F017FA894602468046E6
:101F50002146002044F0E1F8231D019304F1100311
:101F60000125029322462146002311F82300324E18
:101F7000305C01F823000133042BF6D1019B0131C1
:101F80008B42F1D1617963786170617A6171617BB3
:101F90006172A17A6373A378A170A17BA372A37904
:101FA000A171E17BA373E378E170E17AE173E179F8
:101FB000E172E37199F80431AB4234D092F800B089
:101FC0005678917892F803A08BEA060081EA0A031A
:101FD00080EA0307039356F0CBFE8BEA00007840BB
:101FE000107086EA010056F0C3FE46407E405670EF
:101FF000039856F0BDFE4140794091708BEA0A008B
:1020000056F0B6FE8AEA000A029B87EA0A07D770F2
:1020100004329342D2D1284642462146013544F04B
:102020007CF8EDB29EE742462146284605B0BDE861
:10203000F04F44F072B800BF173309002DE9F04F9C
:10204000504C904603F003029B101F2B04EB8214AC
:1020500089469E464C49A8BF4FF01F0E1C2B1D46BB
:10206000A8BF1C2551F822206168033587B025EAF6
:10207000E575294101920391E268A16884462941EE
:1020800000202A410290049105925CF8045B3F4ACB
:10209000154225F0004111D106AA02EB810151F849
:1020A000102C002D40EA0200B8BF5242B8F10108DE
:1020B00049F8042BE9D107B0BDE8F08F344A154246
:1020C00009D154F82120002BBABFCEF100018A407B
:1020D00042FA0EF2E5E72F4A154214D110392E4A82
:1020E000019E52F8212082FB0616AEF10302002A5F
:1020F00044DA51426FF0004242FA01F7B742D0DBB6
:1021000006FA01F2CDE74A04B2F1006FB6BF4A0504
:1021100000210421B2F1005FB8BF92001F4EB8BF8A
:102120000231B2F1804FBCBF52000131B242C7BF91
:102130001B4F1C4E1C4F1D4E924687FB0ABA7768F8
:102140005744924687FB0ABAB7685744924687FBC2
:102150000ABAF768BA448AFB027236691644144A0E
:1021600052F8212086FB0272019ED20082FB067685
:10217000104A52F82120AEEB0202B8E746FA02F20A
:102180008FE700BFC8670900B8670900FCFFFF7F41
:10219000F0FFFF7FC0FFFF7FF86609009979825A40
:1021A0006321851090660900A9BDA029A4660900D5
:1021B000D8660900B86609002DE9F04F00248BB0FD
:1021C000CDE90444664B67486749012225461E68ED
:1021D00046B1D0F80463164204D01D601E68029612
:1021E000029E144304338B424FEA4202EFD15D4B0F
:1021F000D3F87C218AB10022C3F87C21D3F87C314A
:102200000393039B4FF0A04344F00044D3F81035F0
:102210000493564BD3F810350593E3B2D3B1544F22
:1022200001260025344210D0AB0003F1804303F5B2
:10223000C043D3F81005D3F8101557F8253023B153
:10224000C1F30141C0F3052098470135082D4FEA3D
:102250004606E7D1002C7FDA0DF1200B002308930E
:10226000CBF80430DFF804914FF0FF330693079367
:102270000025404B0193A846019A12F9013F0192B3
:102280005A1C50D0C3F3C20000F128020DEB020C1F
:1022900003F007011CF8102CCA40D707DCB203F08A
:1022A0003F0640D5324A17463244A40992F9282005
:1022B00057F822A0BAF1000F0AD1032C33D11BF832
:1022C00000E001228A4042EA0E020BF8002001E001
:1022D000032CF4D01F2E8BBF03F01F0333464A4656
:1022E0004FF0A04203F5E07352F823301CF8182C8D
:1022F000CA40D207C3F3014305D5022B13D1032CE7
:102300000BD1214604E0032B0DD1032C05D1022172
:10231000304630F077FD0135EDB2BAF1000F02D052
:1023200021463046D04708F10103022B4FF0010847
:10233000A2D18DB14FF0A0430499D3F81025D9F85C
:102340001035914202D10599994205D00492089A1C
:10235000CDE90532099B8AE70BB0BDE8F08F00BFDD
:102360000061004000600040206100400003005018
:10237000086A00205F6A0020D0F80031103B102B63
:1023800007D8054A22FA03F313F0010F08BF002013
:1023900070470020704700BF010101002DE9F04F98
:1023A00004468DB00846FFF7E7FF0D460190024650
:1023B000214695F8040143F0B0FE95F80461231D11
:1023C000013E099304F11003F6B20A93627A637B2B
:1023D00062736279627262786271A27A6370A378C2
:1023E000A270A27BA372A379A271E279A373E378AE
:1023F000E270E27AE271E27BE272E3732546224602
:10240000002312F823105148415C02F823100133D5
:10241000042BF6D1099B01329342F1D1019A214656
:10242000304643F07AFE002E00F08C8095F8008054
:10243000AB780093404656F09BFC029056F098FC17
:10244000039056F095FC6F780B90384656F090FC50
:10245000024656F08DFC049056F08AFC82460098A5
:1024600095F803B056F084FC059056F081FC069078
:1024700056F07EFC8146584656F07AFC079056F09E
:1024800077FC089056F074FCDDE9023183EA010C18
:102490000B9B069983EA0C0C82EA0C0C8AEA0C0C62
:1024A00081EA0C0C89EA0C0C009980EA0C0C87EA92
:1024B0000C0C81EA0C0C04995A404A4005998AEAAE
:1024C00002024A40089989EA02024A4042400099C1
:1024D00088EA02024A408BEA02026A70039A05996E
:1024E0005A408AEA02024A4006994A40079989EA14
:1024F00002024A40424088EA02027A408BEA0C0C0F
:102500008BEA020B85F800C085F802B0029A5340AE
:10251000049A53408AEA030A089A89EA0A0981EA76
:1025200009035340584000990A9B88EA000887EA4B
:1025300008077940E9700435AB427FF477AF013E7C
:10254000F6B243E70DB0BDE8F08F00BF0C320900D2
:1025500010B54FF08043D3F80443620707D54FF41A
:10256000847051F09BFF10B11C4B1B689847A30669
:1025700006D54FF48A7051F091FF08B100208047D2
:10258000600607D54FF48C7051F088FF10B1012020
:1025900000239847210608D54FF48E7051F07EFF36
:1025A00018B10F4B00201B689847E20508D54FF47F
:1025B000907051F073FF18B1094B01201B689847C8
:1025C000A3050AD54FF4927051F068FF28B1044B6F
:1025D000BDE810401B680220184710BD886B002022
:1025E0008C6B0020DFED0A7A9FED0A7ADFED0A6A34
:1025F000A0EE277ADFED097AE7EE007AB7EE007AEF
:10260000A0EE267A67EE807A87EE870A704700BFD1
:102610006BD30DBCBA132FBDAEE534BF75AA2A3EED
:102620000248032200211CF03FB900BF00B0004067
:102630000248042201211CF037B900BF00100140FC
:102640000248042202211CF02FB900BF00400240C2
:1026500008B54FF0E0236B4AC3F8082DBFF34F8F46
:10266000694B6A4A6A498B42C0F0BF80694B6A4A2B
:1026700000219342C0F0BE804FF08053D3F8302148
:10268000082A4ED14FF080420021C2F80C11C2F846
:102690001011C2F8381502F54042D3F80414C2F8FC
:1026A0002015D3F80814C2F82415D3F80C14C2F876
:1026B0002815D3F81014C2F82C15D3F81414C2F846
:1026C0003015D3F81814C2F83415D3F81C14C2F816
:1026D0004015D3F82014C2F84415D3F82414C2F8D6
:1026E0004815D3F82814C2F84C15D3F82C14C2F8A6
:1026F0005015D3F83014C2F85415D3F83414C2F876
:102700006015D3F83814C2F86415D3F83C14C2F835
:102710006815D3F84014C2F86C15D3F84434C2F8E5
:10272000703548F06DF918B13C4B3D4AC3F88C2622
:1027300048F066F918B13B4BFB22C3F8182548F066
:102740005FF958B14FF080424FF08051D2F8E43E2B
:10275000D1F8581261F30303C2F8E43E48F050F98F
:1027600020B1314B4FF40072C3F840264FF0805334
:10277000D3F83031082B09D14FF08043D3F800242F
:10278000D20744BF6FF00102C3F80024274AD2F8F1
:10279000883043F47003C2F88830BFF34F8FBFF323
:1027A0006F8F4FF01023D3F80C32DB0725D5204B69
:1027B0000122C3F80425D3F80024002AFBD04FF0EF
:1027C0001022D2F80C3223F00103C2F80C32184B5D
:1027D000D3F80024002AFBD00022C3F80425D3F844
:1027E0000024002AFBD000F069FB52F8040B43F8E8
:1027F000040B38E743F8041B3BE70E4B0E4A1A6004
:1028000039F048FB0000020000200020FC710900A4
:1028100084220020C0220020F879002000500040CF
:102820004881030000F000400090024000ED00E00D
:1028300000E00140002000200090D0030149024840
:102840003DF064BFCC6A00200030004002494FF0E8
:1028500040203DF05BBF00BF006B002008B507487B
:10286000D0F8183143B14FF48C7151F00FFEBDE830
:102870000840034849F00BBB08BD00BF00300240D0
:102880006C6A002008B50748D0F8183143B14FF4FE
:102890008C7151F0FBFDBDE80840034849F0F7BAE0
:1028A00008BD00BF00F00240906A002001490248C4
:1028B00049F014BFB46A002000900040014902486A
:1028C00049F00CBFC06A002000A000400149024846
:1028D00055F0FEBB346B0020002000400149024847
:1028E00055F0F6BB586B0020008002402DE9F04FF8
:1028F000BC4BBD4AD3F80013002385B01C46012011
:102900001D4621FA03F6F6070BD552F8236046B1AF
:1029100000FA03F6344342F82350BFF36F8FBFF33E
:102920004F8F0133192BECD1E10738D5AD4B012284
:10293000C3F81425C3F8102500221546930003F1AF
:10294000804303F51C330132082A5D609D62F5D196
:10295000A44BA6485D629D64C3F85851D3F8002487
:10296000D3F800140A43C3F80024D3F80023C3F8B3
:1029700008239F4AC3F8042300214FF492724AF0BF
:102980007CFB9A4A8DF80850402313831381012160
:102990004FF4807301A8ADF8043013F06FFE14F407
:1029A000006F924D07D08F4BD3F8A836A5F816319B
:1029B000012385F81C31A20204F4800635D5894A2A
:1029C000D2F8143513F4807308D01EB1D2F8003455
:1029D000DB0702D4082041F0DDFA0123814AD2F856
:1029E0001015CF0540F14A8195F81C318BB10023B9
:1029F00085F81C31B5F816319BB24FF4E0620393B1
:102A00000121882301A8ADF80420ADF8083013F0A7
:102A100035FE744B4FF44072D3F8203502930121F8
:102A200001A8ADF8042013F029FE7EB36D4BD3F856
:102A3000006440F201723240F005C3F8002409D569
:102A40000121C3F82C1501A84FF48063ADF80430C0
:102A500013F014FE71050FD5624B0122C3F808254F
:102A60009A65D3F8002312F4001208BFC3F854216A
:102A70004FF40012C3F80423B20507D54FF4A06346
:102A8000012101A8ADF8043013F0F8FD23022ED582
:102A9000544BD3F88014D3F88424D3F888E4D3F8C3
:102AA0008CC4D3F89074D3F89464D3F89804D3F812
:102AB0009C3411F07F0FD2B201D1052A17D04FF408
:102AC000C0688DF808108DF80E00012101A8ADF83E
:102AD00004808DF809208DF80AE08DF80BC08DF880
:102AE0000C708DF80D608DF80F3013F0C7FD414B61
:102AF00023403BB1BFF35B8F3F4B4FF000021A7096
:102B0000BFF35B8F394FDFF8DCB00026B8464FF0DB
:102B1000140AB14606F10C0324FA03F3D80726D5AC
:102B20000AFB06B305EB4611D3F80827D8F80030A6
:102B300013FA82F3C8F80030B1F806C090B2082E3C
:102B40001CFA82F24FEA4613CA8000F0A480B8F85B
:102B50000820824240F09F80CA88B8F8041092B2E0
:102B6000914240F2988016B9244815F0CBF901360D
:102B7000092E08F12008CDD1214B2340002B00F075
:102B80009480184BD3F86C84C3F86C84BFF36F8FB8
:102B9000BFF34F8F14F480641CBFD3F88044D3F884
:102BA0008064DFF848A01DBFC6F3C016C4F3C0148C
:102BB00086F0010626464FF000094FF4E06B28FA34
:102BC00009F1CA0703D4B9F1000F31D184B3054B21
:102BD000142202FB09315FFA89F0D1F80836DAF8DD
:102BE00010100FE00070024000710240E03B002036
:102BF0000514C001FCFB1F00003D00204C7002408A
:102C00000004000151FA83F1CAF8101005EB4911D4
:102C1000B1F816E05EFA83FCA1F816C0B1F816C050
:102C2000BAF814E01FFA8CFCE6455ED941F092F93F
:102C300009F10109B9F1080F0AF1200ABFD10024F6
:102C40004FF0010904F1100328FA03F3DB0701D464
:102C500074B96EB105EB44126301D17A002955D0E5
:102C6000D288B98892B2914250D9E0B241F092F93B
:102C70000134082C07F12007E4D116E0002B7FF483
:102C8000C8AE95F82131002B7FF4C3AE4FF400138A
:102C9000C2F80833BDE62B44DA7A8AB94FF0E02354
:102CA000D3F8F03DD90700D500BE1A4A1A4B13607D
:102CB00010460023536005B0BDE8F04F0AF05AB942
:102CC000DA88A8F8042083F80B90DB888DF8086078
:102CD0009BB24FF4E062012101A8ADF804200393F8
:102CE0008DF8099013F0CAFC41E7C98AADF804B029
:102CF00089B260F07F00039100218DF808008DF803
:102D0000091001A8012113F0B9FC91E72B4483F8C5
:102D10000A90ADE748700020EB83070010B5074C20
:102D2000D4F8003143B10023984720464FF4807116
:102D3000BDE8104051F0AABB10BD00BF000001402B
:102D4000022A2DE9F04159D13B4B826883FB0242B4
:102D50003A4D846985FB046422440A60DFF8F0C0C0
:102D600042688CFB0242364EC46986FB04742244DE
:102D70004A60026883FB0242046A85FB04642244C1
:102D80008A60304E026886FB02422F4C056A84FB43
:102D900005752A44CA604FF06045426885FB02729F
:102DA000C76985FB07E73A440A61826884FB0272BF
:102DB000876986FB07E73A444A61426983FB0272EE
:102DC0008A6102698CFB0272CA61C26883FB02726B
:102DD0000A62C36886FB03234B62036985FB0323F6
:102DE0008B62436984FB0323CB620023C1E9103368
:102DF000C1E90E33C1E90C33BDE8F081134B9024D7
:102E000004FB023202F1480E02F18C0501F1440686
:102E1000683250F8043B55F804795EF804CB1C4640
:102E20008CFB048441F8044B87FB0343AA4246F819
:102E30000439EED1E0E700BFD8E3CEB8281C310753
:102E4000CD3C410D9A615FC9669EA0F650640900B1
:102E500033C3BEB200280CDB4309064900F01F0053
:102E600020330122824041F82320BFF34F8FBFF36C
:102E70006F8F704700E100E04309064900F01F0032
:102E800020330122824041F82320BFF34F8FBFF34C
:102E90006F8F704700E100E00028ABBF00F1604099
:102EA000054B00F5614000F00F004FEA4111B4BF3F
:102EB000195480F80013704714ED00E0BFF34F8FF2
:102EC0000549064BCA6802F4E0621343CB60BFF3C6
:102ED0004F8F00BFFDE700BF00ED00E00400FA05E2
:102EE000014B1868704700BF5420002007EE900A7D
:102EF000F5EEC07AF1EE10FA01D400F009B808B589
:102F000080F0004000F004F8404261EB410108BD50
:102F100070B5FEF77BFD0C4B002204460D46FEF714
:102F200035FEFEF75FFF0646FEF74EFD074B00221B
:102F3000FEF72CFE02460B4620462946FEF706FC0D
:102F4000FEF750FF314670BD0000F03D0000F0413B
:102F500070B510EE105A25F000440123B4F1FF4F74
:102F6000B0EE403A0646036004D320EE003AB0EEDD
:102F7000430A70BD34B9DFEDD07AB7EE007A87EE40
:102F8000273AF4E7B4F1E45F0BD2002DBEBF4FF057
:102F9000FF330360B1EE400A1DF08EFDB1EE403A02
:102FA000E5E7002D80F2C682B4F1964FE3D2B4F18A
:102FB0007A5F9FEDC25A78D2DFEDBF0A20EE050A94
:102FC000002000F015FEF0EE402AF5EE402AF1EE6A
:102FD00010FAD0D023EE220AB0EEC00A85EE000A25
:102FE0001DF06AFDF5EEC02AF1EE10FAB0EE402AAF
:102FF00040F1B9804FF0FF33B4F17E5F336000F0F1
:103000009382B4F1804F00F08F82B1EE433A6B00AF
:1030100000F1DE81AA4B9C4200F2F580B0EE430A3B
:103020001DF04AFDA74B9C42B1EE400A40F29D8044
:10303000B7EE007A37EE437A67EE077ADFEDA26AE1
:103040009FEDA26A9FEDA23AA7EEA66ADFEDA16A04
:10305000E6EE276A9FEDA06AA6EEA76ADFED9F6AFB
:10306000E6EE276A9FED9E6AA6EEA73ADFED9D6A1F
:10307000E7EE866A9FED9C6AA6EEA76ADFED9B6A83
:10308000E6EE276A9FED9A6AA6EEA76ADFED996AD7
:10309000E6EE276A23EE073AA6EEA73AF6EE007AA6
:1030A000A7EE673A33EE003AFFE0B1EE407AB0EEB9
:1030B000470A18F043FAB4EE407AF1EE10FA19D04C
:1030C000F6EE007A27EE277AB0EE470A18F036FAC5
:1030D00037EE400A30EE000AF0EE407AFEEECF7A8C
:1030E00017EE903A062B39D8DFE803F02312121FAF
:1030F0001F2B2B00DFED807A77EEC37A17EE903A24
:1031000003F0010307EE903A9B00B8EEE70AE9E707
:10311000F6EE007A37EEC00ADFED670A20EE050A08
:1031200000F036FBF1EE402A4FE7F7EE007A37EE7B
:10313000C00ADFED610A20EE050A002000F058FD0C
:10314000F0E7F7EE087A30EE670ADFED5B0A20EE73
:10315000050A00F01DFBB1EE400AE3E7F0EE007A4D
:1031600030EE670AE5E7012346E7644B9C4264D9E9
:103170009FED637A33EE477A67EE074A9FED616A07
:10318000DFED616ADFED615A9FED615A9FED613AB3
:1031900064EE877AE7EE866A9FED5F6AA6EEA76A1D
:1031A000DFED5E6AE6EE276A9FED5D6AA6EEA76A2E
:1031B000DFED5C6AE7EEA65ADFED5B6AE5EEA76A33
:1031C000DFED5A5AE6EEA75ADFED596AE5EEA76A37
:1031D000DFED585AA7EEA55ADFED575AE5EE275A0C
:1031E0009FED565AA5EEA75ADFED555AE5EE275A40
:1031F000E5EE876AA6EEE73ADFED527A94EE863A7C
:1032000033EE673A4EE7504B9C4206D9B0EE007A57
:1032100037EE437A9FED280A0EE74C4B9C4206D9C5
:103220009FED4B7A9FED240A33EE477AA4E7F7EE41
:10323000007A33EE673A9FED200A9FED467ADFED84
:10324000467ADFED466AE3EE077A9FED457AA7EE10
:10325000837ADFED447AE7EE037A9FED437AA7EEB7
:10326000837ADFED4D7AE7EE037A9FED407AE3EE65
:10327000076A9FED3F7AA6EE837ADFED3E6AE7EEBE
:10328000036A9FED3D7AA6EE837AF7EE006AE7EED9
:10329000036A67EE837A87EEA67AFEEE006AF0EEA6
:1032A000477AE3EE267A37EE803A002DBFF65FAE1E
:1032B00032EE433A5BE600BF00000000DB0F4940FE
:1032C0006666663F1F4A3B3FA283D33767976739DD
:1032D0003F239E3DA1549C3A7E02F23B01F0893D82
:1032E000752C3C384584E23834B6053AC66E3D3B11
:1032F0001599A83C661AA53E0000004B07336D3EA9
:103300000C5BEC3E6B7BA53976F4B7BA67F8663A8E
:1033100085300DBA521CE63107E7C73B474D06BD65
:103320005EB9F73E27F9A3B9FE7771BB3D37933CF1
:103330003C2117BEF7E9AF399916143BFEFC28BCB7
:10334000155A843DCDCDF83D17A6DD3F1FA69D3F04
:10335000C316BB3F5E3C5B3C78756A3EAF72D53DA1
:10336000B24B7A3FE73ABA3FF400223FDBD5523BFB
:10337000DFEF443F2D390840BE2E1D4067FF053862
:10338000B435F13ABDD7F536E440DA3CE6DC153E1B
:103390007ACCA63E5A245C3E3F239EBDD6EE4B3AE5
:1033A00054BF983C6E0F303EC5D0383F3B2DB23FE6
:1033B000E8C4D5BAD23D5B3A5C061CBAFD0C503A63
:1033C000610B36BBABAAAA3D1D7FD63E00000000B4
:1033D000B4F1824FF7EE002A75D2FDEEC35A1FED0D
:1033E000197A5FED196A1FED196AF8EEE57A15EEA4
:1033F000903A73EE677A033BE7EE876A1FED1E7A19
:10340000A6EEA77A5FED1F6AE7EE276A1FED207A26
:10341000A6EEA77A5FED216AE7EE276A1FED227A12
:10342000A6EEA77A5FED236AE7EE866A1FED246AAF
:10343000A6EEA76A5FED256AE6EE276A1FED266A0B
:10344000A6EEA76A5FED276AE6EE276A27EE277ADF
:10345000E6EEA72A87EE223AB6EE007AA7EE873A82
:10346000042B3FF622AFDFE803F02B2825220300D0
:10347000B1EE087A37EE877AF1EE046A77EEA66A43
:1034800066EE876AB1EE007A37EE877A27EE267A03
:10349000B0EE080A37EE800A20EE070AB0EE007A96
:1034A00077EE877A27EE800A1DF006FBFAE5B7EE85
:1034B000007AE1E7F7EE006AE4E7B7EE007AE7E7C3
:1034C000B7EE000AEAE7B0EE430A1DF0F5FAB4F1F0
:1034D000B94F30EE620A24D2C2EE836A5FED4C5AD5
:1034E0001FED4C6A66EEA67AB6EE007AA7EEA56AE4
:1034F0005FED4F5AE6EE275A1FED506AA5EEA76A18
:103500005FED515AE6EE275A1FED526AA5EEA76A03
:1035100033EE477A1FED543AA6EE263AA7EE003A6C
:10352000C3E623EE003AC0E61FED583AC0E61FEDB1
:10353000593A1CE5B4F17E5FF9D0B4F1804FF6D072
:103540001FED5E2A63E500BF7FB510EE105A834A77
:1035500025F000439342044605D8002380ED000A7D
:103560004360002022E07E4A93423AD825F000438F
:10357000002DDFED7C7A7C4A23F00F0318DD9342A7
:1035800030EE670A09BFDFED797A9FED797A9FED1A
:10359000797A30EE670A70EE477A30EE670AC0ED4E
:1035A000007A30EE470A80ED010A012004B070BDB8
:1035B000934230EE270A09BFDFED6C7A9FED6C7AFB
:1035C0009FED6C7A30EE270A70EE077A30EE670ACC
:1035D000C0ED007A30EE070A80ED010A4FF0FF30AF
:1035E000E4E7654A93426DD89FED647AB0EEC00A75
:1035F000F6EE007AE0EE077AFDEEE77AF8EEE76A9B
:1036000017EE900ADFED577AA6EEE70A1F28DFEDE6
:10361000587A66EEA77A30EE677A09DC5849461E7A
:1036200025F0004251F8261022F0FF028A4207D10D
:1036300017EE102AC2F3C752C2EBD352082A02DC9B
:1036400084ED007A1BE09FED497AB0EE406AA6EE69
:10365000C76A70EE467AE6EEC77A9FED467AD6EEF6
:10366000877A36EE677A17EE102AC2F3C752C2EB9A
:10367000E353192B15DC84ED007AB0EE460A30EEE8
:10368000470A002D30EE670A84ED010A8EDAB1EEAA
:10369000477AB1EE400A84ED007A84ED010A404297
:1036A00084E79FED387AB0EE460AA6EEC70A76EEBA
:1036B000407AE6EEC77A9FED347AD6EE877A30EE1E
:1036C000677ABDE7B3F1FF4F06D330EE400A80EDD5
:1036D000010A80ED000A44E7DA15863AA3EBC253EB
:1036E00007EE903ABDEEE77ADFED286AB8EEC77ACA
:1036F00077EEC77A8DED017A67EEA67ABDEEE77AAE
:10370000B8EEC77A77EEC77A8DED027A67EEA67AC1
:10371000F5EE407AF1EE10FACDED037A19D1B5EE5F
:10372000407AF1EE10FA16D00223214601A800F0EB
:1037300089F8002DBFF63AAFD4ED007AF1EE677A42
:10374000C4ED007AD4ED017AF1EE677AC4ED017A26
:10375000A5E70323E9E70123E7E700BFD80F493FC7
:10376000E3CB1640800FC93FD00FC93F0044353727
:103770004344353708A3852E800F494384F9223FFF
:10378000805D090000A3852E32318D240000804326
:1037900010EE103A23F00043B3F1485FB7EE007A21
:1037A00004D2FDEEC07A17EE902ABAB360EE006A3A
:1037B000DFED1C5A9FED1C6A1C4AA6EEA56A9342D7
:1037C000DFED1B5AE6EE265A9FED1A6AA5EEA66AB1
:1037D000DFED195AE6EE265A9FED186AA5EEA66AA5
:1037E00060EEC00A26EE266AF6EE007AE6EE860A5B
:1037F00066EEA77A04D877EEE07A37EE670A70476C
:103800000F4A93429ABF03F17F4306EE903AF5EEDA
:10381000026A37EE667A77EEE67AECE7B0EE470AB0
:10382000704700BF4ED747ADF6740F319999993E56
:103830007CF293B4010DD037610BB6BAABAA2A3D26
:103840000000483F2DE9F04F9246033A48BF0AF185
:103850000402D7B0D2109B46551C2DB202910BF139
:10386000FF31EB0080460DF16809501A0BF1090C8D
:10387000C24F0393AAEBC50500EB0C064C4600288B
:10388000AABF3B5CDFEDC17A07EE903A00F1010080
:10389000A8BFF8EE677AB042E4EC017AEFD142AF0C
:1038A00008EB8B0309EB8B040193BE46DFEDB77A7F
:1038B00026464046F0EC016A019B36ED017A9842BB
:1038C000E6EE877AF6D101318C45EEEC017A04F10F
:1038D0000404EBD1A949DFEDAA6A9FEDAA6A531847
:1038E00009240593A300049356AB03EB840212ED65
:1038F000140A07EB840006A92246002A45DC284664
:1039000036F032FEB0EE407AB4EE000A27EE000A3E
:1039100017F014FEF2EE007AA0EE677A002DFDEEAD
:10392000C77A17EE906AF8EEE77A37EE677A3EDDEF
:1039300006AA601EC5F1080E52F8203043FA0EF1B7
:103940000E4401FA0EF1591A42F82010C5F107028F
:10395000114100293ADD002201360DF1180E1346FF
:10396000944255DC002D03DD012D62D0022D6AD07A
:1039700002292BD1B7EE000A30EE477A33B328463E
:1039800036F0F2FD37EE407A20E060EE267A013A1A
:10399000FDEEE77AF8EEE77AA7EEC60ABDEEC00ABA
:1039A000A1EC010A30ED010A37EE800AA5E705D146
:1039B000621E06A951F822100912CAE7F6EE007A33
:1039C000B4EEE77AF1EE10FA20DA0021B5EE407A93
:1039D000F1EE10FA40F08480601E00230DF1180E05
:1039E000082838DC002B56D10FA9012251F8040D0C
:1039F000B0B3049B3E1D04EB0B01601C1E4409EB9D
:103A00008101224490422DDD14466BE70221A2E79A
:103A1000DEF8000053B920B1C0F58070CEF8000088
:103A2000012001320EF1040E034699E7C0F1FF00B8
:103A3000F4E704F1FF3E06A850F82E2002F07F02C2
:103A400040F82E2094E704F1FF3E06A850F82E20FF
:103A500002F03F02F4E75EF8202001381343BFE78D
:103A60000132C3E7059B1B5C07EE903AF8EE677ADC
:103A70004446E1EC017ADFED457A8C46F4EC015ADC
:103A8000019B3CED017A9C42E5EE877AF6D1E6ECAB
:103A9000017A0130B6E7013C083D06AA52F824300D
:103AA000DBB12846B7EE000A36F05EFD9FED347AB2
:103AB000381D4FEA840800EB8400234606AD002B36
:103AC0003CDA2346002B63DBDFF8BCE0DFED2F7A26
:103AD00007EB830C0025E01A47E0013C083DDDE7D9
:103AE000039BB0EE470AA3EB0A0036F03DFD9FEDC5
:103AF000257AB4EEC70AF1EE10FA19DBDFED207A71
:103B000060EE277A06AAFDEEE77A0835F8EEE77A46
:103B1000A7EEC70AFDEEE77ABDEEC00A10EE103A36
:103B200042F8243017EE903A013442F82430B8E7D6
:103B3000BDEEC00A06AA10EE103AF6E755F82320AB
:103B400007EE902AF8EEE77A013B67EE807A20EEE6
:103B5000070A60ED017AB2E7FEEC016ABCEC017A7B
:103B600001350A2DE6EE877A01D08542F4DD56AAAA
:103B700002EB800040ED287A013BA3E7005E0900DC
:103B80000000803B00008043C85E09000000000088
:103B90002FA81FED027A00EB08032246002A17DA4D
:103BA000E1B1F1EE477A029BC3ED007ADDED2E7AAA
:103BB00077EEC77A01239C4213DA09B1F1EE677AF6
:103BC000029B06F00700C3ED017A57B0BDE8F08F05
:103BD00073ED017A013A37EE277ADFE7F0EE477AA4
:103BE000E1E7B0EC017A013377EE877AE3E700BFD3
:103BF00010EE103A23F00043B3F1485F04D2FDEE1B
:103C0000C07A17EE903A5BB320EE007ADFED157ABA
:103C10009FED156AA7EE276ADFED147AE6EE077AC4
:103C20009FED136AA7EE876ADFED127A60EE076AEE
:103C3000E6EE077A30B99FED106AA7EE276AA6EE86
:103C4000260A704767EEE67AB6EE006AE0EE867AFC
:103C5000D7EE870ADFED097AE6EEA70A30EE600AB2
:103C6000704700BFD3C92E2F342FD7B21BEF383681
:103C7000010D50B98988083CABAA2ABEABAA2A3EDE
:103C800010EE103A23F00042B2F1465FF0EE407AB7
:103C900014D2BDEEC07A17EE101A29BB431C134391
:103CA00006D1F0EEC07AB7EE007A87EE270A7047A9
:103CB000012800F09B80BFEE007AF6E74C498A426B
:103CC00012D3002B9FED4B7AB8BFF1EE407A37EE5E
:103CD000677ADFED497AB8BFF1EE600A77EEE07AF5
:103CE000DFED460A77EE877A67EEA76ADFED445A82
:103CF0009FED446A9FED445A3D4926EEA67A67EE51
:103D0000A64AA7EE256A8A42DFED405AE6EE075A38
:103D10009FED3F6AA5EE876ADFED3E5AE6EE075A51
:103D20009FED3D6AA5EE876ADFED3C5AE7EE055A46
:103D30009FED3B5AA5EE875ADFED3A5AE5EE075A5A
:103D40009FED395AA5EE875ADFED385AE5EE075A4E
:103D5000B0EE467AA5EEA67AB0EE606AA7EE246AC7
:103D60009FED337AE6EE260AE4EE870A37EEA00AE4
:103D70001DD307EE100AF8EEC76A60EE005A30EE67
:103D8000260A9B1785EE806A03F00203C3F1010344
:103D900007EE103A36EE606AB8EEC77A77EEC67A6A
:103DA000B0EE006AE7EEC66A26EE870A7047012881
:103DB0001CD010EE103A6FF30B0306EE903A76EE3D
:103DC000E77A70EEE70AFFEE007A87EE807AF7EE88
:103DD000007A17EE103A6FF30B0300EE103AE6EE9E
:103DE000807AE0EE807AA7EE870A7047704700BFBE
:103DF00040A12C3FDA0F493F682122330000000028
:103E00005FAE9BB745F4A3388453D937C8261A3A16
:103E100016696B3BA427B33C8988083E7AC0953865
:103E2000B937813948DEBE3A1F37113CD10D5D3DAF
:103E3000ABAAAA3E2DE9F04782B00646DDF828E09D
:103E40000846B4460D46002B4ED18A4214466DD921
:103E5000B2FA82F242B1C2F12003954026FA03F38E
:103E600094401D4306FA02FC260CA7B2B5FBF6F1FE
:103E70004FEA1C4306FB115543EA054301FB07F0DB
:103E8000984209D9E31801F1FF3580F00381984287
:103E900040F20081023923441B1A1FFA8CFCB3FB49
:103EA000F6F006FB10334CEA034C00FB07F36345C6
:103EB0000AD914EB0C0C00F1FF3580F0ED8063455E
:103EC00040F2EA80A444023840EA0140ACEB030C23
:103ED0000021BEF1000F04D02CFA02F30022CEE93B
:103EE000003202B0BDE8F0878B4209D9BEF1000F65
:103EF00001D0CEE900610021084602B0BDE8F0879C
:103F0000B3FA83F1174600294DD1834202D3B2425E
:103F100000F20F81B6EB070C60EB030301201D4696
:103F2000BEF1000FDDD0CEE900C5DAE7002A00F0CF
:103F300098801A46B4FA84F3002B40F0AF800B1B34
:103F4000270CA6B20121B3FBF7F54FEA1C4007FB93
:103F5000153340EA034306FB05F8984507D9E318F3
:103F600005F1FF3002D2984500F2E8800546A3EB48
:103F700008031FFA8CFCB3FBF7F007FB10334CEA85
:103F8000034C06FB00F3634508D914EB0C0C00F15D
:103F9000FF3602D2634500F2CE803046ACEB030C14
:103FA00040EA054095E7C1F120058B4022FA05FC67
:103FB0004CEA030C00FA01F426FA05F3E84002FA91
:103FC00001F943EA04084FEA1C4206FA01FAB0FB81
:103FD000F2F71FFA8CF602FB17004FEA184444EA86
:103FE000004407FB06F0A0420AD91CEB040407F1C9
:103FF000FF3380F09C80A04240F29980023F6444ED
:10400000241A1FFA88F3B4FBF2F002FB104443EACF
:10401000044300FB06F69E4209D91CEB030300F1A2
:10402000FF3480F082809E427FD90238634440EAA8
:104030000740A0FB09749B1BA3423E46A04664D3E5
:1040400061D0BEF1000F0AD0BAEB060263EB0803A1
:1040500003FA05F5CA401543CB40CEE900530021D1
:104060003FE7730843EAC1734A08190C41EA024169
:104070004FEAC67C9BB2B2FBF4F02646A046274628
:104080001F2243EA0143B1FBF4F1A3EB080341EA29
:10409000004158E72946FFE6284615E71A46C3F1CE
:1040A00020019C4026FA01F320FA01F190400343DD
:1040B000270C06FA02FCB1FBF7F0A6B207FB1015BD
:1040C000190C41EA054100FB06F58D423BD9611808
:1040D00001D28D4220D8491B0138B1FBF7F501957B
:1040E00005FB06F8019D9BB207FB151143EA01434E
:1040F000434526D2E31805F1FF31C6D24345C4D269
:10410000A91E2344C1E7BA459BD2B7EB090664EB6D
:104110000C040138A04694E7651B29440238B1FB22
:10412000F7F5019505FB06F8DCE720467FE71F461B
:1041300066E70846F4E6A44402382FE7023D23442C
:1041400015E70199A1E7491BB1FBF7F5019505FBBF
:1041500006F8C7E72DE9F0471C46436816461A796A
:104160001B6886B089460621C3F800151A4B9DF8D6
:104170003870342101FB023387F0010702228046A8
:1041800083F82D207F0154B9144DD8F804002FF086
:10419000A3F9284606B0BDE8F0473CF095BAB4F55F
:1041A000806F4FF00003A2463A4628BF4FF4806A62
:1041B00001A94046CDE902A3CDE904638DF804309E
:1041C0008DF8059000F09EFB044B98420546DCD12B
:1041D000A4EB0A045644D6E7CC6A00200000AD0BDD
:1041E000074A00231168814201D118467047013304
:1041F000082B02F10402F5D14FF0FF30704700BFE9
:1042000014600020034B53F8203013B19A68013238
:104210009A607047DC3A002038B5144B53F82040C0
:10422000ECB120792EF020FE054660792EF01CFEC0
:10423000A2790F49E37940EA450000F0030040EA23
:104240008202A0718A5C134494F908205BB2934205
:10425000E37105DBE3680133E3600023E37138BDFC
:1042600052429342FBDCE368013BF5E734600020F7
:104270004C2209002DE9F04F0546A7B08A460146B9
:1042800000204AF0FDFD09AC002841D1CDE9130022
:104290000CAA7E21284623F0E5F8A94B0F930122B2
:1042A0004023CDE9102316AB12930FAB0E93A54B11
:1042B00009940A9300260820CDE9050648F0A9FDD7
:1042C00007902046CDE903668DF8206048F061FA3A
:1042D000DFF880B2374635469DF85490B9F1000FAB
:1042E00013D0204648F055FAB9F15D0F00F09280E6
:1042F0004AD8B9F13A0F3BD8B9F11F0F14D8B9F128
:104300000A0F31D8B9F1080FE6D88F483CF0DEFD2E
:104310000121284622F06EFA43680A93002309958A
:104320000B938DF85430C5E7A9F12002D2B20123D6
:10433000934013EA0B0F40F00F81844A1340CBD116
:10434000B9F1220FE1D106939DF854100029DCD079
:10435000222940F0A480204648F01BFADDE906102F
:1043600025F0F2FD81462CE0B9F10D0FB4D0CCE779
:10437000B9F15B0FC9D100201BF0A8FF8146002DC9
:104380003AD04FF0010821E0B9F1740F70D039D85C
:10439000B9F1660F4FD0B9F16E0FB6D19DF8543018
:1043A000752BB2D1204648F0F4F96C28ADD12046E7
:1043B00048F0EFF96C28A8D1204648F0EAF94FF010
:1043C0000E09002D00F00E814FF00008604B9F4257
:1043D00040F0F580494628464AF0B5FAB8F1000F9A
:1043E0003FF47AAF049B002B40F0F780012101A835
:1043F00025F05CFB049B1D60484624F0E9FB4D461C
:10440000074669E7B9F17B0F00F0D580B9F17D0F60
:104410007FF47BAF002D3FF478AF039B002B00F0BF
:104420000081013B049A039352F82350284624F05C
:10443000CFFB074650E79DF85430612B7FF465AF02
:10444000204648F0A6F96C287FF45FAF204648F07C
:10445000A0F973287FF459AF204648F09AF96528EF
:104460007FF453AF204648F094F94FF01E09A8E7B7
:104470009DF85430722B7FF448AF204648F089F9FC
:1044800075287FF442AF204648F083F965287FF411
:104490003CAF204648F07DF94FF03E0991E75C299A
:1044A0000CD1204648F075F97528014606D86D28CC
:1044B00008D8622840D0662808BF0C2105A854F00F
:1044C00015F935E0A0F16E03072BF7D801A252F8D9
:1044D00023F000BFF5440200BD440200BD440200C9
:1044E000BD4402003D450200BD440200F944020003
:1044F000FD4402000A21E1E70921DFE74FF000084F
:104500004FF00409204648F044F940F02000A0F1A3
:1045100030025738D2B2C0B2092A88BF0246B9F178
:10452000010942EA0818EDD1414605A854F0F0F817
:10453000204648F02EF907E70821BFE70D21BDE727
:10454000281A080045C70600E5F707000110000417
:10455000400E08000020FF030023069398464946BA
:1045600005A854F0C3F89DF85490B9F12E0F17D058
:1045700009F0DF03452B13D0B9F12B0F12D0B9F19D
:104580002D0F0FD048463CF0F5FB024650B9DDE94F
:104590000610B8F1000F09D013464AF0DFFBE1E640
:1045A0004FF00108204648F0F4F8D8E743460A22C5
:1045B00027F088FBD6E6002025F030FBDEE62EB99A
:1045C000B8F1000F7FF4A1AE4E4685E631464A466B
:1045D000284649F072FE002600E7294601A84AF065
:1045E000B2F909E7BAF1000F11D0B9F1000F3FF4A9
:1045F0008CAE039B002B7FF488AE05A854F0EDF839
:10460000484627B0BDE8F08F204648F0C2F89DF834
:10461000545028463CF0C2FB0028F5D1002DE4D0D0
:1046200073E6A946BAF1000FF1D0E2E7C20713B56D
:10463000044603D5C0F3470002B010BD830707D17D
:1046400002680E4B9A4203D124F0B0FAC0B2F3E7ED
:1046500020464AF045F948B1204624F02FFAFCEEF6
:10466000C07ACDED017A9DF80400E5E7204624F0FC
:10467000AFFA5E22C18802483CF01CFC08F6070035
:104680002B010800F8B5284B1D68284B1B681A68D9
:10469000012151641B68264AD3F84465002314683D
:1046A00014B12179814230D00133082B02F1040288
:1046B000F5D1F8BD6369A069E289218AEB1A89B254
:1046C00011FA82F2301AA189B2FBF1F7C3EB03436E
:1046D00003444FF6FF7001FB17228342A16828BFF5
:1046E000034621F81230238AA2899BB2934203D257
:1046F000238A0133238214E0E3899BB20133B3FBA5
:10470000F2F102FB1133E3810BE0E379002BD1D00E
:104710002EF0AAFB637900F00100834201D0002350
:10472000E3716561A661C4E78C6F002040700020D2
:1047300014600020242B2DE9F047884601D8012B76
:1047400006D1FEF7CDFB162303600020BDE8F087FD
:10475000344E0D46294615F8014B375D17F0080712
:10476000F8D12D2C10D12C7801278D1C33F010019D
:1047700015D1302C0DD1297801F0DF01582908D14D
:104780006C78023510230AE02B2C04BF2C788D1C8A
:10479000ECE7002BF6D1302C14BF0A23082307F1D5
:1047A000004E0EF1FF3E0021BEFBF3F90E4603FB67
:1047B00019EAA4F1300CBCF1090F10D86446A342E9
:1047C0001EDDB1F1FF3F07D0B14516D301D1A2459F
:1047D00013DB06FB0346012115F8014BE9E7A4F1C1
:1047E000410CBCF1190F01D8373CE8E7A4F1610C8A
:1047F000BCF1190F04D8573CE1E74FF0FF31EBE76C
:104800004B1C05D122230360764632B930469DE722
:1048100007B17642002AF9D009B105F1FF38C2F894
:104820000080F3E7F97009002DE9F043344E864625
:104830000D46284615F8014B375D17F00807F8D1EB
:104840002D2C10D12C780127851C33F0100015D1A8
:10485000302C0DD1287800F0DF00582808D16C7872
:10486000023510230AE02B2C04BF2C78851CECE7C2
:10487000002BF6D1302C14BF0A2308234FF0FF3849
:104880000026B8FBF3F803FB08F96FEA0909304684
:10489000A4F1300CBCF1090F10D86446A3421EDD10
:1048A000B6F1FF3F07D0804516D301D1A14513DBF8
:1048B00000FB0340012615F8014BE9E7A4F1410C88
:1048C000BCF1190F01D8373CE8E7A4F1610CBCF149
:1048D000190F04D8573CE1E74FF0FF36EBE7731CA4
:1048E00006D12223CEF80030304632B9BDE8F0833D
:1048F00007B14042002AF9D006B1691E1160F5E700
:10490000F97009002DE9F74F80460D46019252F0EB
:10491000BFFAD8F80430AC4F01225A72D8F80430EC
:104920001E791C68342303FB0677002387F82E309A
:10493000EB6803F06043B3F1005F81468B4607D01C
:10494000A248D8F8043000225A7203B0BDE8F08FB4
:104950009F4BC4F8083397F82F3003F0FF0A23B1B8
:10496000BB689C48C4F80433EBE787F82F20AE46B9
:10497000BEE80F0007F10C0CACE80F00DEF80030C9
:10498000CCF8003087F830A06B78C4F888354FF445
:10499000827120464FF07AFD4FF4927120464FF01D
:1049A00075FDC4F850A5C4F840A52B78032B00F280
:1049B000B380DFE803F0729A52022B6903F0604380
:1049C000B3F1005FBCD14FF48073C4F800326B6860
:1049D000EA68C4F844254FF4A871C4F84835204665
:1049E0004FF054FD4FF4B07120464FF04FFD4FF49F
:1049F000A47120464FF04AFD01232362A360D4F83E
:104A00005031002BFBD04FF4A87120464FF03EFDF3
:104A1000AB682A69C4F84425C4F848356A4B342287
:104A200002FB06336C4A9A604FF4827308226B4F84
:104A30002978654D03291CBF0121A15034227243FE
:104A4000A918AA58002A79D08B68C4F80433634B9C
:104A50009F4200F0A880624873E76B68EA68C4F878
:104A60004425C4F848352B6903F06042B2F1005F79
:104A70007FF466AFAA68C4F834354FF48453C4F8A1
:104A80003825C4F80032504B342202FB063340F282
:104A900002229A6001232362C6E701996B68EA68E3
:104AA000C4F84425C4F848353422474B89B102FB89
:104AB00006334FF48071C4F80012474A9A604FF4ED
:104AC000A47120464FF0E2FC4FF4A473012222624D
:104AD000ACE702FB06334FF4007140F20222C4F847
:104AE00000129A604FF48273F0E76B68EA68C4F8CA
:104AF0003425C4F838354FF48053C4F80032324BB3
:104B0000342202FB063340F202229A600123236220
:104B100000224FF482738AE7314F4FF482730822E8
:104B200086E7D4F8242152B14FF4927120464FF019
:104B3000ADFC0123236263614FF4827323441A683E
:104B4000002AEED03422D4F8C434C4F8C43402FBB2
:104B50000651002281F82F208BB1224A224813F0FF
:104B6000010F08BF104613F0020F02F5803218BF84
:104B7000104613F0040F1D4B18BF1846E1E62046FF
:104B80003FF06CFA00287FF462AF1648D9E652F085
:104B90007FF9814574EB010109D2D8F8043014483B
:104BA00000225A72D1E619F57A794BF10004D8F84F
:104BB00004305A7A002AEAD19B7A042B96BF0D4A18
:104BC000084852F82300C0E6CC6A00200A00AD0B6A
:104BD00002029C010B00AD0B000204000000AD0BB3
:104BE0000400AD0B0100AD0B0000AE0B0200AE0BDC
:104BF0000700AD0BB021090008B510EE103A23F004
:104C00000042B2F17E5FF0EE405A10D308D19FED22
:104C10002F0ADFED2F7A002BB8BFB0EE670A08BD70
:104C200070EE405ADFED297A87EEA50AF7E7B2F178
:104C30007C5F11D2B2F14A5F9FED266A42D920EE25
:104C4000000AFDF7CFFCDFED247AE0EE657A75EE21
:104C5000E75A36EE650AE2E7002BB7EE000AF6EEF9
:104C6000007A14DA75EE805A25EEA70AB1EEC06A12
:104C7000FDF7B8FCDFED197AE0EE067A9FED150A34
:104C800077EE867A30EE670A30EE000AC7E730EE3C
:104C9000650A20EE270AB1EEC05AB0EE407A15EE52
:104CA000103A6FF30B0305EE903AA5EEE57A75EE38
:104CB000257A87EE276AFDF795FCA0EE056A36EEA9
:104CC000250AE1E7B0EE460AA9E700BF00000000B0
:104CD000DA0F4940DA0FC93F6821A2336821A2B335
:104CE00008B510EE103A5A00F0EE407A0FD4B7EE45
:104CF000007A70EE477ABDE8084037EEA77AA7EE53
:104D0000A77AB1EEC70A37EE800A1BF029BE23F05E
:104D10000043B3F18B4F13D2FFEE006AE0EE006A5E
:104D2000BDE80840B1EEE67AF7EE006A37EE007AA9
:104D300086EE870AB0EE007A97EE870A1BF0BCBEBB
:104D40001BF0BAFEDFED027A30EE270A08BD00BF85
:104D50001872313F30B589B0084611461A4602AB89
:104D60000193194B0093032348F0EBFA1749029D76
:104D70000C2049F043FE9DF80C30037245609DF80D
:104D800010300446EBB128460CF048F9606805AADB
:104D900040F2114122F066FB237A5B0043F00103ED
:104DA00005AA00210120079348F028FC49F0A4FD42
:104DB0000546606843F092FB1DB9217A04483CF037
:104DC0008DF8204609B030BD24220900F0640800A7
:104DD0002306080010B58EB003AB51F8044B0193C5
:104DE000194B0093013803231DF05CFF40F22F4163
:104DF000606806AA22F036FB237A5B0043F00103C9
:104E00000893039B099340F626130A93049B5B00C7
:104E100043F001030B93059B6FF0004293421FBFC9
:104E200040F2E6425B000C9243F0010314BF022102
:104E3000012106AA4FF0020018BF0D9348F0DEFBD7
:104E40000E200EB010BD00BF0C22090010B58EB0B0
:104E500003AB51F8044B0193194B00930138032322
:104E60001DF020FF40F23751606806AA22F0FAFADE
:104E7000237A5B0043F001030893039B099340F6F8
:104E800026130A93049B5B0043F001030B93059BDD
:104E90006FF0004293421FBF40F2E6425B000C926B
:104EA00043F0010314BF0221012106AA4FF00200C2
:104EB00018BF0D9348F0A2FB0E200EB010BD00BF2E
:104EC000F421090010B596B003AB51F8044B0193DF
:104ED0002D4B0093013806231DF0E4FE09AA6068FB
:104EE0004FF4A76122F0BEFA237A5B0043F001037E
:104EF0000B93039B0C93049B0D9343F676630E93E5
:104F0000059B5B0043F001030F93069B6FF000428B
:104F1000934235D05B0043F0010343F646621193A0
:104F200010920923032116AA02EB830243F2665072
:104F300042F8340C16AA02EB8300079A520042F0A2
:104F4000010240F8302C089A6FF00040824210D0E5
:104F500016A800EB830043F2365440F82C4C16A8F8
:104F600000EB8303520042F00102013143F8282C88
:104F7000C9B209AA032048F041FB0E2016B010BDAB
:104F800007230221CFE700BFC4210900F0B58BB091
:104F9000084611461A4603AB01931B4B00930723A7
:104FA00048F0CFF9DDE903600E2816D010F00302B7
:104FB00003D10168154B99420CD023F009FEC38838
:104FC000009313484FF4BF734FF4847240F285216D
:104FD0003BF070FF012143F016FC0E49182049F008
:104FE0000DFD9DF820409DF824109DF81C50069F53
:104FF000049A9DF814300573C0E901674473817306
:10500000026103750BB0F0BDC4220900F45F080013
:10501000F80A0800D464080030B58BB004466A462C
:105020004068244D40F2ED4122F01CFA00216A460E
:10503000084648F0E3FA49F05FFC002831D0606888
:105040006A4640F29F2122F00DFA42F2B6530293D3
:10505000A3685B0043F00103039344F23603049317
:10506000237B5B0043F00103059343F676730693BD
:10507000637B5B0043F00103079342F25662112306
:10508000CDE9082304216A46002048F0B7FA2369D5
:105090000E2B03D0217D586843F0A1FB60680BB054
:1050A00030BD07F0A3FFAB6A002BBFD0012021F079
:1050B000C9FCBBE7946B00202DE9F0438BB0084698
:1050C00011461A4605AB0193254B0093052348F082
:1050D00038F90522059802A921F03AFB039FA7F1B0
:1050E0001002102A03D81F4BD340DB0702D41E48FE
:1050F0003BF0ECFE069D022D04DC002D04DC1B4879
:105100003BF094FE062DFAD10798DDF80890C0B95F
:105110008046089808B123F049FD044614494FF42D
:105120008A7049F06BFC434680F80C51C0F810417E
:105130003A464946064643F089FA30460BB0BDE888
:10514000F083012202A921F003FB0028E0D003989C
:1051500040F2511210211DF049FEDDF80880D8E719
:105160006C22090001010100B20608000B050800CD
:105170009064080070B588B003AB51F8045B0193EC
:10518000184B0093013802231DF08CFD0522039873
:1051900005A921F0DDFA069CA4F11002102A03D81B
:1051A000114BD340DB0702D410483BF08FFEDDE902
:1051B000040640B9034628462246314643F046FAE3
:1051C0000E2008B070BD012205A921F0C1FA002807
:1051D000F0D0069840F2511210211DF007FE059BF9
:1051E000E9E700BF5C22090001010100B2060800E6
:1051F00010B50446084649F0CFF8022804DC002820
:1052000004DC04483BF012FE0628FAD184F80C01B5
:105210000E2010BD0B05080038B51C460846114687
:105220004FF002121DF006FD206840F2FB3153F0F2
:10523000F2F90A490446082049F0E0FB6379054683
:105240001BB940F2FB301DF01FFD20792DF0AAFDA7
:1052500020790BF085FD6C60284638BD606408003D
:1052600008B5406842F0A3FFBDE808409FED010A81
:1052700024F03EBD3333534070B5064640683C4D84
:1052800042F095FF3B4A002303212B80C2F8F01522
:105290000121C2F8F435C2F8001519461A0102F1CD
:1052A000804202F5E0420133082BC2F81415C2F81F
:1052B0001015F3D12F4C4FF49053C4F81835736880
:1052C00001265B79C4F814354FF48071C4F81035A9
:1052D0002046C4F82C56C4F830664FF0D7F84FF487
:1052E000827120464FF0D2F84FF4847120464FF07F
:1052F000CDF84FF4867120464FF0C8F84FF48A710C
:1053000020464FF0C3F82660D4F80031002BFBD0C4
:1053100018484FF480714FF0B9F801236360154CC1
:10532000D4F80431002BFBD012484FF482714FF0B7
:10533000ADF80123A360D4F81431002BFBD00D4845
:105340004FF48A714FF0A2F80023C4F80035C4F876
:105350001435C4F810352B881BB223EAE3731813F5
:1053600040EA830080B2400040F0010070BD00BF01
:1053700058700020007000401C4608B508461146D1
:105380004FF002121DF056FC40F2FB31206853F042
:1053900042F90449042049F031FB0348E9213BF07C
:1053A0004DFD00BF44640800B70B08001B2808B57A
:1053B000014604D103212DF005FD012008BD144A4A
:1053C00000231078884206D108462DF00BFD0846D0
:1053D0002DF02CFDF1E70133082B02F10102F0D191
:1053E000282901D00E2904D10A4B1B78002BE4D1C7
:1053F000EAE70D29E8D00929E6D00F29E4D00A29E7
:10540000E2D02A29E0D01529DED00020D6E700BF5F
:105410007A1F0900D47700202DE9F04F2DED088B7D
:105420008FB009AB01936D4B009305231DF03AFC3F
:10543000002109982BF07EF9002180460A982BF074
:1054400079F9044600210B982BF074F9E379012BCC
:1054500005460AD1C379012B07D1A268012A04D9D4
:105460008368012B01D99A4202D05D483BF02EFDA2
:105470006621D8F808004EF0F4FEE6692779059019
:10548000394630464EF07CFEA368A069013B00FB24
:1054900003603946B0EE40AA4EF072FE0C98EE69F9
:1054A0000E28F0EE40AA28D1297930464EF068FE49
:1054B0000D980E28F0EE408A22D1A868AB692979B0
:1054C000013803FB00604EF05BFEEB690493D8F8F3
:1054D0001C300293059BD4F81CB0DB690393B0EE3B
:1054E000409A4FF00009D8F808304B450BD8059882
:1054F0000FB0BDEC088BBDE8F08F23F0DFFAD7E7E3
:1055000023F0DCFAE1E7029898F804104EF038FE38
:10551000029AD8F81830B4EEC0AA1A44F1EE10FA84
:10552000B0EE408A029252DCF4EEC0AAF1EE10FA1C
:1055300050D4A668D4F818A02179013E0027F31BA7
:10554000012B32D80AFB07B006914EF019FE0699DE
:1055500006FB0AB0F0EE40BA4EF012FEAB69049AB8
:105560002979079103FB0720F0EE409A06934EF04D
:1055700007FE049A069B079906FB0320B0EE40BA8B
:105580004EF0FEFD38EE6B8A30EE4B0A79EEEB9A68
:1055900028EE008A88EE290A30EE0B0A039BA3EC62
:1055A000010A039309F101099DE707EB530303FB8C
:1055B0000AB0079106934EF0E3FD069B0799B4EEFF
:1055C000C80AF1EE10FAB4BF1F461E46B7E7B0EEA8
:1055D000680AE3E7B0EE490AE0E700BF6462090049
:1055E00082FC07002DE9F04F2DED048B87B003AB53
:1055F0000193504B009303231DF054FB03980021AB
:105600002BF098F88368012B044640F28C80C67911
:10561000012E02D048483BF059FC00792BF00EF9DE
:1056200081460498E5690E2857D000212BF082F8B6
:10563000C779012F834603D1A26883689A4201D0BB
:105640003E48E8E700799FED3E8A2BF0F7F8824666
:105650002846DBF81C80C847A3694046EE18F0EEE8
:10566000408AD047DBF81830B0EE409A9844A568DD
:10567000BD4211D86B1E00EE103AF6EE007A28EE0D
:10568000278AB8EE400A20EE080A07B0BDEC048B6A
:10569000BDE8F04F24F02CBB3046C847A369404614
:1056A000F0EE409A1E44D04778EEA98A30EE499A2F
:1056B000F0EE486AD9EE286ADBF8183007EE907AE7
:1056C000B8EE677A9844C6EE877A0137B0EE409A12
:1056D00038EE278AF0EE698AC9E705989FED188AA7
:1056E00023F0ECF92846B0EE409AC847A568F0EEE2
:1056F000408AB54202D828EE098ABBE732462179B2
:10570000E0694EF004FD07EE906A78EE808AB8EE0C
:10571000677A78EEC88A0136C8EE877AF0EE408A5A
:1057200038EE278AE5E7074807B0BDEC048BBDE8F3
:10573000F08F00BF4C62090079F7070082F707007D
:1057400000000000020080801E280CD03E280AD0F5
:1057500010F0010307D1820707D10068044BC31A78
:10576000584258417047012070471846704700BFA3
:1057700008F60700044B0548D3F80425002101234F
:1057800002F500422DF050BD0010014094190900AF
:10579000F0B51B288DB006460C46154672D03CD895
:1057A0000E2800F09C8004D8042840F2B580002424
:1057B00030E01028FBD115F0010206D115F00303EB
:1057C000F5D12968704A9142F1D1284648F0E4FDAC
:1057D0000122054609A9204600F024F9102E0A9F4F
:1057E0003DD12179002240201DF088FBA3686B4346
:1057F00000FB03F1E06847F02CFBA368E0606B431B
:10580000A360636803F0FF0363601DB1013DC3192A
:10581000002F34D120460DB0F0BD1D28CBD0242858
:10582000C5D1012203A9284620F092FF002860D0AC
:10583000A10712D12268554B9A420ED1012209A923
:10584000204600F0EFF801230093DDE90901DDE9CE
:10585000032346F0FBFA00285CD11E24DAE7A16896
:105860009DF82C00694300F035F9C3680446CFE782
:10587000184609993A4647F0BFFB013DC319002D70
:10588000F6D1C7E70A68424B9A4290D009A9012293
:10589000204600F0C7F806A90522284620F058FF48
:1058A0009DF82C10002240201DF028FBA168079DC8
:1058B000B5FBF0F5064629449DF82C0000F00AF9E6
:1058C0000446DDE90912C06847F096FBE0680A9BD0
:1058D000069905FB06F2184447F08EFB9AE70A6822
:1058E0002B4B9A423FF463AF2946204641F084F99E
:1058F00090E7EA0702D500203BF098FAAB0703D106
:105900002A68214B9A42F6D0284648F0E9FF002841
:10591000A3D0F0E73E247DE7012209A9204600F04C
:1059200081F8012206A9284620F012FF002894D011
:105930000B9A012A21D05A2A21DC20320146089BE9
:10594000012B1ED05A2B01DC203301469342D2D1C9
:1059500023F00203642BCED0022E01D00029CAD03E
:10596000079B0093DDE90912069B304649F03DFB99
:10597000002814BF3E241E244CE74222DDE700210C
:10598000DDE74223E0E700BF08F60700281A080019
:1059900078190800F0B5012885B007460E4608D0F2
:1059A0008B0727D10B681C4A934202D01B4A9342B3
:1059B00020D1012201A9304620F0CAFED0B13946DB
:1059C000002240201DF09AFA029BB3FBF0F100FB8D
:1059D00001F5AB4202D012483BF078FA384600F0AD
:1059E00079F8019904462A46C06847F005FB20462D
:1059F00005B0F0BD304624F03BF858B145102946BB
:105A0000384600F067F82B463A463146044641F0E6
:105A100039F9ECE70546F2E7780E0800281A080085
:105A20006901080070B50D460179044601F07F0157
:105A30001646402000221DF061FAE3682B60A26840
:105A400042436A60227902F07F02AA602168094A13
:105A500091420BD194F90420002A01DBB20707D44C
:105A60006268C2F3172200FB02332B60002070BD76
:105A70000120FCE778190800074BC1E9003000233A
:105A8000C1E90233054B02689A4202BF4368C3F37F
:105A900017238B6008467047882108007819080092
:105AA00038B50D461C4611462846094A1DF0C2F875
:105AB000206825F04DFA012D007804D1BDE838406A
:105AC000002100F007B86168BDE83840FFF762BF09
:105AD000040002007828F8B505460E4602D10F48AA
:105AE0003BF0F4F90022014640201DF007FA0C4B70
:105AF0000C490746012D18BF1946102048F07EFFBB
:105B00000571436803F0FF030446C0E9013606FB54
:105B100007F047F09BF9E0602046F8BDC30108009C
:105B2000FC200800281A080070B50A79012A0546E9
:105B30000C460DD1184949F087F9D4E902212846CD
:105B400026F0DEFF28461549BDE8704049F07CB9D3
:105B5000134949F088F9A368002BF3D0114928466E
:105B600049F072F90026A368B34204D80E492846CA
:105B700049F06AF9E6E71EB10C49284649F064F994
:105B80003246E16820791DF093FA01220146284649
:105B900024F04AFB0136E6E7829107006B9A070082
:105BA0008E9107009991070063E50700BEE60700A4
:105BB0002DE9F04F044687B00D4616460AB9002578
:105BC000D0E011F003078068DFF82CA240F0DF80FE
:105BD0000B68814A934240F0DA806A4649F093FAB2
:105BE00010B97E483BF022F92179042E01F07F01A3
:105BF0003A464FF0400000F096801DF07FF916F015
:105C00000302054655D131688B7B002B42D001EB56
:105C100083031869724B98423CD13179402001F0DE
:105C20007F011DF06BF9A84202D06E483BF04EF99F
:105C300033685345D6E9028B38D17368C3F317290B
:105C400005FB09F9DDE900062368E768361A5345C4
:105C5000A8EB06062FD194F90430002BAFDA002E02
:105C6000E3D16368C3F3172305FB037705FB08F251
:105C70000BEB090105FB007047F0E9F90199A268F7
:105C8000009B521A08EB03006A4305FB017105FBF8
:105C9000007039E0544B99420BD1012DC5D105223A
:105CA00003A9304620F054FDDDE903B84FF00009A8
:105CB000C8E74E4896E7002ED8DD6368B6EB132F91
:105CC0002FD9A16831446943384647F0C2F8636868
:105CD000E06066F31F2382466360BB4508BF8346CE
:105CE0000098A268019940443244121A6A4301FBA9
:105CF00005A105FB00A047F0AAF9009805FB08F2F2
:105D00000BEB090100FB05A047F0A1F96368C6EBA6
:105D1000132262F31F236360A3683344A3600E253C
:105D200020E0BA46DCE71DF0E9F82168009B514508
:105D300006461BD1B3F1807F03DB2D492D4852F07D
:105D4000D2FA102048F05AFE054694E80F0085E884
:105D50000F00009A02EB112363F31F216960019B7E
:105D60009B1AAB60284607B0BDE8F08F01992079F7
:105D7000C91AFFF7AFFEDDE90032E168D21A054625
:105D8000724306FB0311C06847F036F9EAE70023C7
:105D90002A460146206820F0F9FC23685345024654
:105DA00020790ED16368042E02EB13220BD0030678
:105DB0007FF505AFE168334600F07F001DF056FC2B
:105DC000ADE7042EF6D1E16800F07F0007B0BDE832
:105DD000F04F1DF06DB900BFA8180800DEF90700EC
:105DE000B15B0200F7FB0700780E080034020800E0
:105DF00064FB07007C1408007819080010EE102AD4
:105E000008B522F00043B3F17E5FB0EE406A12D3D2
:105E100019BF76EE467A9FED1F7ADFED1F7A9FED70
:105E20001F7A12BF87EE276AE0EE077AB0EE676A44
:105E3000B0EE460A08BDB3F17C5F0BD2A3F50003B8
:105E4000B3F1645FF4D320EE000AFCF7CBFBA0EEC5
:105E5000066AEDE7B0EEC06AB7EE000A30EE460A19
:105E6000F6EE007A20EE270AB1EEC06AFCF7BAFB24
:105E7000002ADFED0B7AA0EE066AB0EE007AE6EEBD
:105E8000077A9FED066A36EE676AB8BFB1EE466ADA
:105E9000CEE700BF0000000000008003DA0FC93F1A
:105EA0006821A2B31FB58DED010A019B23F00042CA
:105EB000B2F18B4F00EE102A4FEAD3700AD31AF0DA
:105EC000FBFDDFED1E7A30EE270A08B1B1EE400A85
:105ED00005B000BD5B0014D5B7EE007AF0EE476A5E
:105EE000E0EE006AF1EEE67A77EE807AC7EE276A96
:105EF000F0EE007AE0EE276AB0EE660A1AF0DCFDFA
:105F0000E3E7B2F1665F10D320EE007AF7EE006AA5
:105F100037EE266AF1EEC67A77EEA67AC7EE276AE2
:105F200036EE800A1AF01CFDCFE7DFED057A70EE41
:105F3000277ACDED037A039BC7E700BF1872313F84
:105F40000000807B08B5044B1A68044B9A4202D0CB
:105F50000D2033F073FD08BD009C0320EF2978016C
:105F60001FB50446E0B10E281AD04FF01023007977
:105F7000D3F80C32DB0703D5A0F10903012B02D9BA
:105F800030F004F960B940F2C713039301A9204629
:105F900003AB02AA16F0AAFE039902483AF09EFF4C
:105FA00004B010BD710B0800F4EE400AF1EE10FAD7
:105FB00010B5F0EE407A04D770EE207AB0EE670AA2
:105FC00010BD10EE902AB2F17E5F03D1BDE8104003
:105FD00000F082B810EE103A940F04F0020444EA84
:105FE000D37433F0004308D1022C59D09FED317A9D
:105FF000032C08BFF0EE477AE0E732F0004209D107
:10600000DFED2D7A9FED2D7A14F0010F08BFF0EE31
:10601000477AD3E7B2F1FF4F10D1B3F1FF4F04F14C
:10602000FF3407D1022C3ED8254B03EB8403D3ED7C
:10603000007AC3E7022C39D8224BF6E702F150610F
:106040009942DDD3B3F1FF4FDAD0A10703D503F1B5
:10605000506393420CD387EEA00AB0EEC00A00F062
:106060003BF8012CF0EE407A04D1F1EE407AA5E73E
:10607000DFED157A022C0AD0002C9FD09FED137A09
:1060800077EE877A9FED127A77EEC77A96E79FEDE3
:106090000F7A77EE877A9FED0E7A77EE677A8DE743
:1060A000DFED0B7A8AE7DFED0B7A87E7DFED067A23
:1060B00084E700BFDB0F49C0DB0FC9BFDB0FC93F5F
:1060C000545D0900485D0900000000002EBDBB338F
:1060D000DB0F4940DB0F493F10EE102A22F000434E
:1060E000B3F1994F82B04FEAD2700ED3B4EE400AAA
:1060F000F1EE10FA07D69FED410ADFED417A002854
:1061000018BFB0EE670A02B070473E498B420BD809
:10611000B3F1665F5AD212F0FF4FF4D160EE007A0D
:10612000CDED017A019BEEE7374A9342F0EEC07A5B
:1061300037D8A2F5D002934229D8F0EE006ABFEE1C
:10614000007AA7EEA67A002377EEA67A87EE270AD2
:106150005A1C60EE006A9FED2D6ADFED2D7ADFEDAF
:106160002D5A26EEA67AE7EE067A9FED2B6AA7EE69
:10617000876ADFED2A7AE7EE257A67EE877AE6EE20
:10618000267A67EE807A24D130EE670ABBE7B7EE55
:10619000007A77EEC76A77EE877A012386EEA70A40
:1061A000D6E71F4A93420BD8F7EE086AB7EE007A9B
:1061B000A7EEA67A022337EEE66A86EE070AC7E75D
:1061C000BFEE007A87EE270A0323C1E74FF0FF33C3
:1061D000BEE7144A144902EB830201EB830393EDFB
:1061E000007A77EEC77A37EEC00AD2ED007A37EE42
:1061F000C00A002887D0B1EE400A84E7DA0FC93F11
:10620000DA0FC9BFFFFFDF3EFFFF973F25AC7C3DA4
:106210000DF5113E4712DABDA9AAAA3E98CA4CBE96
:10622000FFFF1B40705D0900605D09002DE9F84F1C
:10623000D1F800800128064640468CBF01F1040BCE
:106240004FF0000B0F46914623F02EFB30B940462D
:1062500022F0BEFCC18827483AF02CFE06F1FF3A36
:10626000B9F1000F2DD0D9F80050C5F3DC051AEBB9
:10627000050404D02C44A00046F0CBFD04460022C7
:10628000924520D804EB86000022954221D11A4E77
:10629000DFF868903168D9F800000131090146F053
:1062A000D8FD3368C9F800005A1C32601A0100EBAF
:1062B000031340F802A0C3E90158DC603868BDE868
:1062C000F88F4D46D3E75BF8223044F82230013294
:1062D000D6E7D9F80830083053F8323040F80C3C93
:1062E000D9F8083003EBC20301325B6840F8083C80
:1062F000CBE700BF900A0800646100205C610020C9
:10630000F0B50023DFF838E00C4E19460E27DEF812
:106310000020934201D30E20F0BD346804EB031239
:106320004FEA031C9568854208BF44F80C1003F13E
:10633000010304BFC2E90117D160E8E75C610020F6
:106340006461002038B590F82330FF2B044629D033
:10635000154B01225A600022C3F8002590F8263020
:106360009B0707D590F821002CF01CFD94F8220023
:106370002CF018FDFF2594F8210033F075FB94F8FC
:10638000220084F8215033F06FFB94F8230084F846
:10639000225033F069FB054B84F8235000221A6029
:1063A00037F068FC0E2038BD00500240FC69002028
:1063B0002DE9F04788B0084611461A4602AB019312
:1063C000434B0093062346F0BCFF9DF81C700298D7
:1063D00040F261210FB33CF051FF40F22E510546CF
:1063E00003983CF04BFF40F2B3210446049852F06E
:1063F00012F940F297318246059852F014F9354966
:106400008046282048F001FB0646B8F1000F0DD069
:10641000314840F297313AF011FD52F0FCF840F269
:106420002E510546039852F0F6F8DCE72B4BD3F8D3
:106430000080B8F1000F02D029483AF021FD186021
:1064400028799DF818900AF08BFC20790AF088FCD6
:106450009AF804000AF084FC96F8263067F34103AA
:1064600086F826301F4B2A7986F82120C3F8642548
:10647000227986F82220C3F868259AF8042086F845
:106480002320C3F8702507B3287941462CF09AFCE5
:10649000207941462CF096FC0122124B0121C3F8D1
:1064A00004254F400022C3F80825C3F80C15C3F893
:1064B0001075C3F81C15C3F82025C3F8249537F0D0
:1064C000F3FB304608B0BDE8F0873A46E5E700BF89
:1064D000AC23090014640800B70B0800FC69002015
:1064E000150808000050024010B5044690F823003B
:1064F00041F057FE20460AF083FE10B905483AF0F5
:10650000BFFC94F8263043F0200384F826300E2098
:1065100010BD00BFD50508002DE9F04F0D4685B030
:1065200055F8044B064694F82300174641F039FE0F
:1065300002AB0193664B0093701E294602233A4634
:106540001CF0B0FB2046029D9DF80C600AF058FE3E
:1065500058B1604A0123536094F8263043F0080391
:1065600084F826302023C2F80833284625F03AFE66
:1065700094F82630656066F3861384F826302A7B0B
:106580006968544FD20884F82520AB7BE87B6D7B8B
:1065900084F82450003B18BF0123DB0143EA0023A9
:1065A000E08C013A03F4C07320F4C07018BF0122DC
:1065B0000343E384C7F81C2594F824305A1E534241
:1065C0005341C7F8283594F8263013F002033DD024
:1065D0000B4694F82500638394F8243048435843CD
:1065E00000014FF47A73B0FBF3F0033020F00300A6
:1065F00080B2208346F02AFCA060208B46F026FC67
:10660000E060606841F088FA0023C4E9043384F84C
:10661000203094F8263023F03C0343F00403204656
:1066200084F8263017F084F8228B2A4B9208C3F89E
:1066300050252022C3F804230122C3F800251A6044
:1066400017F058F80E2005B0BDE8F08F2248DFF8AB
:106650009090B7EE007A9E4698461E46D7F81C25C5
:10666000012A01D182793AB307EE901A1B4AD0F879
:1066700000B0B0F904C099FBFCFCF8EE676A02F1C7
:10668000580A55689CFBF5F507EE905AF8EEE77A44
:1066900076EEE77AF0EEE77A87EEA66AB4EEC76A9E
:1066A000F1EE10FA05D5D2F800E0B0EE467A2B46AE
:1066B000D84608329245E4D10136092E00F108008F
:1066C000CCD1044AC2F81885C2F814E581E700BFAE
:1066D0009C2309000050024054230900FC220900B9
:1066E0000048E80110B5044690F8230041F059FD38
:1066F000064A0123536094F8263043F0080384F8D7
:1067000026302023C2F808330E2010BD005002406E
:1067100038B5084B1B6800220446C3F80025FF2546
:10672000007933F0A1F96079257133F09DF9657135
:106730000E2038BD142100202DE9F0432DED028BF1
:106740008BB0084611461A4603AB0193444B0093A5
:10675000072346F0F6FD40F28D21039851F05BFFD0
:106760004FF42D718046049851F055FF059E002E80
:10677000074604DC4FF48E6101201CF025FB069DCA
:10678000082D06D0102D04D040F2622135483AF091
:10679000A5FB089BA3F10802F72A01D85B0702D0EA
:1067A00040F2EB31F2E709989DF81C9020B322F0FB
:1067B00085F9B0EE408A40F2AB4201210020B0EEF4
:1067C000480A46F0D3FD2849082048F01EF904463F
:1067D00098F804000AF0C4FA38790AF0C1FA84F88B
:1067E000069098F8042022713B796371B6F57A5FC0
:1067F00005D01E483AF06AFB9FED1D8ADBE7EDB23B
:10680000102D01D01B48F5E71B4BDFED1C7A1B68F0
:106810001B49C3F840256279C3F8442528EE278A2E
:106820004FF00462C3F804250022C3F82025FCEED3
:10683000C87A2822C3F81825C3F81C250122C3F8FA
:10684000002517EE900AC3F86015C3F864251A6096
:1068500020F03AF820460BB0BDEC028BBDE8F08387
:10686000DC230900020B0800F8630800F2F90700B6
:10687000AE47E13D07FA07001421002000007A44EA
:10688000E86100202DE9FF411446074600790D46D6
:1068900041F081FC01A9204622F062F948B9204666
:1068A00022F096F95E22C388344840F283313AF0F0
:1068B00001FB019C40F283320021204646F080FD1E
:1068C000AB0706D12A682E4B9A4202D12D483AF0E6
:1068D000ADFA062201A928461FF03AFF9DF80C10D8
:1068E000029D002240201CF009FBB5FBF0F5A542FB
:1068F00002D225483AF0EAFA039B482B01D02348FC
:10690000F8E7DFF89480019DD8F800300122C3F841
:106910000825C3F86055C3F864451D4B4FF4485033
:1069200043F001039847D8F800300022C3F808214B
:10693000184AC3F8602501222E46C3F86425D8F80A
:106940000030D3F808316BB105EB4405B5420CD1EA
:10695000BB7983B124F00104640044F0010004B069
:10696000BDE8F08106F042FBE9E73388A3F5004378
:1069700026F8023BEAE724F00304EDE7EF0A0800FB
:106980006C1709008E080800190808007CFF070032
:1069900020240900E8610020142100202DE9F04F97
:1069A0002DED028B89B0426B079390F83030B3FA2B
:1069B00083F35B0980F830300A33044650F82370C3
:1069C000037BDB08B2FBF3F8436C0193836C5B0839
:1069D0000493C36C0393BA46B8F1000F0FD194F837
:1069E0003030079A0A33012054F823301360626B69
:1069F000149B1A6009B0BDEC028BBDE8F08FE36B0D
:106A00004BBB94F8413033B994F84030ABB1606D72
:106A100098B141F081F8606D60B104F13C0204F17D
:106A2000380141F02EF802280AD100236365E363A0
:106A300084F84130617B0D0216E000236365EAE7CC
:106A4000227BE36BD208B3FBF2F3E363431E5842AD
:106A5000584184F84100617B636D0D02002BE9D041
:106A6000E36B9D4228BF1D46454528BF45466068EB
:106A7000B5FBF1F189B234F067FC04F1200037F086
:106A800061FCF7EE007AB4EEE70AF1EE10FA30DDC1
:106A900004F1200037F056FCFDEEC07A17EE909A14
:106AA000F7EE000A04F124009FED5F0A50F0C7FAE8
:106AB00004F11400F0EE408A37F044FCD4ED067A7D
:106AC00094ED077A77EEC07AF0EEE77AF4EEC77AC3
:106AD000F1EE10FA02DB20460AF006F9616D11BBF7
:106AE000A37B227B43B1D2086A43384646F0C5FAFD
:106AF0000BE04FF00109D3E7102A0FD107EB450255
:106B00003B464FF40041934205D1A8EB050807EB43
:106B10004507AA4460E723F8021BF4E7D2086A435A
:106B200080215046E2E74FEAC933A3F5DA43603BE0
:106B30006FF0704292FBF3F30593A36B029309F19C
:106B4000FF334FF0000B06935D45227B08D1A36B0A
:106B5000D20805FB0233A363E36B5B1BE363D4E75B
:106B6000102A029B3DD133F91B60226D019B511C01
:106B7000B9F1010F216523F8126049D0069A049BF0
:106B8000B3FBF2FC226D00210CF1FF3C013A0846F8
:106B9000894530DC059937F0F1FD0090DDED007A94
:106BA000F8EEE77A022167EEA87AFDEEE77A17EEB3
:106BB000900A304437F0E2FD227B102A2AD127F8D0
:106BC0001B00A27B1AB980F4004027F81B00039B2E
:106BD000226DB2EB530F24BF002323650BF1010B91
:106BE000B2E7A27B13F90B60002ABED186F07F06C4
:106BF000F64376B2B9E7002ABCBF039B02EB53020F
:106C0000019B33F912E001317044A2EB0C02BFE7A3
:106C10000096C3E7A27B12B10AF80B00D7E780F019
:106C20007F00C043F8E700BF000000002DE9F04FEF
:106C30002DED028B8DB0084611461A4603AB019329
:106C40005E4B0093092346F07CFB4FF467734FF4CF
:106C50007A620121039846F0A7FB40F2832306469F
:106C600002220B98012146F09FFBDDF820B0BBF11A
:106C7000000F824604DC4FF48E6101201CF0A4F862
:106C8000099D082D04D0102D02D04D483AF01EF970
:106C90004C49582047F0B2FE0446DDE906809DF8D5
:106CA000283025730025DDE90497A37384F80DA02F
:106CB000C4F804B0E573A060606346F0C7F8626B87
:106CC000A06218B960736064E0620BE0294646F088
:106CD000D4F9606B46F0BAF8626BE06228B9607371
:106CE0006064A06210463AF077F8294646F0C5F98C
:106CF00035486565012384F83030002F18BF3846C9
:106D000040F2215204F12001C4E90E55A4F840508C
:106D100037F0F0FA2D489FED2E8A04F1140740F267
:106D2000C3223946B9F1000F18BF484637F0E2FADE
:106D3000284840F2B13204F12401B8F1000F18BF25
:106D4000404637F0D7FAD4ED017A637B2661B8EE7E
:106D5000677A5B00C7EE087A07EE106AB8EE477AEA
:106D600067EE877A07EE103AB8EEC77A67EE877A51
:106D7000FCEEE77A17EE900AC4ED137A46F066F857
:106D8000E26C606410B96073A0629DE7294646F02A
:106D900074F9D4ED017AF8EE677A384688EE277AEE
:106DA00084ED077A37F0CEFA204609F09DFF2046A1
:106DB00025650DB0BDEC028BBDE8F08F58240900AD
:106DC000B701080078630800020000C00200C8C2D2
:106DD00000007A44020080BFF0B50D4685B055F83A
:106DE000044B0646607B174640F046FE02AB01931B
:106DF000154B00933A4602232946701E1BF052FFA2
:106E0000029D9DF80C6029460022204606F06EF88F
:106E10002846656584F8406040F07EFE04F13C023F
:106E2000606D04F1380140F02CFE227BE36BD20848
:106E3000B3FBF2F3E363431E5842584184F8410028
:106E4000204605B0F0BD00BF482409002DE9F04FF1
:106E50002DED068B8FB0D0F854A00D930B1E0A9326
:106E600014BF134600230B9390F84030426CDFEDC3
:106E7000ACAAB3FA83F35B0980F840300E330446C2
:106E800050F823300193037BDB08B2FBF3F302934A
:106E9000019B0493029B002B00F09680E36C4BBB9C
:106EA00094F8513033B994F85030ABB1E06E98B1EA
:106EB00040F032FEE06E60B104F14C0204F1480192
:106EC00040F0DFFD02280AD10023E366E36484F882
:106ED0005130617B0B0216E00023E366EAE7227B78
:106EE000E36CD208B3FBF2F3E364431E584258410B
:106EF00084F85100617BE26E0B02002AE9D0E26C5B
:106F0000934228BF1346029A60689A4228BF1A46E5
:106F1000B2FBF1F189B2934634F016FAF7EE000AAB
:106F200004F134009FED7F0A50F089F8F7EE000A73
:106F300004F1200070EE008A9FED7A0A50F07FF88D
:106F400004F11400B0EE409A37F0FCF9D4ED067A63
:106F500094ED077A77EEC07AF0EEE77AF4EEC77A2E
:106F6000F1EE10FA02DB204632F0AAFC04F1240311
:106F70001846069340F08BFBA36D627BE16E5B08C5
:106F80000393E36D013AD3405B080793002940F077
:106F9000DD80F4EEEA8AF1EE10FA2BD8A37B227B97
:106FA00033B1029B0198D2085A4346F066F80BE0D1
:106FB000102A19D14FF40043019A22F8023B0192A2
:106FC000029A013A0292F7D194F840300D9A0E33AA
:106FD000012054F823301360626C1E9B1A600FB0BE
:106FE000BDEC068BBDE8F08F029B0498D2085A4393
:106FF0008021DAE70E46F7EE009A0A9B002B4FD06D
:107000000B9B012B52D1079B002B4FD0656E9846EE
:1070100094F85270B8F1000218BF0122002F67D017
:1070200008EB1523A76E3AF913302F4408EE103AF7
:107030003B0A4FEA152B0593059B5B453AD8F4EEC6
:10704000E89AF1EE10FAB8EEC88AD4BFF0EE697A89
:10705000F0EE687A67EE887A227BFDEEE77A102AF6
:1070600017EE903A60D1019A22F81630A27B22B92D
:10707000019A83F4004322F8163094F85230002B22
:107080005DD0039B1B02B7FBF3F503FB1575B8F14D
:10709000000F59D06566029B0136B342ADD893E725
:1070A000627BB6FBF2F302FB1363AAE7256E4FF097
:1070B0000008ADE7039BBBFBF3F903FB19B9C1441F
:1070C000617B3AF919300698089207EE903AF8EE8B
:1070D000E77A0BF1010B67EE897AFDEEE77A17EE9E
:1070E000903A1BB240F082FA089A2AF81900A3E7F6
:1070F00005EB0809617B3AF91930069808EE103A59
:10710000F8EEC87A013567EE897AFDEEE77A17EE78
:10711000903A1BB240F06AFA2AF819008FE700BFD4
:107120000AD7233C00000000049A9355A27B002A52
:10713000A3D1049A83F07F03DB4393559DE7039B20
:107140009D4228BF0025A2E72566A4E7F4EEEA8A5F
:10715000A36C0893F1EE10FA40F288800026B34544
:107160006ED0227B089B102A40F0828033F91630C3
:107170000A99002900F086800B99012940F0888047
:107180000799002900F08480656E0591059994F8AF
:107190005270003907EE903A18BF0121B8EEE78A25
:1071A0000991002F77D0059BA76E03EB15232F4481
:1071B0003AF91330102A09EE903A4FEA17234FEAB2
:1071C00015280C9300F0A7800C9B434540F2A68045
:1071D000039BB8FBF3F903FB1989059B617B0698B8
:1071E0009944F0EE487A3AF9193007EE103AB8EEC1
:1071F000C77A6FF07F02E7EE097A08F10108FDEE29
:10720000E77A17EE903A9342B8BF13467F2B099A5C
:10721000A8BF7F2340F0EAF940B22AF81900D3E76B
:10722000227B102A089A0BBF0199049932F9132086
:10723000D2560CBF21F81320CA5401339B45EFD11D
:10724000029B227BA3EB0B030293019B03EB4B03FB
:107250000193049B5B440493A36CD2080BFB0233A1
:10726000A364E36CA3EB0B03E36413E60023E5E7FD
:10727000A17B9B5700297FF47BAF83F07F03DB4327
:107280005BB275E7607BB6FBF0F100FB116174E760
:10729000256E002179E7059B05EB0308F0EE487A9F
:1072A0003AF9183009EE903AB8EEE97A102AE7EE8A
:1072B000097AFDEEE77A17EE900A6CD000F3070327
:1072C000099A617B069840F091F9013540B26DE072
:1072D000039BB8FBF3F903FB1989059B9944B0EEB6
:1072E000487A3AF9193007EE903AF8EEE77A41F623
:1072F000EF31A7EE897A08F10108FDEEC77A17EEA3
:10730000900A37F03BFA099A617B0346069840F0F1
:107310006DF92AF819000C9B4345D9D8B0EE007AD4
:1073200037EE687AF7EE007AF4EEC77AF1EE10FAEB
:10733000F4EEE87AD8BFB0EE677AF8EEE99AF1EEAB
:1073400010FAC8BFF0EE687A67EEA97A41F6EF311D
:10735000E7EE087AFDEEE77A17EE900A37F00EFABC
:10736000237B102B25D1019B23F81600A37B23B987
:10737000019B80F4004023F8160094F852300BB3C0
:10738000039B1B02B7FBF3F503FB1575059BF3B1DC
:1073900065660136E3E641F6EF3137F0EFF9099A19
:1073A000617B0346069840F021F901352AF8180060
:1073B000B4E7A37B13B1049B9855DEE780F07F0010
:1073C000C043F8E7039B9D4228BF0025DEE7256602
:1073D000DFE700BF2DE9F04F2DED028B8FB008469F
:1073E00011461A4603AB0193614B00930B2345F002
:1073F000A8FF4FF467734FF47A620121039845F0B8
:10740000D3FF40F2832308EE900A02220C98012158
:1074100045F0CAFF099E002E054604DC4FF48E613C
:1074200001201BF0D1FCDDF828B0BBF1080F05D01E
:10743000BBF1100F02D04F4839F048FD4E49702083
:1074400047F0DCFA04469DF8341008989DF82C208B
:1074500084F85210DDE906A865730025DDE904977C
:1074600084F80CB0A2736660E573A060606445F0B8
:10747000EDFCA06328B9204641F015F9606C39F0A5
:10748000ABFC626C294645F0F8FD606C45F0DEFC13
:10749000E0630028EFD0626C9FED388A294645F002
:1074A000ECFD012384F84030627BE566514604F12F
:1074B0002400C4E91255A4F8505001F081FC304872
:1074C0004FF42E72002F18BF384604F1200136F019
:1074D00011FF2C4804F1140740F2C3223946B9F1D8
:1074E000000F18BF484636F005FF274840F2B1327A
:1074F00004F13401B8F1000F18BF404636F0FAFE2F
:10750000D4ED017A637BC4ED048AB8EE677AC7EEE6
:10751000087AB8EE687A67EE877AFCEEE77A17EEBB
:10752000900A58434000E06545F090FC606520B942
:10753000204641F0B8F8E06DA1E7E26D294645F03C
:107540009CFDD4ED017AF8EE677A384688EE277A0A
:1075500084ED077A36F0F6FE204632F0B1F9204687
:10756000C4E918550FB0BDEC028BBDE8F08F00BF29
:1075700028260900B70108009863080000007A4433
:107580003233B3BF0200FAC3020000BFF0B50D46AC
:1075900085B055F8044B0646607B174640F06CFA00
:1075A00002AB0193154B00933A4602232946701E05
:1075B0001BF078FB029D9DF80C60294600222046B6
:1075C00005F094FC2846E56684F8506040F0A4FA83
:1075D00004F14C02E06E04F1480140F052FA227BC3
:1075E000E36CD208B3FBF2F3E364431E5842584104
:1075F00084F85100204605B0F0BD00BF18260900F0
:107600002DE9F04F2DED068B8FB0C76B0B930B1E42
:10761000039390F8383090F80D80D0F850A0B3FA6A
:1076200083F34FEA531380F8383003F10C03044618
:1076300050F82390037B08BF0022DB08B7FBF3F769
:10764000002948D0012A46D1A8F102014B424B4102
:1076500008934FEA08230793DFED819ACDF8049051
:107660004FEA4A030A93002F00F0E580636C002B79
:1076700047D194F8493033B994F848306BB3A06ED1
:1076800058B340F049FAA06E50BBB7FBF8F1606800
:1076900089B233F059FE04F1100036F053FE04F1C4
:1076A000140036F04FFE04F1180036F04BFE04F1E2
:1076B0001C0036F047FE04F1200036F043FEA37BA9
:1076C000227B002B00F0AF80D2087A43002148468D
:1076D00045F0D3FCAFE00023BAE70023A366D2E76E
:1076E00004F1440204F1400140F0CBF9227B636CC9
:1076F000D208B3FBF2F3421E50425041636484F857
:107700004900A36E6068002BBFD0079A636C9FEDA1
:10771000558A934228BF1346BB4294BF04930497F3
:10772000236C0593049BB3FBF8F189B233F00CFE94
:10773000D4ED097A94ED0A0AF8EE670A04F1100014
:107740004FF07DFCF3EE040AB0EE409A04F1140011
:10775000B0EE690A4FF073FCF7EE000AB0EE40AAF3
:1077600004F11800B0EE690A4FF069FCDFED3E0A43
:10777000F0EE40AA04F11C009FED3C0A4FF05FFCC4
:1077800004F1200060EE088AF7EE000AB0EE690A04
:107790004FF055FCD4ED097AF8EE677AB0EE496AFD
:1077A00077EEC97A20EE088AA7EEAA6A204600265C
:1077B000B0EE490A13F0F2FDB0EE460A06902046FC
:1077C00013F0ECFDD4ED017A069BB8EE677AC31A8C
:1077D000CAEE077A0993B6EE007AB4EEE77AF1EED4
:1077E00010FAD8BFF0EE477A9FED217A67EE877ADC
:1077F000FDEEE88AFCEEE77ABDEEC88AC4ED197AA0
:10780000049B9E4236D1019B227B33440193236C1F
:10781000D20806FB02332364636C9B1BBF1B09EB7E
:10782000460963641FE7102A15D14FF40043013F56
:1078300029F8023BFBD194F838300B9A0C33012025
:1078400054F823301360E26B1E9B1A600FB0BDEC3E
:10785000068BBDE8F08FD20801987A43802137E784
:107860000000000000FEFF463333733F333373BF25
:107870000000804F039B002B78D1B6FBF8F008FB8B
:107880001060431E58425841237B102B059B6FD13B
:1078900033F91650636E04EB8002D16D1944434BEB
:1078A000D165A3EBD13C4FEAD13E099B3EEA210EC4
:1078B00028BFE646A3FB0E1C090C069B41EA0C41BF
:1078C00019440028E36C0A9808BF00200344506D57
:1078D000029050441FFA81FCA0EB11418A4598BFE9
:1078E000A1EB0A0100294CD0481E33F911B033F93D
:1078F00010100C93A1EB0B0118EE903A0CFB01F168
:107900000BEB214B0BFB03F00F210D9236F0DCFF4C
:107910000021284436F0D8FF029A0C9B23F812006D
:10792000531C0D9A534508BF0023536518EE103AB7
:10793000B3F5A47F0DDD0BFB03F00F2136F0C4FF80
:1079400094F82C3003B3281A41F6EF3136F016FFC5
:107950000546237B102B19D129F81650A37B1BB9A0
:1079600085F4004529F81650013649E708988BE759
:107970009D57A37B002B8DD185F07F05ED436DB224
:1079800088E70AF1FF30B0E72844DDE76FF07F03B6
:107990009D42B8BF1D46A27B7F2DA8BF7F2512B197
:1079A000019B9D55E0E75D40FAE700BFFFFF010046
:1079B0002DE9F04F2DED028B91B0084611461A4685
:1079C00004AB0193674B00930C2345F0BAFC4FF4D2
:1079D000677364220121049845F0E6FC40F283239A
:1079E00008EE100A02220F98012145F0DDFC0C9DE3
:1079F0000290002D04DC4FF48E6101201BF0E4F9AD
:107A00000D9B082B04D0102B02D0574839F05EFA9A
:107A1000564903936C2046F0F1FF0446039B0B98F4
:107A2000099E9DF828B09DF83810E063DDE90787CE
:107A3000DDE905A923736560029BA17300256373CB
:107A4000E573A06045F0FFF9E26B206328B960732D
:107A5000E0646063104639F0BFF9294645F00DFB3C
:107A6000E06B45F0F0F9E26B606318B96073E064B5
:107A70002063EFE7294645F000FB3D48A56601235A
:107A8000BAF1000F18BF5046DFF8ECA084F8383088
:107A900040F2AE3204F11001C4E91055A4F8485088
:107AA00036F028FC4FF4856204F11401B9F1000F9F
:107AB00014BF4846504636F01DFC40F2C92204F17E
:107AC0001801B8F1000F14BF4046504636F012FCC2
:107AD00040F20B3204F11C01002F14BF384650460F
:107AE00036F008FC002E14BF3046504640F2B1324A
:107AF00004F1200136F0FEFBD4ED017ADFED1D6AC2
:107B000084ED098AB8EE677AB8EE488AC6EE877ABD
:107B1000667B84F82CB0C4ED0A7AC7EE267A67EE4D
:107B2000887AFCEEE77A17EE903A02335E437600ED
:107B30002365304645F087F9E06420B9C4E90C00BC
:107B40006073304687E73246294645F096FA20466C
:107B5000C4E91555C4E91755656611B0BDEC028B33
:107B6000BDE8F08FB8250900B70108005863080088
:107B7000020000C000007A44020080BF10B5044635
:107B8000407B3FF079FFE16D094A9FED0A0ACB0B7C
:107B9000A2EBD13233EA210328BF134607EE903A15
:107BA000F8EEE77ABDE8104087EE800A22F0A0B830
:107BB000FFFF010000FF7F47F0B50D4685B055F887
:107BC000044B0646607B17463FF056FF02AB01931D
:107BD000154B00933A4602232946701E1BF062F8AB
:107BE000029D9DF80C6029460022204605F07EF992
:107BF0002846A56684F848603FF08EFF04F14402F1
:107C0000A06E04F140013FF03CFF227B636CD20880
:107C1000B3FBF2F36364431E5842584184F84900B1
:107C2000204605B0F0BD00BFA82509002DE9F04FA2
:107C30002DED048B8DB00029099314BF134600234A
:107C4000069390F82430876AB3FA83F35B0980F8CF
:107C5000243000EB83030446D3F81CB0037BDB081D
:107C6000B7FBF3F7836B0293D0E93A239A42C0F053
:107C7000E681B2FBF3F30593DA468FE10023C4F803
:107C80000831A1E1227B236BD208B3FBF2F3421E41
:107C900050425041236384F83500D4F80831002B5A
:107CA00000F0A481617B226B60680B02934228BFC5
:107CB0001346BB4294BF03930397E36A0493039B69
:107CC000B3FBF1F189B233F03FFB04F1100036F061
:107CD00039FB04F118008DED0B0AF7EE000A9FED59
:107CE000250A4FF0ACF9042204F114010BA830EE80
:107CF000008A45F06DF920B19DED0B0A204615F084
:107D0000F9F804F1A003079304F144030025B0EE51
:107D1000009AF7EE008A08932FE1102A25D14FF43C
:107D200000422BF8132001339F42FAD8617B606830
:107D3000B7FBF1F189B233F007FB04F1100036F024
:107D400001FB04F1180036F0FDFA94F82430099A8A
:107D500004EB83030120DB691360A26A1A9B1A609B
:107D60000DB0BDEC048BBDE8F08FD2087A438021C2
:107D7000504644E100000000069B012B00F04281C8
:107D8000637BB5FBF3F803FB185808F1FF33D3F11D
:107D9000000848EB0308237B102B049B40F035813F
:107DA00033F91530D4E90F1201FB0822029921F8AA
:107DB000123000222646A44601929CF8441061B37A
:107DC000DCF84810E06B029A090AB1FBF0F900FBFD
:107DD000191900FB0899013132F91990B1FBF0F241
:107DE00000FB121100FB0811029ADCF8500032F976
:107DF0001110DCF84820A1EB09015FFA82FE0EFBAE
:107E000001FED4F8FC10019A31F9101009EB2E2E66
:107E100001FB0EFE02EBEE320192079A0CF1140CFC
:107E20006245CAD179EE487AD4F8F810019AF4EE96
:107E3000E78AD017F1EE10FAA1FB022C01FB00CC6F
:107E4000D4BFB0EE686AB0EE676AD20B07EE903A24
:107E500042EA4C42B8EEE77A07EE902AF4EEC88A7E
:107E6000F1EE10FAF8EEE77AD4BFF0EE686AF0EEC1
:107E7000486A66EEA77A41F6EF31E6EE077AFDEE44
:107E8000E77A17EE900A36F079FC237B102B40F04E
:107E9000C6802BF81500A37B1BB980F400402BF89B
:107EA0001500637B012B02D0B8F1000F64D096F867
:107EB000443063B1D6E912321344B364336D726D4A
:107EC00001339342336524BF002386F84430079B77
:107ED0001436B342EBD1D4F8E430002B40F0AD803F
:107EE0001946142208984A43825C002A40F0A08078
:107EF00094ED3C7AD4F8E800B5EEC07AF1EE10FAD1
:107F000019DD07EE900AF8EE677A67EE877AFCEEE5
:107F1000E77A17EE903A73B1D4F8F42082EA42324D
:107F200082EA524282EA42120133C4F8F420B2FBE0
:107F3000F3F603FB1623D4E90F623244121AD21A65
:107F4000B2FBF6F306FB1323142202FB01421B02D1
:107F5000012182F844109364D4F80431D3640023DF
:107F6000C2E91430059BC4F8E430236CE26B0133A2
:107F7000934228BF002323640135039B9D427FF475
:107F8000FBAE227BE36AD20805FB0233E362236B7C
:107F90005B1B7F1B0BEB450BAA442363002F3FF4B5
:107FA000D4AE236B002B7FF478AE94F835305BB9F8
:107FB00094F83430002B3FF461AED4F80801002867
:107FC0003FF45CAE3FF0A8FDD4F8080170B104F1B5
:107FD000300204F12C013FF054FD02287FF452AE30
:107FE0000023C4F80831236384F83530A37B227B57
:107FF000002B3FF492AED2087A430021584645F058
:108000003CF893E6DDF81880C5E6A27B5B57002AB2
:108010007FF4C8AE83F07F03DB435BB2C2E6A37B91
:1080200013B10AF805003CE780F07F00C043F8E791
:10803000013108297FF455AF94E7013B93E7012311
:1080400019E600BF2DE9F04F2DED068B8DB00846E7
:1080500011461A4602AB01938C4B00930A2345F05C
:1080600070F90B9840F283230222012145F09CF91C
:10807000089D002D064604DC4FF48E6101201AF0A5
:10808000A3FEDDF81080B8F1010F03DC4FF450714E
:108090000220F4E705984FF432730822012145F0DD
:1080A00083F9DDF824B0BBF1080F074605D0BBF11A
:1080B000100F02D0764838F009FF76494FF48670E9
:1080C00046F09CFC04460698DDE902A920F0F6FC87
:1080D00007989DF828306560002584F80CB0A373DC
:1080E0006673E573A060A062B0EE408A44F0AEFE15
:1080F000E06128B9204640F0E1FAA06A38F06CFE51
:10810000A26A294644F0B9FFA06A44F09FFE2062AB
:108110000028EFD0A26A294644F0AFFF012384F87B
:10812000243040F2814204F110015046C4E90B555D
:10813000C4F80851A58636F0DDF840F2B13204F1FA
:108140001801484636F0D6F8082F28BF0827012F17
:10815000B5EEC08A38BF0127F1EE10FAC4F8E88006
:10816000C4F8EC7029D4B7EE000AB4EEC08AF1EE80
:1081700010FAD8BFB0EE480A474B657BC4F8F4301C
:108180004FF48033B3FBF7F3B3F5004F28BF4FF440
:10819000004308FB05F5C4F8F830AD004FEA48038A
:1081A00084ED3C0AE363284644F050FEA06338B9EE
:1081B000204640F083FA2846A0E79FED380ADBE727
:1081C0002A46002144F059FFD4F8E850C4F8005181
:1081D00000236D002364284644F038FEC4F8FC00F8
:1081E0000028E5D0D4F80031DFED2D8A9FED2DAACF
:1081F000012B83BF03F1FF3307EE903AB8EE678A95
:10820000B7EE008A0025B7EE009AF6EE009AD4F891
:1082100000319D421FD3002384F8443084F8583045
:1082200084F86C3084F8803084F8943084F8A83076
:1082300084F8BC3084F8D030C4F8E43004F1100085
:1082400036F080F8204614F055FE20460DB0BDEC07
:10825000068BBDE8F08F07EE905AB8EE670A20EE65
:10826000280A80EE080A0DF0C9FBD4F8FC3039EE7C
:10827000400A20EE290A20EE0A0ABDEEC00A10EEDE
:10828000102A23F815200135C1E700BF5825090041
:10829000B701080018630800CDAB341200000000DD
:1082A000DB0FC94000FEFF46F0B50D4685B055F81E
:1082B000044B0646607B17463FF0DEFB02AB0193A2
:1082C000164B00933A4602232946701E1AF0EAFC28
:1082D000029D9DF80C6029460022204604F006FE0F
:1082E0002846C4F8085184F834603FF015FC04F1C6
:1082F0003002D4F8080104F12C013FF0C2FB227BCC
:10830000236BD208B3FBF2F32363431E5842584158
:1083100084F83500204605B0F0BD00BF48250900AF
:1083200010B50446084620F0C9FBB5EEC00AF1EED0
:1083300010FA0CD4F7EE007AB4EEE70AF1EE10FA78
:10834000D8BFF0EE407AC4ED3C7A0E2010BDDFEDD0
:10835000017AF8E7000000002DE9F04F2DED068BC3
:108360008BB0D0F85CA009930B1E049314BF134686
:108370000023069390F83C30026CB3FA83F35B0958
:1083800080F83C3000EB830304465B6B0093037B77
:10839000DB08B2FBF3F30193036D427B0593436D5E
:1083A000B3FBF2F34FEA530B21B1069B012B08BF3D
:1083B000D0F860A0236BDB03A3F5DA43603B6FF0DA
:1083C0007042B2FBF3F30893009B0393F0EE009A24
:1083D000019BCBB9049B002B00F05881069B012B1D
:1083E00040F05481C4F860A094F83C30099A04EB42
:1083F000830301205B6B1360226C1A9B1A600BB025
:10840000BDEC068BBDE8F08FA36C4BBB94F84D30F0
:1084100033B994F84C30ABB1606E98B13FF07CFB4F
:10842000606E60B104F1480204F144013FF029FBA1
:1084300002280AD100236366A36484F84D30617B6F
:108440000D0216E000236366EAE7227BA36CD208E4
:10845000B3FBF2F3A364431E5842584184F84D0025
:10846000617B636E0D02002BE9D0A36C9D4228BF97
:108470001D46019B60689D4228BF1D46B5FBF1F17A
:1084800089B232F061FFF7EE000A04F120009FED9F
:10849000810A4EF0D4FDF7EE000A30EE008A04F1B6
:1084A0001C009FED7C0A4EF0CAFD636E0293B0EE95
:1084B00040AA0BB1636C02930027F7EE008ABD421D
:1084C00017D1019B5B1B0193009B03EB45030093BA
:1084D000039B2B440393636E002B3FF479AF227B05
:1084E000636CD20805FB02336364A36C5B1BA3645B
:1084F0006EE7049B002B40F0AE80637BB7FBF3F983
:1085000003FB1979B9F1010F666E14BF4FF0000932
:108510004FF001090BFB09F936B1237B102B029BAD
:1085200040F09C8033F91760226B002A00F0A08095
:10853000E06AA16A031F079301EB820C4FF0000869
:108540000798B1EC017A50F8043F0790ABEB0303B6
:108550005344B3FBFBFE0BFB1E3305984B448C4589
:1085600030F9133007EE903AF8EEE77A67EE877A43
:10857000FDEEE77A17EE903A9844E1D1012A06D051
:1085800040460899079236F0F9F8079A8046059B0D
:10859000D14433F91900237B07EE900AF8EEE77A0D
:1085A000002A08BF804667EE8A7A102BFDEEE77A34
:1085B00017EE900A30445DD141F6EF3136F0DEF827
:1085C00079EEC87A059BF4EEE78AF1EE10FAD4BF93
:1085D000B0EE686AB0EE676A07EE906AB8EEE77AC6
:1085E00007EE908AF4EEC88AF1EE10FAF8EEE77A18
:1085F000D4BFF0EE686AF0EE486A66EEA77A23F818
:108600001900E6EE077A41F6EF31FDEEE77A17EE54
:10861000900A36F0B3F8237B102B2ED1009B23F861
:108620001700A37B23B9009B80F4004023F81700B8
:10863000627B012A07D0049B2BB9B7FBF2F302FB44
:108640001373012B05D10AF1010AD34598BF4FF0EE
:10865000000A013733E7069B012B55E7DE57A37B62
:10866000002B7FF461AF86F07F06F64376B25BE7BE
:1086700090468CE700F30700A2E7A37B13B1039BAE
:10868000D855D5E780F07F00C043F8E7C4F85CA078
:10869000AAE600BF000000002DE9F04F2DED028B8F
:1086A0008DB0084611461A4602AB0193594B009310
:1086B0000A2344F046FE4FF467734FF47A620121B7
:1086C000029844F071FE40F2832308EE900A0222E1
:1086D0000B98012144F068FE089E002E054604DC3C
:1086E0004FF48E6101201AF06FFBDDF824B0BBF16E
:1086F000080F05D0BBF1100F02D0474838F0E6FB59
:108700004649682046F07AF90446DDE9059707985E
:108710009DF8282065730025DDE9038A84F80CB0F4
:10872000A2736660E573A060206444F08CFB606314
:1087300028B920463FF0CAFF206C38F04DFB226C70
:10874000294644F09AFC206C44F07DFBA06300288D
:10875000EFD0226C9FED328A294644F08EFC3148DE
:108760006566012384F83C304FF42E7204F11C013D
:10877000BAF1000F18BF5046C4E91155A4F84C5087
:1087800035F0B8FD284840F2B13204F12001B9F1CA
:10879000000F18BF484635F0ADFDD4ED017A637B7C
:1087A000C4ED048AB8EE677AC7EE087AB8EE687A44
:1087B00067EE877AFCEEE77A17EE900A584340009E
:1087C000A06544F040FB206520B920463FF07EFFC5
:1087D000A06DB2E7A26D294644F04FFCD4ED017ABA
:1087E000F8EE677A414688EE277A204684ED067ACD
:1087F00008F01AFD2046C4E91755C4E90955C4E933
:108800000B55394608F04AFD20460DB0BDEC028BF1
:10881000BDE8F08FF8240900B7010800F8620800ED
:1088200000007A443233B3BF020000BFF0B50D46FA
:1088300085B055F8044B0646607B17463FF01CF99F
:1088400002AB0193154B00933A4602232946701E52
:108850001AF028FA029D9DF80C6029460022204655
:1088600004F044FB2846656684F84C603FF054F9F8
:1088700004F14802606E04F144013FF002F9227BEA
:10888000A36CD208B3FBF2F3A364431E58425841D1
:1088900084F84D00204605B0F0BD00BFE824090073
:1088A0002DE9F04F2DED048B8BB00029079314BFF9
:1088B00013460023069390F83030476B456A427B9D
:1088C000B3FA83F35B0980F830300A33044650F87A
:1088D0002390037BDB08B7FBF3F7436C0393036A36
:1088E0005B08B3FBF2FB002D00F08181C36C0293A7
:1088F0006D08B5FBF2F5CA46F0EE009A2BE10023B5
:10890000E3653DE1227BE36BD208B3FBF2F3421E49
:1089100050425041E36384F84100E36D002B00F0C6
:108920003F81617BE26B60680B02934228BF134674
:10893000BB4294BF04930497A36B0593049BB3FBC2
:10894000F1F189B232F000FD04F1100035F0FAFCCB
:1089500004F118008DED090AF7EE000A9FEDA50A53
:108960004EF06DFB042204F1140109A830EE008AD8
:1089700044F02EFB20B19DED090A204631F000F8AD
:108980000026F7EE008AD5E0102A25D14FF40042E8
:1089900029F8132001339F42FAD8617B6068B7FB46
:1089A000F1F189B232F0D0FC04F1100035F0CAFCCC
:1089B00004F1180035F0C6FC94F83030079A0A33F9
:1089C000012054F823301360626B189B1A600BB0BF
:1089D000BDEC048BBDE8F08FD2087A43802150466D
:1089E000E7E0069B012B00F0E780637BB6FBF3F822
:1089F00003FB186808F1FF33D3F1000848EB0308C4
:108A0000237B102B059B40F0DA8033F91630227F50
:108A1000019308FB0BF0A2B9A26C0244002D00F0F8
:108A2000D880216D029B08FB051133F91110039BBF
:108A300023F81210226D08FB052CDDE9012323F831
:108A40001C20616D039B00EB11200A0A33F9100012
:108A5000F5B1A16C91428CBFDC464FF0000C944400
:108A6000BCEB010E14D0AE4512D8226D7244B2FB9D
:108A7000F5F305FB132208FB0522029BA1EB0C0179
:108A800033F9122029444A4300FB0E2292FBF5F0F1
:108A900079EEC87A06EE900AF4EEE78AF1EE10FA63
:108AA000F4EEC88AD4BFB0EE686AB0EE676AF8EE3A
:108AB000E66AF1EE10FADDED017AD4BFB0EE687A25
:108AC000B0EE487AF8EEE77A27EE267A41F6EF31F3
:108AD000A6EE277AFDEEC77A17EE900A35F04EFE25
:108AE000237B102B7AD129F81600A37B1BB980F4C5
:108AF000004029F81600637B012B02D0B8F1000F6B
:108B000017D0227F62B9A36C01335B4528BF13469F
:108B1000A3642DB1236D0133AB4238BF1A462265E1
:108B2000D4E915321344B3EB0B2F28BFA3EB0B236F
:108B300063650136049B9E427FF453AF227BA36B97
:108B4000D20806FB0233A363E36B9B1BBF1B09EB3D
:108B50004609B244E363002F3FF42EAFE36B002BD2
:108B60007FF4DBAE94F8413053B994F84030002BD9
:108B70003FF4C5AEE06D00283FF4C1AE3EF0CCFF3F
:108B8000E06D68B104F13C0204F138013EF079FF78
:108B900002287FF4B7AE0023E365E36384F8413035
:108BA000A37B227B002B3FF4EFAED2087A43002157
:108BB000484644F062FAF0E6DDF8188020E7A27B30
:108BC0009B57002A7FF423AF83F07F03DB435BB224
:108BD0001DE7039B019923F8121032E7A37B13B121
:108BE0000AF8060087E780F07F00C043F8E70295A7
:108BF00081E600BF000000002DE9F04F8DB008466F
:108C000011461A4603AB01934D4B0093092344F0E0
:108C100098FB0B9840F283230222012144F0C4FB0D
:108C2000DDF82090B9F1000F074604DC4FF48E61A7
:108C300001201AF0C9F8099D082D04D0102D02D08A
:108C4000404838F043F94049602045F0D7FE0446DB
:108C5000DDE9058607989DF8283025730025DDE9B4
:108C600003BAA3736773C4F80490E573A0606063EC
:108C700044F0ECF8A06228B920463FF030FD606B6C
:108C800038F0AAF8626B294644F0F7F9606B44F0BB
:108C9000DDF8E0620028EFD0626B294644F0EDF980
:108CA000012384F8303040F2814204F1100158462B
:108CB000C4E90E55E565A4F8405035F01BFB40F2C1
:108CC000B13204F11801504635F014FBF9B240F20C
:108CD0002D5249002577404644F05EFBC4F82080C1
:108CE000404644F0B3F8606420B920463FF0F7FCFA
:108CF000206AC5E7226A294644F0BFF96662E6B1F8
:108D0000304644F0A3F8E06420B920463FF0E7FC89
:108D1000606AB5E7626A294644F0AFF90023C4E906
:108D20001433A36404F1100035F00CFB204630F03E
:108D300027FE20460DB0BDE8F08FE664EEE700BFE9
:108D4000A0240900B701080038630800F0B50D46FB
:108D500085B055F8044B0646607B17463EF08CFE06
:108D600002AB0193154B00933A4602232946701E2D
:108D700019F098FF029D9DF80C60294600222046BC
:108D800004F0B4F82846E56584F840603EF0C4FE7F
:108D900004F13C02E06D04F138013EF072FE227BEA
:108DA000E36BD208B3FBF2F3E363431E584258412E
:108DB00084F84100204605B0F0BD00BFE827090057
:108DC0000E29F7B5944604463FD011F003032ED187
:108DD00008681F4DA84227D10E461E4F56F8045F63
:108DE000AB420DD101F1080605FB0CF22160E068F1
:108DF000110144F02EF8C4E90165E06003B0F0BD54
:108E000056F8040F82070AD01FF0E2FEC38812480A
:108E1000009340F21232F123752138F04BF80268CA
:108E2000BA42F1D10133DBE70A4B98420AD0084637
:108E30001FF0CEFEC388009308489D23F12240F224
:108E40001231EAE726460125CEE700263546CBE774
:108E500044EC0700B4590800740B0800F80A080035
:108E60002DE9F04F2DED0E8B85B00446039390F85D
:108E70002C30076BB3FA83F35B0980F82C3000EBDE
:108E80008303D3F82480037BC146DB08B7FBF3F7E9
:108E9000002F00F02881A36B002B32D194F83D30D5
:108EA00033B994F83C30F3B1206CE0B13EF034FEBD
:108EB000206C60B104F1380204F134013EF0E1FDB0
:108EC000022813D100232364A36384F83D30A37BDD
:108ED000227B002B00F0E780D2087A430021404635
:108EE00044F0CBF8E8E000232364E1E7227BA36BA6
:108EF000D208B3FBF2F3A363431E5842584184F8EF
:108F00003D00236C002BE2D0617BA36B6068D4F83A
:108F100034A09FEDC88A0D029D4228BF1D46BD4268
:108F200028BF3D46B5FBF1F189B232F00DFAF7EEFC
:108F3000000A04F110009FEDC00A4EF080F8DFED4A
:108F4000BF0A04F11400F0EE408A9FEDBD0A4EF016
:108F500076F820EE080A10F075FAF3EE080A04F12C
:108F60001800F0EE40BA9FEDB70A4EF068F820EE18
:108F7000080A10F067FAF7EE000AB0EE40AA04F112
:108F800020009FEDAD0A4EF05AF8267FB0EE409AD1
:108F9000002E40F0BD80DFEDAC7A77EEE88ADFEDA1
:108FA000AB7AB4EEE79AF1EE10FA40F2E880DFED2A
:108FB000A8AA9FEDA8BA4FF0000BAB4500F0D180F6
:108FC000237B0293102B40F0DC803AF91B3007EE34
:108FD000903AB8EEE78A237F68EE2B7A012BFDEEFC
:108FE000E7CAB7EE00CA08D11CEE902A617F324072
:108FF0000CEE902A002900F00C81B8EEEC0A022B4E
:1090000020EE2A0A00F0C880032B00F0F0805BB944
:10901000F0EE680AB0EEC00A2EF0EAF81CEE903AC4
:10902000002B01DAB1EE400A637F019320EE0A0AB9
:109030005BB1B5EEC00AF1EE10FA40F3E580B1EE97
:10904000400A10F0FFF93CEE400A20EE0B0A019BAB
:10905000FDEEC07A63B917EE903A7F4A9342B8BFEB
:10906000134647F6FF718B42A8BF0B4607EE903AB6
:10907000F8EEE77A3CEE49CA67EE897A029BE8EEA1
:109080000C7A102BFDEEE77A17EE903A40F0C8808C
:1090900028F81B30A17B19B983F4004328F81B3052
:1090A0000BF1010B89E7102A2DD14FF4004228F86B
:1090B000132001339F42FAD8617B6068B7FBF1F15E
:1090C00089B232F041F904F1100035F03BF904F1B6
:1090D000140035F037F904F1180035F033F904F1D4
:1090E000200035F02FF994F82C30039A04EB830319
:1090F00001205B6A1360226B1C9B1A6005B0BDECFB
:109100000E8BBDE8F08FD2087A4380214846E7E60F
:10911000032E09D1DFED4C7A38EEA87A77EEE87AA3
:10912000C7EE278A00263AE7012EFBD1B2EE0C0AE1
:1091300028EE800A30F008FEBCEEC00A10EE103AAD
:109140009E4076422BE7227B102A0BBF3AF9132070
:109150001AF9032028F8132009F803200133AB4241
:10916000F1D1227B636BD20805FB02336363A36BEF
:109170005B1B7F1B08EB4508A944A36388E600231B
:10918000EDE7A17B1AF90B3000297FF420AF83F0C3
:109190007F03DB435BB21AE7DFED307A60EE27CA6C
:1091A000F0EEEC7AB1EEE70AFEEE087A20EE270A3E
:1091B00010F048F9B0EE40DAB0EE6C0A10F042F967
:1091C000F0EE40DA3DEE0C0AB1EE6CEA2CEEC00A8D
:1091D00010F038F9F0EE40CAB0EE4E0A10F032F955
:1091E0007DEEECCA70EE2D7A8CEEA70A1CE778EEC5
:1091F0008C7AB0EE4C7A67EE807AB0EEC00AA0EEC0
:10920000287A87EE870A0FE710F01CF930EE4C0A37
:109210001BE7F8EEEC7A67EE8A7AFDEEE77A1AE75A
:10922000A17B11B109F80B303AE783F07F03DB43F0
:10923000F8E700BFE3C8EB3D00000000000070420B
:10924000000070C20000A0C24703803F0AD7233C41
:109250000000003800FEFF460180FFFFC0B12F3F35
:109260002DE9F04F91B0084611461A4605AB01931F
:10927000404B00930B2344F064F80F9840F2832393
:109280000222012144F090F80C9E002E834604DC5B
:109290004FF48E61012019F097FD0D9F082F04D027
:1092A000102F02D0344837F011FE089D35B1284602
:1092B000324940F2B53219F0D7FD2D7930494420BA
:1092C00045F09CFB0446079B0B989DF838209DF8C1
:1092D00024800293DDE905A90A9B66600026A2733B
:1092E000277384F80DB0E673A0602063039343F006
:1092F000ADFD226B606220B96073A062104637F04A
:109300006BFD314643F0B9FE206B43F09FFD226BAD
:10931000A06210B960736062F0E7314643F0ADFEC1
:10932000012384F82C3004F110015046C4E90D6685
:109330002664A68740F2E22234F0DCFF04F1140137
:10934000484640F20D4234F0D5FF029804F118016E
:1093500040F20B4234F0CEFF039840F2B13204F1F8
:10936000200134F0C7FF2046257784F81D8011B016
:10937000BDE8F08F90270900B70108007C62080063
:10938000B862080010B50446407B3EF075FB217FB3
:109390000248BDE8104040F0DFBC00BF7C6208001E
:1093A000F0B50D4685B055F8044B0646607B174670
:1093B0003EF062FB02AB0193154B00933A46022349
:1093C0002946701E19F06EFC029D9DF80C6029461E
:1093D0000022204603F08AFD2846256484F83C607C
:1093E0003EF09AFB04F13802206C04F134013EF0A7
:1093F00048FB227BA36BD208B3FBF2F3A363431EAB
:109400005842584184F83D00204605B0F0BD00BFE9
:109410008027090038B50C460546054940F2B532AB
:10942000204619F021FDA3882B770E2038BD00BF00
:109430007C6208002DE9F04F2DED028B87B00446C9
:10944000059390F82C30066BB3FA83F35B0980F830
:109450002C3000EB8303F7EE008AD3F82480037BE3
:10946000CDF80080DB08B6FBF3F6002E00F0A880F4
:10947000A36B04F12007002B42D194F8413033B99B
:1094800094F840305BB3606C48B33EF045FB606CD1
:1094900060B104F1380204F134013EF0F2FA02281E
:1094A00020D100236364A36384F84130617B60684A
:1094B000B6FBF1F189B231F047FF384634F042FF94
:1094C00004F110003EF0E3F8A37B227B002B6FD069
:1094D000D20872430021404643F0CFFD70E00023E4
:1094E0006364D4E700F1FF3E227BA36BDEF1000052
:1094F00040EB0E00D20884F84100B3FBF2F3A36303
:10950000636C617B6068002BD0D0A36B0D029D4221
:1095100028BF1D46B54228BF3546636BB5FBF1F148
:1095200089B2019331F010FF9FED900AF7EE000A27
:1095300038464DF084FDDFED8E7AB4EEE70AF1EEA9
:1095400010FAB0EE408A6FD9E369002B5AD0002799
:10955000AF4259D2637BEA1B013B22FA03F3B3F516
:10956000807F28BF4FF4807302937B000493019B9C
:1095700003EB470303930021627B029B03FB02F092
:10958000884253D84FF00009A2694A4572D8049B1B
:1095900003EB080A009B4FF0000903EB070B627B0B
:1095A000029B03FB02F1494500F283800F44CFE7A1
:1095B000102A15D14FF40043013E28F8023BFBD19D
:1095C00094F82C30059A04EB830301205B6A136046
:1095D000226B129B1A6007B0BDEC028BBDE8F08FC6
:1095E000D20800987243802176E7227B102A019AE4
:1095F00015BF009932F91320D25628F8132018BF4E
:10960000CA540133AB42F0D1009B227B2B44009320
:10961000636BD20805FB02336363A36B5B1B761B92
:1096200008EB4508A36320E70023EBE7B1FBF2F06A
:1096300002FB101202F1FF3CDCF1000242EB0C02D3
:1096400000EB0220227BE36B102A06D1039A32F949
:10965000112043F8202001318EE7019A94F80EE0A2
:109660003A445256BEF1000FF3D182F07F02D2434A
:1096700052B2EEE7626952F829B0584608F032FF5C
:109680004FF0000A617B5FFA8AFC614502D809F15C
:10969000010979E7E069E26B029B09FB01C100EB7C
:1096A000011102EB8C2258464DF06CFC0AF1010AC4
:1096B000E8E7B9FBF2F102FB1192531E5A425A41FC
:1096C00001EB0221E26B02EB8103D3ED007A227BF6
:1096D000F8EEE77A102A78EEC86A67EE887A1FD12A
:1096E000039B33F9193007EE103AB8EEC77A41F60A
:1096F000EF31E7EE267AFDEEE77A17EE900A35F0C5
:109700003DF8AAF80000A27B1AB980F40040AAF83C
:10971000000009F101090AF1020A0BF1010B3EE711
:10972000019BA17BDA1912F9092061B107EE102A19
:10973000B8EEC77AE7EE267AFDEEE77A17EE902AC2
:109740008BF80020E5E782F07F02D24352B207EEA9
:10975000102AB8EEC77A6FF07F02E7EE267AFCEEA9
:10976000E77A17EE903A5A40EAE700BF000000009F
:109770000AD7233C2DE9F0438BB0084611461A4620
:1097800003AB0193304B0093072343F0DAFD0998B4
:1097900040F283230222012143F006FE069E002EA2
:1097A000814604DC4FF48E61012019F00DFB079D0A
:1097B000082D04D0102D02D0244837F087FB24490F
:1097C000482045F01BF904469DF820300598257384
:1097D0000025A373DDE9038784F80D906660E573C7
:1097E000A060206343F032FB226B6062294643F0A5
:1097F00044FC206B43F02AFB226BA062294643F015
:109800003CFC607B012384F82C30800243F01EFB7B
:10981000627BE0632946920243F02FFC627B656421
:10982000414604F11000C4E90D55A4F84050FFF77B
:10983000C7FA384640F2B13204F1200134F05AFD43
:1098400020460BB0BDE8F08348270900B7010800A7
:10985000D8620800F0B50D4685B055F8044B0646B1
:10986000607B17463EF008F902AB0193154B00935D
:109870003A4602232946701E19F014FA029D9DF8FB
:109880000C6029460022204603F030FB2846656420
:1098900084F840603EF040F904F13802606C04F155
:1098A00034013EF0EEF8227BA36BD208B3FBF2F357
:1098B000A363431E5842584184F84100204605B036
:1098C000F0BD00BF382709002DE9F04F2DED068BC4
:1098D0008FB004460B930B1E089314BF134600234E
:1098E000099390F82C30056BB3FA83F35B0980F889
:1098F0002C3000EB8303D3F82480037BC346DB08C2
:10990000B5FBF3F5002D00F0FB80A36B04F110090B
:1099100004F11407002B43D194F83D3033B994F887
:109920003C307BB3A06C68B33EF0F6F8A06C60B13D
:1099300004F1380204F134013EF0A3F8022824D1E6
:109940000023A364A36384F83D30617B6068B5FBAA
:10995000F1F189B231F0F8FC484634F0F3FC3846B6
:1099600034F0F0FC04F1180034F0ECFCA37B227B13
:10997000002B00F0BD80D2086A430021404643F02E
:109980007CFBBDE00023A364D0E7411E227BA36BD8
:1099900048424841D20884F83D00B3FBF2F3A36388
:1099A000A36C617B6068002BCFD0A36B0E029E423C
:1099B00028BF1E46AE42636B029328BF2E46B6FBFD
:1099C000F1F189B231F0C0FCD4ED080A9FED820AB2
:1099D00048464DF034FBDFED810A3846B0EE40AA30
:1099E0009FED7F0A4DF02BFBF7EE000AB0EE408AA8
:1099F00004F118009FED780A4DF021FBDFED796A44
:109A000020EE260ABDEEC00A10EE103A1BB2B3F5E6
:109A1000A47F049340F3A58094ED087ACAEE077AF8
:109A20000027B7EE007A37EE676A37EE877A28EEBE
:109A3000268AC6EE077ABDEEC88A67EEA67A18EEC9
:109A4000103AFDEEE77A1BB2079317EE903A1BB27D
:109A500005935B420A93B74275D0089B002B40F0F8
:109A60008280627BB7FBF2F302FB13735A1E5342F0
:109A70005341227F12FB03F20392227B102A029AA7
:109A800073D132F917200192626C32F91300079BEF
:109A90000F21584334F018FF019B0021184434F083
:109AA00013FF039B81464FEA430A0022237F934220
:109AB00064D8039B626C003B18BF01230F2122F87E
:109AC0001390049B09FB03F034F0FEFE019B02217E
:109AD000184434F053FE237B102B73D128F8170061
:109AE000A37B1BB980F4004028F817000137B2E7C8
:109AF000102A15D14FF40043013D28F8023BFBD159
:109B000094F82C300B9A04EB830301205B6A1360FA
:109B1000226B1E9B1A600FB0BDEC068BBDE8F08F68
:109B2000D2086A438021584629E7227B102A029AEC
:109B30000BBF32F91320D25628F813200BF803205C
:109B40000133B342F1D1227B636BD20806FB0233AF
:109B50006363A36B9B1BAD1B08EB4608B344A36375
:109B6000D0E60023EDE7099B80E7A17BD2570029CF
:109B700089D182F07F02D24352B284E70A9B0D92D0
:109B800009FB03F00F2134F09FFE236C069333F999
:109B90000A300021184434F097FE059A03460F213D
:109BA00050430C9334F090FE0021484434F08CFE76
:109BB000069B0D9A23F80A00DDF8309001320AF175
:109BC000020A73E7A37B13B10BF807008EE780F05E
:109BD0007F00C043F8E700BF000000006666663FF4
:109BE000CDCCCC3D00FEFF462DE9F04F8DB00846B0
:109BF00011461A4603AB01933E4B0093092343F0F1
:109C0000A0FB0B9840F283230222012143F0CCFBFE
:109C1000DDF820B0BBF1000F824604DC4FF48E610A
:109C2000012019F0D1F8099D082D04D0102D02D083
:109C3000314837F04BF931494C2044F0DFFE0446FF
:109C40009DF828309DF81870079825730025A37398
:109C5000DDE90396DDF8148084F80DA0C4F804B0A3
:109C6000E573A060206343F0F1F8226B606229463F
:109C700043F003FA206B43F0E9F8226BA062294617
:109C800043F0FBF9607BA564012384F82C309840F5
:109C9000C4E90D55A58743F0D9F8627B6064294675
:109CA000520043F0EAF9D4ED017A154BFBEEEF7A5E
:109CB0000E2E08BF1E46C4ED087A04F11001484676
:109CC00040F2213234F016FB04F11401304640F228
:109CD0000B3234F00FFB40F2B13204F11801404670
:109CE00034F008FB204639463EF000FD20460DB01A
:109CF000BDE8F08FF0260900B7010800986208005F
:109D00003233B3BFF0B50D4685B055F8044B064667
:109D1000607B17463DF0B0FE02AB0193154B0093FC
:109D20003A4602232946701E18F0BCFF029D9DF89A
:109D30000C6029460022204603F0D8F82846A56486
:109D400084F83C603DF0E8FE04F13802A06C04F1B8
:109D500034013DF096FE227BA36BD208B3FBF2F3F5
:109D6000A363431E5842584184F83D00204605B085
:109D7000F0BD00BFE02609002DE9F04F2DED028B6C
:109D800093B0826C0E9390F84430B3FA83F35B097E
:109D900080F8443000EB83030446DB6B0193037BC4
:109DA000DB08B2FBF3FBB04B1B1A0D93BBF1000FAA
:109DB0000FD194F844300E9A04EB83030120DB6B3F
:109DC0001360A26C1E9B1A6013B0BDEC028BBDE841
:109DD000F08F236D6BBB94F855303BB994F8543039
:109DE000C3B1D4F83801A8B13DF096FED4F83801DB
:109DF00068B104F1500204F14C013DF042FE02282A
:109E00000CD10023C4F83831236584F85530617BC8
:109E10000D0218E00023C4F83831E7E7227B236DF8
:109E2000D208B3FBF2F32365431E5842584184F82D
:109E30005500617BD4F838310D02002BE7D0236D3B
:109E40009D4228BF1D465D459FED888A606828BFFA
:109E50005D46B5FBF1F189B231F076FAF7EE000A12
:109E6000B0EE480A04F114004DF0E9F8F7EE008A6C
:109E7000B4EEE80AF1EE10FA00F38880B4EEC08A7E
:109E8000F1EE10FAC8BFB0EE480ADFED797A20EEA5
:109E9000270AF7EE000ABDEEC00A04F1380010EE02
:109EA000103A1BB20393C3F500431BB29FED6F0A38
:109EB0000A934DF0C4F830EE000AF0EE007A77EE27
:109EC000C07A9FED6C7AF4EEE78AF1EE10FAD8BF13
:109ED000F0EE687AF4EEC08A67EE877AF1EE10FA57
:109EE000D8BFB0EE680AFDEEE77A20EE070A17EE5B
:109EF000903ABDEEC00A1BB2089310EE103AF7EE8E
:109F0000000A1BB29FED590A099304F110004DF0AD
:109F100096F8B4EEE80AF1EE10FA3ADCB4EEC08A34
:109F2000F1EE10FAD8BFB0EE408ADFED537A28EE9A
:109F3000278A4FF00008BDEEC88AC14618EE103AD5
:109F400003F5B34319331BB2079304F11803184602
:109F500004933DF09CFB04F12803184605933DF063
:109F600096FBE36C06934746454515D1019B227B42
:109F700003EB45030193E36CD20805FB0233E36472
:109F8000236D5B1BABEB050B23650FE7B0EE680A97
:109F90007BE7B7EE008AC8E7D4F8383113B1069BE7
:109FA00033F91830617B0293B5FBF1F201FB1252D9
:109FB000029B0498D2B23DF019FB42F2222358438F
:109FC000112134F081FC002F0CBF0823102304EB77
:109FD00043030B93C4F178030F9004EB47064FF053
:109FE000000A0C930B9BB34248D147F6E1201121A4
:109FF00000FB0AF034F068FCB9F1000F04F593722D
:10A000000CBF0421082102EB4906034602EB41097B
:10A01000B14565D1617BB5FBF1F201FB1252D2B2C1
:10A0200005983DF0E3FA089B064602980F21584335
:10A0300034F04AFC099B81465E431E200F21704389
:10A0400034F042FC41F6EF31484434F097FB019B79
:10A0500023F81800637B022B01D1002F5AD0002770
:10A06000B94608F101087FE7BCFEFFFF00000000D1
:10A07000CDCC4C4600FEFF46295C0F460C9AB6F943
:10A08000B83052F81620B6F8D80032F913C0CDE92E
:10A090001032039B10FB03F00A9B0F210CFB030003
:10A0A000E24434F011FC079BA6F8D8000F21584376
:10A0B00034F00AFC0F9B0021184434F005FCDDE964
:10A0C000103222F81300B6F8B830B6F95610013342
:10A0D0001BB29942D8BF0023A6F8B830023681E7F8
:10A0E0000D9A52F8162036F9021F32F9110003EBCF
:10A0F000600C22F811C0C01A012134F0E5FB32884F
:10A1000036F9301C013212B29142D8BF0022034608
:10A1100032807DE74FF004090827A2E72DE9F04FD0
:10A120008FB0084611461A4604AB0193844B009346
:10A130000A2343F006F90D9840F2832302220121FD
:10A1400043F032F90A9D002D064604DC4FF48E617F
:10A15000012018F039FE9DF8303013B9794836F0F7
:10A16000B5FEDDF82CA0BAF1100F01D07648F6E765
:10A1700076494FF49E7044F041FC0446DDE90870D6
:10A18000DDE906B39DF83020A273DDE9049865602F
:10A19000002584F80CA06673E573A060A0640393A7
:10A1A00042F051FEE06328B920463EF0B7FAA06CB9
:10A1B00036F012FEA26C294642F05FFFA06C42F01E
:10A1C00042FE20640028EFD0A26CDFF89CA1294653
:10A1D00042F053FF012384F84430627BC4F83851C5
:10A1E000594604F11800C4E91355A4F85450FEF779
:10A1F000E7FD627B039904F12800FEF7E1FDB9F168
:10A20000000F14BF4846504640F25E4204F1100170
:10A2100034F070F8B9F1000F14BF4846504640F2D0
:10A220005E4204F1100134F065F8B8F1000F14BF7C
:10A230004046504640F2B22204F1140134F05AF87C
:10A24000002F08BF5746B8F1000F14BF40465046D4
:10A2500040F2B22204F1140134F04CF8384640F2D6
:10A26000B13204F1380134F045F8384640F2B132E9
:10A2700004F1380134F03EF83549364A364840F2A8
:10A280005C43A4F85630354B2367C4E91612C4E981
:10A290001A12C4E9183040F25163A4F87430F6B2CF
:10A2A00004F1540704F17408A946B5EBC60F12D3A4
:10A2B0002B4A2C4BC4E93E23C4E94023002504F17A
:10A2C000F60704F58278A946B5EB860F1FD3204622
:10A2D0000FB0BDE8F08FB7F90200400042F0B3FDC7
:10A2E00048F8040F38B904EB450520463EF016FA4D
:10A2F000B5F956005CE737F9022F0021520042F011
:10A30000BCFE0135A7F86290A7F88290CDE7B7F9B7
:10A310000200400042F097FD48F8040F30B97C3548
:10A3200020463EF0FBF934F9150041E737F9022FDA
:10A330000021520042F0A1FE0135A7F83090C3E79A
:10A3400090260900B2F80700BE0108005C62080010
:10A35000A404FD044C058E0551065C04D3051506C6
:10A360002C02B9015501E100020080BFF0B50D4695
:10A3700085B055F8044B0646607B17463DF07CFBE4
:10A3800002AB0193164B00933A4602232946701EF6
:10A3900018F088FC029D9DF80C602946002220469A
:10A3A00002F0A4FD2846C4F8385184F854603DF00A
:10A3B000B3FB04F15002D4F8380104F14C013DF034
:10A3C00060FB227B236DD208B3FBF2F32365431EAF
:10A3D0005842584184F85500204605B0F0BD00BFF2
:10A3E0008026090070B58AB0084611461A4606ABA9
:10A3F0000193264B0093042342F0A3FF0698052205
:10A4000003A91CF0A5F9059C622C0ED0682C0FD076
:10A41000482C1FD0422C01D1002507E0012C1BD075
:10A420001B4840F2732136F059FD0125012401E05B
:10A43000012502249DF8243083B9079B049A6343C5
:10A440005B00B2FBF3F103FB11223AB1114840F279
:10A450007321E8E70025ECE70025EBE70E4918201B
:10A4600044F0CCFAE4009DF824309DF81C10089AC2
:10A47000039E0473049CC373002306618573846088
:10A480004173426003750AB070BD00BF2824090003
:10A490001B0B080091060800D86308002DE9F04165
:10A4A0001C460D4692B011462846824A18F0C2FB5F
:10A4B0002668814B3340062B05D0B10710D1326896
:10A4C0007E4B9A4208D144F2A62231467C4843F0A2
:10A4D0008BF88207064603D132687A4B9A4202D043
:10A4E000794836F0DFFC012D14D9062208A96068EE
:10A4F0001CF02EF940F273230998089F4FF48062F4
:10A50000082118F08FFC4307054605D06F48082145
:10A5100036F0E4FC00252F466D49402044F06EFAE9
:10A52000044606630022002306F1080040F0DEFA2C
:10A53000206B10226B460DEB0201083040F0C3FD8A
:10A5400010B1052036F086FC009B102B0BD1614921
:10A55000042204A842F03CFD28B95F49082206A85D
:10A5600042F036FD18B140F20D3018F08DFB206B33
:10A5700004226B460DEB0201083040F0A4FD0028D8
:10A58000DFD1009B042B02D1019A282A02D953481B
:10A5900036F09CFC206B6B4608A9083040F093FD18
:10A5A0000028CED1019A282A03D0BDF82030012BF3
:10A5B0000CD1BDF82210022908D8BDF82E30102B7E
:10A5C00004D8122A04D1BDF830208AB14448DFE70C
:10A5D000282A0DD1BDF820004FF6FE729042F5D129
:10A5E000BDF83820012AF1D1BDF832209A42EDD1D0
:10A5F000082B099A237394BF00230123A3734FF4FC
:10A600000073A360002362606173E373206B6B4689
:10A61000042202A9083040F056FD002891D1009E86
:10A62000042E8ED12F49324602A842F0D1FC80463A
:10A63000206B6B46324603A9083040F044FD0028E9
:10A640007FF47FAF009B042B7FF47BAF206B039ADA
:10A65000B8F1000F0AD0D0E91013521843F10003EB
:10A66000083040F043FA0028D0D06AE72262036C39
:10A67000A38465B94FF48070E06242F0E7FB0346C3
:10A680002061E06A63B9A561657336F0A5FB6D08CA
:10A6900027612F44E562A761204612B0BDE8F08132
:10A6A00042F0D4FBA0610028F6D1E06A2561657311
:10A6B000EBE700BF040002000F0080FF7CF40700FE
:10A6C0002C1708006C170900B4FE0700FE080800EC
:10A6D000B8630800ACE50700B1E50700CF06080045
:10A6E00069070800B2B107002DE9F04F2DED048B8A
:10A6F00095B005460B920893426A002943D00B9B04
:10A70000012B00D1826A229BA9691960296A2B7FDB
:10A71000914240F01584D5E90421002B18BF114661
:10A72000089B069119602B7F83F001032B77AB699F
:10A730009B080A9305F130030E9300230C930593B5
:10A7400095F82C300C9A93421FDC059B3BB9069A76
:10A750000A99059B02EB8101914240F0D183AB7BCA
:10A76000002B00F0D0832B6A01332B620B9B002B54
:10A7700040F0ED836B6A01336B62012015B0BDECD4
:10A78000048BBDE8F08F0B91BDE70E9B53F8046F6F
:10A790000E93B3680993002B40F0A6830C9B013302
:10A7A0000C93CDE7B360059B002B00F0A28301233F
:10A7B0000593F3E773699B087361431E5842584140
:10A7C00070730998697B407B3469736988424FEAEA
:10A7D000012240F0A0809A4228BF1A46079B93426C
:10A7E00094BF04930492049B6868B3FBF1F189B2AF
:10A7F00030F0AAFDF7EE000A06F118009FEDB10A4D
:10A800004CF01DFCDFEDB00AB0EE408A06F11C00F2
:10A810009FEDAE0A4CF02FFCDFEDAD7A6A7B28EE9F
:10A82000278A022ABCEEC88A18EE103A1FFA83FA69
:10A8300077D110F4004F47F6FF7315BFC0181B1AED
:10A8400080B24FF400400AFB00F00CBF9BB24FF403
:10A8500000430AFB03F3C11303914FEAE33A336A5F
:10A860001193736A12930598099B297B5B7B0027E0
:10A870001397002840F07E81102940F0F480A97BD6
:10A88000002900F082809A427DD0049BCDF834B03C
:10A890004FEA530904EB8909A14563D054F8048BAE
:10A8A000039B1FFA88F0CDE900A340EA084012ABF1
:10A8B00011AA13A93CF02CFA119F3F0437FB00FEAC
:10A8C000129F4FEA074C3CFB10F02EF3CF3720F3DA
:10A8D000CF30C7EA00470D9840F8087B039F0D90E2
:10A8E0004FEA18400004CDE900A740EA18403CF0C8
:10A8F0000FFA119B1B0433FB00F3129A120432FB74
:10A9000010F223F3CF3322F3CF32C3EA02430D9A7E
:10A9100042F8043CC0E75B00934228BF1346079A05
:10A920005DE7CDF80CA09AE7039B54F8270011AA25
:10A93000CDE900A313A912AB3CF0EAF9119B1B046B
:10A9400033FB00F3129A120432FB10F223F3CF33DD
:10A9500022F3CF32C3EA02434BF827300137049B7E
:10A96000BB42E1D1049A079B687B9B1A0793099B22
:10A970005B7B98420BEB820BD6E9041200F08782D6
:10A98000049B5B0884E2059FE9E79A4267D0049B39
:10A990005B0804EB8303D9460D930D9B9C42E1D0E9
:10A9A00054F8043B4FF0802293FA42F8039B1FFABD
:10A9B00088F0CDE900A340EA084012AB11AA13A920
:10A9C0003CF0A6F9119F3F0437FB00FE129F4FEAAF
:10A9D000074C3CFB10F02EF3CF3720F3CF30C7EA03
:10A9E000004749F8087B4FEA1840039F0004CDE96F
:10A9F00000A740EA18403CF08BF9119B1B0433FB85
:10AA000000F3129A120432FB10F223F3CF3322F335
:10AA1000CF32C3EA024349F8043CBEE754F82700AA
:10AA200090FA48F0039B11AACDE900A313A912AB39
:10AA30003CF06EF9119B1B0433FB00F3129A1204D5
:10AA400032FB10F223F3CF3322F3CF32C3EA0243B7
:10AA50004BF827300137049BBB42DFD182E7059FCB
:10AA60004FF08028F7E79A42049B4FEA430931D11F
:10AA7000059F4FF080284F45BFF474AF34F817009E
:10AA80004DF05AFCAB7B0BB990FA48F0039B11AA2E
:10AA9000CDE900A313A912AB3CF03AF9119B1B04BA
:10AAA00033FB00F3129A120432FB10F223F3CF337C
:10AAB00022F3CF32C3EA024049F076FE2BF81700AA
:10AAC0000137D8E70000000000FE7F3F00FE7FBF97
:10AAD00000000047DDF8148008F101034B45BFF486
:10AAE00041AF34F808004DF027FCAB7B07461BB99B
:10AAF0004FF0802390FA43F7039BB8B2CDE900A34F
:10AB000040EA074012AB11AA13A93CF001F9119BCE
:10AB10001B0433FB00FC129B1B0433FB10F32CF3D0
:10AB2000CF3C23F3CF33CCEA034049F03DFE039BF7
:10AB30002BF81800380C0004CDE900A340EA1740B8
:10AB400012AB3CF0E5F8119B1B0433FB00F3129AA7
:10AB5000120432FB10F223F3CF3322F3CF32C3EAD5
:10AB6000024049F021FE0BF1020323F8180008F11E
:10AB70000208B1E7102940F0F380A97B002973D0C7
:10AB80009A424BD0049B5B0804EB8303D8460D9399
:10AB90000D9B9C423FF4E6AE54F8049B039B1FFAC6
:10ABA00089F0CDE900A340EA094012AB11AA13A92C
:10ABB0003CF0AEF8119F3F0437FB00FE129F4FEAB6
:10ABC000074C3CFB10F02EF3CF3720F3CF30C7EA11
:10ABD000004758F8080B97FA10F748F8087C4FEA36
:10ABE0001940039F0004CDE900A740EA19403CF05A
:10ABF0008FF8119B1B0433FB00F3129A120432FBF3
:10AC000010F223F3CF3322F3CF32C3EA024358F8D2
:10AC1000042C93FA12F348F8043CB9E7049BABF117
:10AC2000040704EB830844453FF49CAE039B54F8AF
:10AC3000040B11AACDE900A313A912AB3CF068F8EC
:10AC4000119B1B0433FB00F3129A120432FB10F227
:10AC500023F3CF3322F3CF32C3EA024357F8042F52
:10AC600093FA12F33B60DEE79A424FD0049B5B08F5
:10AC700004EB8303D9460D930D9B9C423FF472AEC7
:10AC800054F8043B4FF0802293FA42F8039B1FFADA
:10AC900088F0CDE900A340EA084012AB11AA13A93D
:10ACA0003CF036F8119F3F0437FB00FE129F4FEA3D
:10ACB000074C3CFB10F02EF3CF3720F3CF30C7EA20
:10ACC000004759F8080B97FA10F749F8087C4FEA43
:10ACD0001840039F0004CDE900A740EA18403CF06B
:10ACE00017F8119B1B0433FB00F3129A120432FB7A
:10ACF00010F223F3CF3322F3CF32C3EA024359F8E1
:10AD0000042C93FA12F349F8043CB5E7049BABF129
:10AD1000040704EB83084FF0802944453FF422AE3A
:10AD200054F8040B90FA49F0039B11AACDE900A353
:10AD300013A912AB3BF0ECFF119B1B0433FB00F398
:10AD4000129A120432FB10F223F3CF3322F3CF32E4
:10AD5000C3EA024357F8042F93FA12F33B60DCE78F
:10AD600004999A424FEA41010D9140F08D80ABF178
:10AD700002084FF080290D9B9F42BFF4F3AD34F8D9
:10AD800017004DF0D9FAAB7B0BB990FA49F0039B51
:10AD900011AACDE900A313A912AB3BF0B9FF119B97
:10ADA0001B0433FB00F3129A120432FB10F223F35C
:10ADB000CF3322F3CF32C3EA024238F8020F4DF00C
:10ADC000BBFA92FA10F049F0EFFC0137A8F8000046
:10ADD000D1E7E05B4DF0B0FAAB7B80461BB94FF09A
:10ADE000802390FA43F8039B1FFA88F0CDE900A373
:10ADF00040EA084012AB11AA13A93BF089FF119B4E
:10AE00001B0433FB00FE129B4FEA034C3CFB10FC7F
:10AE10002EF3CF332CF3CF3CC3EA0C433BF817009F
:10AE20000F934DF089FA0F9B93FA10F049F0BCFC98
:10AE3000039B2BF817004FEA18400004CDE900A34C
:10AE400040EA184012AB3BF063FF119B1B0433FB3D
:10AE500000F3129A120432FB10F223F3CF3322F3E1
:10AE6000CF32C3EA02423BF819004DF065FA92FA7C
:10AE700010F049F099FC02372BF8190009F102098A
:10AE80000D9B4B45A5D86DE54FF00109F8E7049BF4
:10AE9000C6F820A001EB8301D21AC6E90412039B75
:10AEA0007362079B002B3FF482AC7369002B7FF425
:10AEB00088AC737B33B9337B002B3FF473ACB06841
:10AEC0003CF02AFEB06800283FF47BAC06F1140287
:10AED00006F110013CF0D5FD02287FF46BAC002395
:10AEE000B360736173735EE40A9BDDF818B0079377
:10AEF000D7E7079B05999A00584642F0BEF856E4FA
:10AF000042F8043B28E42B7B0A9A102B069B03EBA8
:10AF100082020AD04FF080309A423FF424AC196884
:10AF200081FA40F143F8041BF6E74FF0802093428A
:10AF30003FF419AC196891FA40F143F8041BF6E7A5
:10AF40001BB92B69089A136010E46B69FAE70B9B35
:10AF5000012B7FF412ACAB6A2A7B0133AB62089BF6
:10AF60001B6803EBD203089A136006E42DE9F0474F
:10AF700088B0084611461A4602AB0193364B00933F
:10AF8000062342F0DEF94FF4A463FF220121029868
:10AF900042F00AFA40F28323064602220498012175
:10AFA00042F002FA079D002D804604DC4FF48E61CA
:10AFB000012017F009FFDDF814A0BAF1080F05D041
:10AFC000BAF1100F02D0254835F080FF06F10D00D0
:10AFD0002349800043F012FD039F9DF8189004461A
:10AFE000F8088000A06141F031FF03462061A069AC
:10AFF0001BB96373636135F0EFFE41F027FF6061B9
:10B0000018B960732061A069F5E765600025A76045
:10B0100084F80CA084F80E9084F80D80E57384F811
:10B020002C6004F13007B5420ADB94F82C0004F1DF
:10B0300034011FF029F82063204608B0BDE8F087EE
:10B04000002308481A46194600F06AF8013547F807
:10B05000040F4460E7E700BFBC290900B7010800FE
:10B060003C620800A0290900F0B50C4687B054F8EE
:10B07000045B0646687B17463CF0FEFC03AB01937D
:10B08000124B00933A462146701E032317F00AFE26
:10B0900095F82C20049840F21F53013A002142F009
:10B0A00083F9C0B205EB8000039E446B9DF81470D9
:10B0B00060680122314601F019FF2046A66027731F
:10B0C0003DF03AFB284607B0F0BD00BF88290900D3
:10B0D000F0B50D4685B055F8044B0646607B174623
:10B0E0003CF0CAFC03AB01930C4B00933A46294653
:10B0F000701E012317F0D6FD94F82C20039840F21F
:10B100001F53013A002142F04FF9C0B204EB800412
:10B110000022636B0E209A6005B0F0BD8029090003
:10B1200010B508461146002217F084FD0B4928206F
:10B1300043F064FC00230446836000F118014FF4DF
:10B140006172074833F0D6F8064840F2EE3204F157
:10B150001C0133F0CFF8204610BD00BFA029090024
:10B16000020000C0020080807FB502AB51F8044BA2
:10B1700001930B4B00930138022317F093FD029DBE
:10B1800060689DF80C600122294601F0AFFE204660
:10B19000A56026733DF0D0FA0E2004B070BD00BF4C
:10B1A000702909001FB503AB0193064B51F8044BFE
:10B1B00000930138012317F075FD00230E20A360D2
:10B1C00004B010BD682909002DE9F04FAFB0446A02
:10B1D00004902CB9389B02201C602FB0BDE8F08F82
:10B1E00000290499896814913899149C0C60049979
:10B1F00091F9541008BF00228A42049913D104988F
:10B2000091F9551000EB8101496B01EB42021A6084
:10B21000FF2380F85430389B1A68836D03EB520388
:10B2200083650120D9E791F84410049CB1FA81F1BB
:10B23000490984F8441084F85510C2F1010204EB66
:10B24000810184F854204A6B1A60069241F0ACFFE9
:10B250000498002141F083FF049B044670B99A686A
:10B260000146069841F009FF389B1C60049B93F847
:10B27000450080F001004000C0B2AEE7049ADB6AEE
:10B28000126BD21A0992049A12690392002A01F0F1
:10B290001C85049A0398576A1F4439463AF000FB0C
:10B2A000411C064601F01585039BD3F80090B9F1C7
:10B2B000000F00F04381D3F80480B8F1000F00F0D4
:10B2C0003D8199F800B099F81C303C18BBF1000F93
:10B2D0003ED1032B4FF0090114BF4FF0200A4FF06D
:10B2E000110A2AA8CDE92A4BCDE92CBA4DF0D8FC99
:10B2F000C8F8000099F81C30032B14BF0321052166
:10B300002AA84DF0CDFC454645F8040F039BD3F821
:10B31000BC379B450DDB4FF0000B039BD3F8C437C4
:10B320009B4580F2C880902303FB0B850023059387
:10B3300092E005F1100301212AA805934DF0B0FC1D
:10B34000059B45F8040F9D42F5D10BF1010BDDE79C
:10B35000032B4FF0080114BF4FF0110A4FF0090AF8
:10B3600000232AA8CDE92B332A94CDF8B4A04DF0C0
:10B3700097FCC8F8000099F81C30032B14BF022179
:10B3800001212AA84DF08CFCC8F80400C3E70C2169
:10B390002AA84DF085FC0921A8622AA84DF080FC5E
:10B3A0000821E8622AA84DF07BFC286399F8003058
:10B3B000002B14BF092104212AA84DF071FC0121A2
:10B3C00068632AA84DF06CFCA863002856D00221BF
:10B3D0002AA84DF065FC0121E8632AA84DF060FC25
:10B3E000052128642AA84DF05BFC052168642AA881
:10B3F0004DF056FC0023EB64A86403212AA84DF00D
:10B400004FFC032128652AA84DF04AFC03216865FA
:10B410002AA84DF045FCEB6BA86533BBC5E90A33A0
:10B420006B63E86DC0F11400286699F80030002BBA
:10B430003FD101212AA84DF033FC686601212AA8DA
:10B440004DF02EFC0121A8662AA84DF029FC059B91
:10B45000E866013305934835039B059AD3F8BC375A
:10B460009A4294DB0BF1010B57E7022B04D12B6CB2
:10B4700013B90823EB65D4E70723FBE7C5E90F0001
:10B4800005212AA84DF00CFC052168642AA84DF07E
:10B4900007FC0521A8642AA84DF002FC0421E864F9
:10B4A0002AA84DF0FDFB0321E8652AA84DF0F8FB22
:10B4B000BAE70020C1E7039A0999D8F80080C2F8DA
:10B4C000D88706EB0A028A1A03990992D1F8B817AD
:10B4D000039A04EB0A05D2F8B027002960D0002AAD
:10B4E00040F0AA80039BD3F8CC27099B934280F2BB
:10B4F000B480069903983AF0F3FE4FF0FF34149AA3
:10B500000698002141F0B9FD049B93F845300BB932
:10B51000E31C21D8049B06989A68002141F0ADFDF8
:10B52000389A002313600334049A4FF001038CBF50
:10B530000020012082F8453098404EE60699039895
:10B540003AF0CEFE6FF00604049B099A1B6B9B1A1F
:10B55000049AD362002CD2D1049B149A9B6D03EB06
:10B560005203049A9365104641F01EFE0498002190
:10B5700041F0F5FD049B049A1B6BD26A9A1A049B56
:10B580009B6A9B1AB3F5007F044607DD049AAE4B15
:10B5900002F11400C2E9053201F0ECFC20461CE681
:10B5A000002A49D10399DDF824B00122C1F8B0275F
:10B5B000A9465946484605933AF0A6FE421C059B0B
:10B5C00018D019F800C039788C4509EB00021DD15C
:10B5D00092F801C079788C4518D197F802C091781B
:10B5E0008CEA0101032911D81CF0020F18BF02F1E7
:10B5F000FF32501B039A0028C2F8B4070CDA0699F0
:10B6000010463AF06DFE6FF002049DE7033002F140
:10B610000309ABEB000BCCE7039A0644D2F8C02732
:10B6200056445643039AD2F8C8275343039AF60068
:10B6300096FBF3F3C2F8B837039BD3F8B4271B6823
:10B6400043B15B69003B18BF01231344039AC2F85E
:10B65000CC3747E74FF0FF33F7E7039B0399D3F865
:10B66000DC37434501F11C003DDBA3EB08014246FA
:10B6700041180A9041F0EBFC039BD3F8D807D3F8AC
:10B68000CC270A9B2946184441F0B6FC039B03993A
:10B69000D3F8CC27D3F8D8371344C1F8DC37DB0014
:10B6A0001093039B099903F2DC738A1A1A930023FF
:10B6B00009920C930593039B059AD3F8C4379A42D9
:10B6C00081F21E837C235343119390235343199398
:10B6D000119B013B1F93119B08931A9B1893002306
:10B6E0000D939B46FEE32946184441F085FC039BDD
:10B6F0000399D3F8CC27D3F8DC3703981344C1F867
:10B70000DC37099B06999B1A09936FF001043AF004
:10B71000E7FD19E7039B1E68002E00F0D4805B68EC
:10B720000793002B00F0CF80039B9D68002D00F055
:10B73000CA800A9B22930023CDE923330C9A109BE5
:10B740009A18D31D48BF02F10E03DB1025930C9B02
:10B750001BB1194622A84DF0A3FA059B317890221F
:10B760005A43482303FB0B22079B1A44536BD2F81E
:10B770003CC0002940F04E81344810F8136000EBC3
:10B780004300BCF1020F477862D1D2F84090B9F182
:10B79000000F10D0089B884605EB0309314622A80C
:10B7A0004DF07EFA08F10108B8F1080F09F8010B15
:10B7B000F4D14FF00309119B05EB03080D9B98444E
:10B7C00009EB49039844314622A84DF069FA314605
:10B7D00088F8170022A84DF063FA314688F818005F
:10B7E00022A84DF05DFA09F10109B9F1060F88F8B8
:10B7F000190008F10308E6D1089BEE18394622A883
:10B800004DF04EFA394686F8290022A84DF048FA44
:10B81000394686F82A0022A84DF042FA09F10109BA
:10B82000B9F10C0F86F82B0006F10306E6D1059A54
:10B830007C2353433E2202FB0B332B44002283F82C
:10B840003B209A8724E000BFD12B04005C5C0900F8
:10B85000059B002B3ED10D9BDDF8148005EB030901
:10B86000314622A84DF01CFA08F10108B8F10B0F7F
:10B8700009F8010BF4D10D9B1D44394622A84DF067
:10B880000FFA05F8080008F10108B8F1150FF4D116
:10B89000059B189A90265E434820079B00FB0B6689
:10B8A00033449B6A5360229B0A9A9B1A249AC2EBE8
:10B8B000C302D71007D4189B53F804CF1893109BDA
:10B8C000634580F2ED81069903983AF009FD6FF027
:10B8D000070439E64FEA0B13079A083302EB030912
:10B8E00052F80380B8F1000F1FD00D9B8846EB186B
:10B8F0001F9913F8012B5A5408F10108B8F1060FEB
:10B90000F6D1D9F80430FBB9089B4FF0060805EBD7
:10B91000030A314622A84DF0C3F90AF8080008F1DD
:10B920000108B8F10B0FF4D121E0089B05EB030AE5
:10B93000314622A84DF0B4F908F10108B8F1060F1C
:10B940000AF8010BF4D1DCE7059C3E2303FB0BF363
:10B950007C20EA1800FB04332B4491799971D1794A
:10B96000D971117A1972517A5972927A9A72D9F8F8
:10B9700008306BB9089B0B2605EB0308394622A853
:10B980004DF08EF908F806000136102EF6D112E0BF
:10B99000059C3E2303FB0BF37C20EA1800FB0433D9
:10B9A0002B44D17AD972117B1973517B5973917BD6
:10B9B0009973D27BDA73D9F80C306BB9089B1026D7
:10B9C00005EB0308394622A84DF06AF908F806008D
:10B9D0000136152EF6D112E0059C3E2303FB0BF336
:10B9E0007C20EA1800FB04332B44117C1974517C31
:10B9F0005974917C9974D17CD974127D1A75059A09
:10BA00007C2353433E2202FB0B332B4400225A7506
:10BA10009A753DE7366A16F0010603D0BBF1010FB7
:10BA200000F0B280B3F5C87F7BDA1911052291FBD3
:10BA3000F2F2269202EB8202891AC3F38102289263
:10BA400003F0030300222791299311461346BCF10A
:10BA5000020F40F0CE80059C902060434827079C51
:10BA600007FB0B002044006C002808BF4FF0010CBE
:10BA700001EB41018948614410F821702A9700EBDD
:10BA8000810148782B908878C9782C902D910EB33D
:10BA9000BBF1010F1ED10DF1980C05F1FC070DF162
:10BAA000A80E664603CE764538607960B44607F145
:10BAB0000807F6D10DF1A80C05F58677664603CE8A
:10BAC00079602EA98E423860B44607F10807F5D197
:10BAD000C5F8F820059990224A43482101FB0B2222
:10BAE00007990A445366D36B022B40F0C580176C4C
:10BAF000002F00F0A880089B0026EF18269922A8A6
:10BB00004DF0CEF80136062E07F8010BF6D14FF0B6
:10BB100001080327119B05EB030A0D9B0AEB0304A5
:10BB20008BE0B3F5FA7F12DAA3F5C87399100522FA
:10BB3000B1FBF2F2269202EB8202891A03F00303B0
:10BB40000022279128932992134601217FE7A3F52C
:10BB5000FA730321B3FBF1F101EB41020598269141
:10BB60009B1A0022CDE9282290224243482000FB64
:10BB70000B22079827930244126C0AB1CDE92713D0
:10BB800000220123022162E7B3F5B47F03F0010232
:10BB90004FEA630110DA242091FBF0F3269300FBB7
:10BBA0001313062093FBF0F100FB113328930023BD
:10BBB0002791299303214AE7F3290CDCB4390B11AF
:10BBC0002693C1F38103279301F0030100232891F9
:10BBD000299304213BE7F4390323B1FBF3F32693C4
:10BBE00003EB4303C91A00232791CDE9283305212C
:10BBF0002DE74FF0000C3BE726AB22A853F828A016
:10BC000051464DF04DF85146F07522A84DF048F8D8
:10BC10005146307622A84DF043F8033609F1010968
:10BC2000B0752AAB53F828209145E5DB08F10108EF
:10BC3000B8F1040F3FF4FBAD4F4407EB4706264431
:10BC40004FF00009EDE7B84664E753F8261022A844
:10BC50004DF026F809F8010B013726AB5AF82620DB
:10BC60009742F2DB0136042E0DD0B84404EB0809EC
:10BC700000270DF1A80AF1E7089B4FF00008EC1827
:10BC8000464626ABF2E7059A7C2353433E2202FB4D
:10BC90000B331D440023AB756B75F9E57C5C090023
:10BCA000039B1D68002D00F0C2815B680B93002B85
:10BCB00000F0BD81039B9B68002B00F0B881039BC3
:10BCC000D968002900F0B38102F0070313930C9B9D
:10BCD000139AC3EBC70313441C93BCEB03030793F2
:10BCE00000F1A5810A9B6A6B3B441D930B9B1E448C
:10BCF000B36B002B00F02381F36B022B40F01F810C
:10BD0000336C002B40F00381059C9023634300FBC0
:10BD10000B330B9803440320DB6D013393FBF0F3EB
:10BD200002EB4303B3F92E0000EB40004FF4107216
:10BD3000059C9023634348250B9C05FB0B33234450
:10BD4000DB6A5B00B3F5107FA8BF4FF4107393421A
:10BD5000D4BF2C932C920A932D938342D4BF2B9360
:10BD60002B9001EB8B03209303F580530A9AC3F8C1
:10BD700000224FF4106303FB0B131593139B0F93D7
:10BD80001D9B0C93002316930E93199B4033E318CD
:10BD900021930E9B169F01332AAA0E9352F823304B
:10BDA0001693A3EB070EBEF1000F23DD159B0E9A31
:10BDB0000C9903EB8707219B53F82250B14B03EBFF
:10BDC000C5031E790F9B5A4202F0070213462AB19F
:10BDD00011F8010BC2F1200200FA02F2002E40F02D
:10BDE000C08033463A1D47F8263042F826300236E6
:10BDF000B645F8DC00230F9A0C991A4401EBE201D6
:10BE000002F007020F92079A0C91D31A07930E9B28
:10BE1000032BBED1109B1C9A9B1A0E93079B002BE1
:10BE200000F09F82159B0A9A0C9803EB8205059AF5
:10BE300090235343482202FB0B330B9AD318924AA8
:10BE4000DB6E52F823200B92904A52F823100F9B7E
:10BE50005B4203F007031A462BB110F8016BC3F1E4
:10BE6000200306FA03F3079CA61A0A9C4FF0000968
:10BE7000C4F50F7AC1F120014F460AF1010A0A9177
:10BE8000BA4500F3F081209B03F58052D2F80032CE
:10BE90003B44C2F800320022B3F5107FC0F2638247
:10BEA000079A0F9B13440C9A02EBE30203F007037B
:10BEB0000C93089B0A923E3308930D9B3E330D93DF
:10BEC000199B4833199313461D9A9B1A00F1AF80B2
:10BED000139AC2EBC3030C9A13440E9AD31A10930D
:10BEE0000BF1010B039BD3F8BC379B45FFF612AC5B
:10BEF0000599039838F0E8F8013040F05785069925
:10BF000003983AF0EDF96FF00904FFF71DBB2B78A9
:10BF10005BB9059C9023634300FB0B330B980344F0
:10BF2000DB6D013332F9130000E7B2F93600B2F9E4
:10BF30003430C31AB2F90C0000EB4300F6E6059B5F
:10BF400090255D43482303FB0B550B9B1D44EB6D74
:10BF50002D6E013332F913002B44013332F91320D3
:10BF6000E6E64B4850F825C04A4800EB4C001790D5
:10BF70000798012EA0EB030040F08E80454C34F86A
:10BF80001C6006F00F064FF000094FF0004AC6F1A2
:10BF900020060F2853DD8C46C3F118081CF8025BFD
:10BFA000497805FA08F5C3F1100801FA08F10D43C4
:10BFB0002A431033103861460A2BEADD22FA06F5CF
:10BFC000179C013534F815504FEA153C15F0F00F69
:10BFD00002FA0CF218BF02F0004CA3EB1533C5F3C4
:10BFE00003181EBF520003F1FF334CEA080815F492
:10BFF000706FC5F3032C1FBF03F1FF3302F0004540
:10C0000045EA0C0C52004B4511DB47F8088BAEF1AA
:10C01000020EBEF1000F47F804CCCDDCA3EB090300
:10C02000079A0344D31A079A93427FF6E4AE06991F
:10C0300003983AF055F96FF00804FFF785BA1D1818
:10C04000002DF4DD002812DD082891F800C0C8BFDB
:10C050004878C3F118080CFA08FCC8BFC3F11003F4
:10C0600042EA0C02C9BF98400131024302316B1E03
:10C070004AFA03F31A404FF00B0905F10B030020B5
:10C080009AE700BF58390900545C09004C5C09006C
:10C090007C5B0900583A0900A6F1020CBCF1010FC3
:10C0A000C5D8DFF8F0C25CF83580DDF85CC000244C
:10C0B000129408F101041B94C8F120041E940F2867
:10C0C00027DD8946C3F1180A19F8025B497805FA99
:10C0D0000AF5C3F1100A01FA0AF10D432A4310339D
:10C0E000103849460A2BEADDBCF8009009F00F0928
:10C0F000C9F1200522FA05F501353CF815505FEA33
:10C10000153A2AD1A3EB090302FA09F20CEB450C0C
:10C11000E8E71D18002D8ADD002812DD082891F8B7
:10C120000090C8BF4878C3F1180A09FA0AF9C8BFD5
:10C13000C3F1100342EA0902C9BF9840013102432A
:10C1400002314FF000406B1E40FA03F30B201A40FF
:10C15000129005F10B030020C4E7C5F30319B9F1F0
:10C160000F0FA3EB0A0302FA0AF2C5F3032523D14A
:10C17000032E24D11B9C00EB030C002D0CBFA24608
:10C1800004F1010AE2453FF752AF9C46E24552DC1A
:10C190000344B3EB0C0006D5581E9C464FF00043F9
:10C1A00003411A4000201E9B22FA03F909F10F09EE
:10C1B000ACEB080302FA08F2B9F1000F05D002F067
:10C1C000004C49EA0C095200013B0F2D1DD1032EF2
:10C1D0001CD11B9C1D18AC423FF729AF9C461B9CF1
:10C1E000644533DC0344B3EB0C0006D5581E9C4673
:10C1F0004FF0004303411A4000201E9B22FA03F532
:10C200000F35ACEB080302FA08F22DB102F0004C36
:10C2100045EA0C055200013B129CA342FFF607AF12
:10C22000AEF1020EBEF1000FC7E9009518DDDDF892
:10C230005CC0083756E711F8019BCCF1180409FAE5
:10C2400004F942EA09020CF1080C9FE711F8015BBE
:10C25000CCF1180A05FA0AF52A430CF1080CBEE7DE
:10C26000129A9B1ADCE60F2E56DD8446C2F1180E98
:10C270001CF8021B407801FA0EF1C2F1100E00FA10
:10C280000EF001430B431032103E60465745BFF697
:10C29000F7AD092A7FF7F4AD0A990B9C23FA01F157
:10C2A00021443B4C615C4FEA111C03FA0CF311F082
:10C2B0000808A2EB11121FBF03F0004802F1FF3281
:10C2C0005B0048F0010811F0040E1FBF03F0004EA0
:10C2D00002F1FF325B004EF0010E11F0020C1FBFA5
:10C2E00003F0004C02F1FF325B004CF0010C11F046
:10C2F00001011FBF03F0004102F1FF3241F00101D3
:10C300005B004A45FFF6BFAD45F8108B043745E9A1
:10C3100003EC45F8041CB9E7B11800297FF7B3AD69
:10C32000002E12DD082E90F800C0C8BF4678C2F17A
:10C33000180E0CFA0EFCC8BFC2F1100243EA0C033F
:10C34000C9BF96400130334302304A1E4FF00044CB
:10C3500044FA02F213404FF00A0901F10A020026E2
:10C3600094E7079F8FE5159941F82320013393E562
:10C37000059903982A4638F067FE01300CD10699DA
:10C38000039839F0ADFF6FF00A04FFF7DDB800BF86
:10C39000FC5B0900583909000135039BD3F8BC3711
:10C3A0009D42E5DB039AD268002A00F08684039A56
:10C3B00052690B92002A00F08084039A92690792D6
:10C3C000002A00F07A84039AD2F8C867059A564387
:10C3D000069A5E43022B02EB460640F0E9820B9B75
:10C3E0001193331D089300230E93079B03F500530D
:10C3F0000D930E9B0D9A0799119803F001030F936B
:10C400000B9B03F580554FF00077D5F8183B009350
:10C41000D2F800220F9B38F0F7FAD5F81C3B0D9AA2
:10C42000079911980093D2F800220F9B803100F5F4
:10C43000106038F0E9FA0F9B0D9A5B42D2F80022A7
:10C4400003F488631344079A02EB830B4FF0000C4C
:10C4500052F82320DBF85C306046C2FB007C6FF0B2
:10C460007301C3FB017C4FF00076DBF88020DBF822
:10C47000DC300546C2FB0065C3FB01654FF455790E
:10C48000DBF80430DBF85820C3FB097C834BC2FB8C
:10C49000037CDBF88410DBF8D820C1FB0965C2FB04
:10C4A000036541F6D478DBF80830DBF85420C3FB91
:10C4B000087C7B4BC2FB037CDBF88810DBF8D420C4
:10C4C000C1FB0865C2FB036546F2B86EDBF80C30B1
:10C4D000DBF85020C3FB0E7C724BC2FB037CDBF805
:10C4E0008C10DBF8D020C1FB0E65C2FB03656E4AE1
:10C4F000DBF81030DBF84C10C3FB027C6B4BC1FB4C
:10C50000037CDBF89000DBF8CC10C0FB0265C1FBBC
:10C510000365DBF81420DBF84830C2FB0E7C45F2E3
:10C520008401C3FB017CDBF89420DBF8C830C2FB3C
:10C530000E65C3FB0165DBF81820DBF84430C2FB55
:10C54000087C40F22C71C3FB017CDBF89820DBF8FF
:10C55000C430C2FB0865C3FB0165DBF81C20DBF8B7
:10C560004030C2FB097C7421C3FB017CDBF89C20BA
:10C57000DBF8C030C2FB0965C3FB01650C243846FB
:10C580004FF014080CFA04F34CFA08FC20FA08F0F7
:10C5900040EA030039F0D8FD089B23F8040C30462C
:10C5A00005FA04F345FA08F520FA08F040EA03001A
:10C5B00039F0CAFD089B0BF5805723F8020C3B6845
:10C5C0004FF4D0704FF000724FF0000CC3FB002C02
:10C5D0004FF00073D7F880100026C1FB003641F6FB
:10C5E0007C007968C1FB002CD7F88410C1FB0036B1
:10C5F00049F2FC70B968C1FB002CD7F88810C1FB68
:10C6000000362B49F868C0FB012CD7F88C00C0FB22
:10C61000013628493D69C5FB012CD7F89050C5FB70
:10C6200001366FF0B3057969C1FB052CD7F894107A
:10C63000C1FB05364FF41275B969C1FB052CD7F85B
:10C640009810C1FB05366FF0130EF969C1FB0E2C73
:10C65000D7F89C101D46C1FB0E5610460CFA04F389
:10C660004CFA08FC20FA08F040EA030039F06CFDAF
:10C67000089B9887284606FA04F346FA08F620FA3B
:10C6800008F040EA030039F05FFD089B0A49D887AB
:10C6900004331293089B043B13930FE0D4F8FFFF7D
:10C6A0007CAFFFFF3CB6FDFF78940400C449020054
:10C6B0004CE803002464FFFF38350900D1F840E05E
:10C6C000DBF80051DBF85C014FF000730022C5FB82
:10C6D0000E324FF000764C6C4FF00009C5FB046938
:10C6E000C4F1000CC0FB0C32C0FB0E69DBF8DC01AE
:10C6F000DBF8804115904FF000774FF0000AC4FB43
:10C700000E7A4FF00075486C4FF00008C4FB0058DB
:10C710001598C0FB0C7AC0FB0E58D1F848E0DBF846
:10C7200004C1DBF85801CCFB0E32CC6CCCFB0469A5
:10C73000C4F1000CC0FB0C32C0FB0E69DBF8D80161
:10C74000DBF884411590C4FB0E7AC86CC4FB00581A
:10C750001598C0FB0C7AC0FB0E58D1F850E0DBF8FE
:10C7600008C1DBF85401CCFB0E324C6DCCFB0469E4
:10C77000C4F1000CC0FB0C32C0FB0E69DBF8D40125
:10C78000DBF888411590C4FB0E7A486DC4FB005855
:10C790001598C0FB0C7AC0FB0E58D1F858E0DBF8B6
:10C7A0000CC1DBF85001CCFB0E32CC6DCCFB046924
:10C7B000C4F1000CC0FB0C32C0FB0E69DBF8D001E9
:10C7C000DBF88C411590C4FB0E7AC86DC4FB005891
:10C7D0001598C0FB0C7AC0FB0E58D1F860E0DBF86E
:10C7E00010C1DBF84C01CCFB0E324C6ECCFB046963
:10C7F000C4F1000CC0FB0C32C0FB0E69DBF8CC01AD
:10C80000DBF890411590C4FB0E7A486EC4FB0058CB
:10C810001598C0FB0C7AC0FB0E58D1F868E0DBF825
:10C8200014C1DBF84801CCFB0E32CC6ECCFB0469A2
:10C83000C4F1000CC0FB0C32C0FB0E69DBF8C80170
:10C84000DBF894411590C4FB0E7AC86EC4FB005807
:10C850001598C0FB0C7AC0FB0E58D1F870E0DBF8DD
:10C8600018C1DBF84401CCFB0E324C6FCCFB0469E1
:10C87000C4F1000CC0FB0C32C0FB0E69DBF8C40134
:10C88000DBF898411590C4FB0E7A486FC4FB005842
:10C890001598C0FB0C7AC0FB0E58D1F878E0DBF895
:10C8A0001CC1DBF84001CCFB0E32CC6FCCFB046921
:10C8B000C4F1000CC0FB0C32C0FB0E69DBF8C001F8
:10C8C000DBF89C411590C4FB0E7AC86F1691C4FB2F
:10C8D00000581599C1FB0C7AC1FB0E580C24184660
:10C8E000142102FA04F342FA01F220FA01F040EABC
:10C8F000030039F029FC129B23F8040C3846142756
:10C900000AFA04F34AFA07FA20FA07F040EA0300A9
:10C9100039F01AFC129B23F8020C304609FA04F392
:10C9200049FA07F920FA07F040EA030039F00CFC55
:10C93000139BA3F87C00284608FA04F348FA07F88A
:10C9400020FA07F040EA030039F0FEFB139B16992A
:10C95000A3F87E00129B04331293139B043B1393A2
:10C96000DE4B40318B420BF5807B7FF4A7AE0D9BF5
:10C970000F9AD3F800329B1A0D9A03F00703C2F8FE
:10C9800000320E9B01330E93119B80331193089B51
:10C99000803308930E9B122B7FF42BAD059B013344
:10C9A00005931A9B08331A93FEF785BE0025F4E41D
:10C9B000079B4036002703F5005807F001030E934C
:10C9C0000B9B0B98079903F5805300EBC710D3F826
:10C9D000183B0093D8F8002207F0010338F014F850
:10C9E00007F00103D8F800225B4203F48863134484
:10C9F000079A02EB8309002052F82310D9F85C2033
:10CA00004FF000730446C1FB04306FF07301C2FBAA
:10CA100001304FF4557ED9F80420D9F85810C2FBE4
:10CA20000E30AF4AC1FB023041F6D47CD9F8082061
:10CA3000D9F85410C2FB0C30AA4AC1FB023046F2AE
:10CA4000B865D9F80C20D9F85010C2FB0530A64AB9
:10CA5000C1FB0230A54AD9F81010C1FB0230A44A2C
:10CA6000D9F84C10C1FB0230D9F81410D9F848207D
:10CA7000C1FB053045F28401C2FB0130D9F8181022
:10CA8000D9F84420C1FB0C3040F22C71C2FB0130BC
:10CA9000D9F81C10D9F84020C1FB0E307421C2FB1C
:10CAA00001300C2402464FF0140A184602FA04F32F
:10CAB00042FA0AF220FA0AF040EA030039F044FB95
:10CAC00009F5805126F8400C0A684FF000700023E9
:10CAD0004FF4D075C2FB050341F67C054A68C2FBE2
:10CAE000050349F2FC758A68C2FB0503814DCA68DB
:10CAF000C2FB0503804A0D69C5FB02036FF0B30555
:10CB00004A69C2FB05034FF412758A69C2FB05032B
:10CB1000CA696FF01301C2FB010303FA04F243FA7E
:10CB20000AF320FA0AF040EA020039F00DFBDFF8C0
:10CB3000CCA126F8200CA6F140030D930896DAE963
:10CB400010ECD9F80021D9F85C114FF000700023E7
:10CB5000C2FB0E034FF000754FF0000BC2FB0C5BE5
:10CB6000CCF10002C1FB0203C1FB0E5BDAE912EC5F
:10CB7000D9F80411D9F85821C1FB0E03C1FB0C5B95
:10CB8000CCF10001C2FB0103C2FB0E5BDAE914EC3D
:10CB9000D9F80811D9F85421C1FB0E03C1FB0C5B75
:10CBA000CCF10001C2FB0103C2FB0E5BDAE916EC1B
:10CBB000D9F80C11D9F85021C1FB0E03C1FB0C5B55
:10CBC000CCF10001C2FB0103C2FB0E5BDAE918ECF9
:10CBD000D9F81011D9F84C21C1FB0E03C1FB0C5B35
:10CBE000CCF10001C2FB0103C2FB0E5BDAE91AECD7
:10CBF000D9F81411D9F84821C1FB0E03C1FB0C5B15
:10CC0000CCF10001C2FB0103C2FB0E5BDAE91CECB4
:10CC1000D9F81811D9F84421C1FB0E03C1FB0C5BF4
:10CC2000CCF10001C2FB0103C2FB0E5BDAE91EEC92
:10CC3000D9F81C11D9F84021C1FB0E03C1FB0C5BD4
:10CC4000CCF10001C2FB0103C2FB0E5B0C241421DA
:10CC500003FA04F243FA01F320FA01F040EA020079
:10CC600039F072FA0D9B23F8020F14210D93284618
:10CC70000BFA04F34BFA01FB20FA01F040EA03003F
:10CC800039F062FA089B23F8020D0893134B0AF15E
:10CC9000400A9A4509F580797FF451AFD8F80032FF
:10CCA0000E9A01379B1A03F00703122FC8F80032BF
:10CCB00006F140067FF481AE70E60699039839F0DC
:10CCC0000FFB6FF00B04FEF73FBC6FF00404FEF7A0
:10CCD0003BBC6FF00504FEF737BC00BFF838090015
:10CCE000D4F8FFFF7CAFFFFF3CB6FDFF7894040053
:10CCF000C44902004CE803002464FFFF38350900F2
:10CD00000024FEF721BC00BF2DE9FF411C460D4663
:10CD100028461146424A15F08DFF2768414B3B409B
:10CD2000062B05D0BA070AD13A683F4B9A4206D182
:10CD300039463E4844F2A62240F056FC07460121FF
:10CD4000384619F057FD067C16F0010602D0384827
:10CD500034F0A8F8012D2BD96068062201A919F03A
:10CD6000F7FCDDE9015633495C2041F04EFEEB074C
:10CD700004461FD50135013EB6F5305F1CD905F5D7
:10CD800090536563A6F5105605F51055A3636562CB
:10CD9000A6620023C4E90B334BF010FF206100288A
:10CDA00035D120463BF0DDFC234924484BF09BFA6B
:10CDB0003546D8E7002DDFD14FF40068C4F828804D
:10CDC000404640F043F8606228B920463BF0C9FC79
:10CDD000404634F001F8B6F5105F04D3656305F5FD
:10CDE0009055A563D5E74FF4905040F02FF860635D
:10CDF00028B920463BF0B5FC4FF49050E9E74FF4DA
:10CE0000905040F023F8A0630028C2D1F1E72046FB
:10CE1000394604F00DFB204604B0BDE8F08100BFA8
:10CE2000040002000F0080FF7CF407002C170800AC
:10CE3000B4FE07001C6208003308080000F4070075
:10CE400010B50446407B3AF017FEA3689FED107AB8
:10CE50005A0800EE102A94F8442004EB820423F0D0
:10CE60000103626B13449A4209D1F1EEC77ABDE81F
:10CE70001040B8EEC00A87EE800A1CF039BF32F9C4
:10CE8000021B07EE901AF8EEE77AA7EEA77AEAE718
:10CE90000000000038B504460D46407B3AF0ECFD3A
:10CEA00044F2A6222946044840F09EFB0146204653
:10CEB00004F0BEFA0E2038BD2C17080038B50D4618
:10CEC0000446407B3AF0D8FD0121284619F092FC37
:10CED000037CDB0702D5044833F0E4FF20462946F3
:10CEE00004F0A6FA0E2038BDB4FE0700F8B50C46D3
:10CEF0000546084617461FF075F9667B30463AF03E
:10CF0000BBFD62686B689A4204D04FF48E610D4895
:10CF100033F0E4FF6B7B0FB1022B04D0B34202D09D
:10CF200040F28321F3E7227B2B7B9A4202D040F22E
:10CF30006621ECE7A27BAB7B9A4202D040F29241A1
:10CF4000E5E7F8BD56040800064A00231370064AB8
:10CF50001370064B01221A71054B1B780BB10BF0B5
:10CF6000A1BD7047D6770020D4770020C06F002085
:10CF7000D577002010B5044604F084FEE3681BB9A1
:10CF80000A4A1168A14203D1BDE8104004F090BEE6
:10CF9000A360074B1968E160196809B119688C60D2
:10CFA000116801B914601C60EEE700BF60610020E9
:10CFB0006861002008B504F065FE044A1368013B6F
:10CFC0001360BDE8084004F073BE00BF5461002048
:10CFD00008B504F057FE044A136801331360BDE836
:10CFE000084004F065BE00BF546100202DE9F04107
:10CFF000154E01F09DFF2AF00DF833680BB3134D69
:10D0000004F040FE2C681CB1BDE8F04104F050BEB5
:10D010000F4A01232B603368346014601BB92B68FE
:10D02000013B2B60F0E7D3E900689F68C3E9024445
:10D0300004F03EFE0EB14046B04704F023FE3B46EE
:10D04000ECE7BDE8F08100BF606100205461002082
:10D050006861002008B51BF0BBFDC1880348972913
:10D0600014BF9722422233F025FF00BF06010800BB
:10D0700010B5064A002352F83340844202EBC30144
:10D0800001D90133F7E7486810BD00BF68210900E6
:10D09000F0B595B0054601A80E4617461C4647F068
:10D0A000C7F910B1002015B0F0BD3A463146284608
:10D0B00016F088F825F048FE830703D10268034B79
:10D0C0009A42EFD020600120EDE700BF54F4070042
:10D0D000014A04232AF014BCCC310900F0B587B012
:10D0E000084611461A4602AB0193294B00930423CC
:10D0F00040F027F9049D002D04DC40F2213101208D
:10D1000015F062FE2349182041F07FFC059B036166
:10D11000214B9D428CBF0123B3FBF5F3C3601F4B32
:10D12000D3F8A831DDE9027604465BB30FF030FA9C
:10D1300080F00105EDB204F11503009300222B46A7
:10D140004FF48F61384609F099FF04F116036060CF
:10D150000022009340F279412B46304609F08EFFC1
:10D1600001221146A06060680AF00CF80122A06854
:10D1700011460AF007F8204649F026F920B90520A3
:10D1800033F068FE0125D6E7204607B0F0BD00BFAA
:10D19000482909000062080020A10700946B0020C4
:10D1A000F0B50C4687B054F8045B0646284617468F
:10D1B0003BF002F828463BF00CF802AB0193094B18
:10D1C00000933A462146701E042315F06BFD059B23
:10D1D00000932846DDE90323029948F0CEF80E209B
:10D1E00007B0F0BD28290900F0B50C4687B054F807
:10D1F000045B0646284617463AF0DEFF28463AF01A
:10D20000E8FF02AB01930A4B00933A462146701E99
:10D21000042315F047FD01230193059B0093284645
:10D22000DDE9032302994BF05AFC0E2007B0F0BD54
:10D2300008290900F0B50C468BB054F8045B06468B
:10D24000284617463AF0B8FF28463AF0C2FF03AB2B
:10D2500001930E4B00933A462146701E072315F0AA
:10D2600021FD00230193079B0093DDE90312069B38
:10D2700028464BF034FC099B00932846089B059AEE
:10D28000039948F07AF80E200BB0F0BDD0280900C1
:10D290002DE9F0410D4686B055F8044B0646204670
:10D2A00017463AF089FF20463AF099FF02AB019306
:10D2B000244B00933A4604232946701E15F0F2FCD5
:10D2C000DDF80880B8F1000F04DC40F25B2101209A
:10D2D00015F07AFD40F2034301220021039840F04B
:10D2E00063F840F2F733012200210646C5B20498E4
:10D2F00040F05AF840F265230922074608210598B4
:10D3000040F052F8104AB2FBF8F308FB132202B1C6
:10D3100001332361237DC3F38002AA420AD066F35E
:10D32000820323756B1E594260684FF00002594119
:10D3300009F028FF237D0E2067F3C303237506B091
:10D34000BDE8F0819828090020A107002DE9F041EF
:10D3500086B0084611461A4603AB01932D4B009345
:10D3600003233FF0EEFF2C49182041F047FB2B4BE5
:10D37000059ED3F8A831DDE903870446002B47D08A
:10D380000FF006F980F00105EDB204F115030093EA
:10D3900000222B464FF42371404609F06FFE217D99
:10D3A00060600022C1F3800109F0ECFE04F1160375
:10D3B000009301222B4640F2BD31384609F05EFE53
:10D3C000227DA060B0F10E0318BF012363F3410278
:10D3D0009307227503D50022114609F0D3FE04F10C
:10D3E0001703009301222B464FF46C71304609F06D
:10D3F00045FE05232361237DE06023F00D030E2805
:10D4000018BF43F001032046237506B0BDE8F08144
:10D410000125BAE7B8280900E4610800946B0020F0
:10D420002DE9F04F0D468DB055F8044B06462046C9
:10D4300017463AF0C1FE20463AF0D1FE08AB019300
:10D440004A4B009329460423701E3A4615F02AFCE5
:10D45000062205A9089819F07BF99DF81C100022F6
:10D46000402015F04BFD099B04930546069B0A9945
:10D47000B3FBF0F303AA04A8039346F0F1FF049E64
:10D48000039B6E435D4304960395002D4BD0237D93
:10D49000DF0704D436484FF46C7133F01FFD980752
:10D4A000DDF814A0DDF82C90276940D4554406EB34
:10D4B0000A0835445FFA89F64FF0080B4FF0000A6E
:10D4C000237D990703D5A068F1093CF0A5FF217DD4
:10D4D0000A0735D4384625F07FFD217D606881F04C
:10D4E0000401C1F380013CF097FF0DF10B01E068EE
:10D4F0003CF079FF9DF80B30217D43EA4A0A0B0787
:10D500002BD4384625F068FD217D6068C1F3800189
:10D510003CF082FF7600BBF1010BF6B2D0D108F8E7
:10D5200001AB4545C6D10E200DB0BDE8F08FA06817
:10D5300000213CF071FF0028B8D0052033F08AFCB0
:10D54000C1F3800181F00101606801F001013CF04C
:10D5500063FF384625F040FDC7E76068C1F38001EE
:10D560003CF05AFF384625F037FDD3E7B42A0900CE
:10D57000320608002DE9F04F0D468BB055F8044BEC
:10D580000646204617463AF017FE20463AF027FE98
:10D5900007AB0193434B0093294603233A46701E81
:10D5A00015F080FB052204A9079819F0D1F89DF821
:10D5B00018100022402015F0A1FC089B039305469B
:10D5C000059B0999B3FBF0F302AA03A8029346F066
:10D5D00047FF039B029A6B43554303930295002D2B
:10D5E0005CD0227D920704D42F4840F2BD3133F045
:10D5F00075FC049AD4F810A002EB03084FF0000960
:10D6000098F80070B9F1000F0AD1A068F9093CF050
:10D6100003FF064648B1052033F01CFCD846EFE76F
:10D620000026A068F9093CF0F7FE217D0B0708F100
:10D63000010B19D4504625F0CFFC217D606881F0A4
:10D640000401C1F380013CF0E7FE504625F0C4FC24
:10D65000217D6068C1F380013CF0DEFE0136082EBA
:10D6600018D07F00FFB2DCE7C1F3800181F0010137
:10D6700001F0010160683CF0CFFE504625F0ACFCA3
:10D68000217D6068C1F380013CF0C6FE504625F064
:10D69000A3FCE3E709F101094D45BFD10E200BB012
:10D6A000BDE8F08FD42A0900320608002DE9F04FBA
:10D6B0000D4697B055F8044B0646204617463AF0FB
:10D6C0007BFD20463AF08BFD10AB0193614B00933C
:10D6D00029460623701E3A4615F0E4FA05220DA9E4
:10D6E000109819F035F89DF83C100022402015F0F4
:10D6F00005FC129B1399099306460E9BB3FBF0F3AE
:10D7000008AA09A8089346F0ABFE06220AA91198B8
:10D7100019F01EF89DF830100022402015F0EEFBA5
:10D72000149B1599079305460B9BB3FBF0F306AAD0
:10D7300007A8069346F094FE089A099B069973433E
:10D740005643079A09936A434D43AE42089607929F
:10D75000069502D0404833F0B9FB002E75D00D99E4
:10D76000C8180390207D850706D4CD1825B140F256
:10D77000BD313A4833F0B2FB0A9DC00705EB020AFF
:10D7800005D4BAF1000F02D04FF46C71F1E7CF5C11
:10D79000A068D4F810B0F9093CF03EFE00283AD059
:10D7A000052033F057FB7F00FFB2A068F9093CF079
:10D7B00033FE217D0A0732D4584625F00DFC217D29
:10D7C000606881F00401C1F380013CF025FE0DF199
:10D7D0001701E0683CF007FE9DF81730217D43EA11
:10D7E00049090B0728D4584625F0F6FB217D6068CF
:10D7F000C1F380013CF010FE0135082DD3D10AF8A9
:10D80000089008F1010846451FD0039B002513F836
:10D810000870A946C9E7054680468146C9E7C1F3B5
:10D82000800181F00101606801F001013CF0F4FD2C
:10D83000584625F0D1FBCAE76068C1F380013CF08F
:10D84000EBFD584625F0C8FBD6E70E2017B0BDE823
:10D85000F08F00BF842A0900810108003206080009
:10D860002DE9F04F0D4687B00021924622F062FF6D
:10D8700004460021284622F05DFF2379662B02D062
:10D880000379662B02D1C84833F020FB00230390B4
:10D8900008208DF817303FF0BCFA074608203FF00B
:10D8A000B8FA064608203FF0B4FA0399CDE90060C3
:10D8B00005463B460DF11702204646F01DFB039935
:10D8C00050B938460EF0ACFC30460EF0A9FC2846A4
:10D8D0000EF0A6FCB548D7E70AF1FF3A9DF817000D
:10D8E000D4F81C90D1F81C802279BAF1030F05D826
:10D8F000DFE81AF0E901BD0398053B08AA46B346E4
:10D900002379D4F81C90D1F81C80422B40F0C180C0
:10D910000A79422A3DD1394646F09BFCC269044649
:10D920000020134698F800C099F8001001EA0C0195
:10D9300003F8011BDAF80410D4F810C0DBF804E097
:10D9400003918844991A8C45F144EBD8DBF8001018
:10D95000DAF800200CFB1E11894403990CFB1122FC
:10D960009044E2680130904211D338460EF058FCE2
:10D9700030460EF055FC28460EF052FC204607B00B
:10D98000BDE8F08F5A461C46D3469246B8E71A4681
:10D99000C7E7622A28D13946682246F05AFCC16995
:10D9A00004460023002298F900C099F8000000EA1C
:10D9B0000C0021F8020B2069DBF804E0DAF804C05F
:10D9C00001328242F144E044EDD3DBF8002000FB59
:10D9D0001E229144DAF8002000FB1C229044E268E9
:10D9E00001339342DED3C0E7482A27D1394646F0B7
:10D9F00030FCC169044600230022B8F800C099F841
:10DA0000000000EA0C0021F8020B2069DBF804E0BA
:10DA1000DAF804C001328242F144E044EDD3DBF88D
:10DA2000002000FB1E229144DAF8002000FB1C229B
:10DA30009044E26801339342DED396E7682A41F0CE
:10DA40003782394646F005FCC169044600230022AE
:10DA5000B8F800C099F8000000EA0C0021F8020BA9
:10DA60002069DBF804E0DAF804C001328242F144B4
:10DA7000E044EDD3DBF8002000FB1E229144DAF8ED
:10DA8000002000FB1C229044E26801339342DED365
:10DA90006BE7622B40F08C800A79622A2CD13946E0
:10DAA00046F0D7FBC26904460020134698F800C030
:10DAB00099F8001001EA0C0103F8011BDAF80410D0
:10DAC000D4F810C0DBF804E003918844991A61454A
:10DAD000F144EBD3DBF80010DAF800200CFB1E1148
:10DAE000894403990CFB11229044E2680130904272
:10DAF000BFF43BAF1A46D8E7482A27D1394646F04B
:10DB0000A8FBC169044600230022B8F800C099F9B7
:10DB1000000000EA0C0021F8020B2069DBF804E0A9
:10DB2000DAF804C001328242F144E044EDD3DBF87C
:10DB3000002000FB1E229144DAF8002000FB1C228A
:10DB40009044E26801339342DED30EE7682A0B4625
:10DB500021467FF417AF394646F07BFBC169044686
:10DB600000230022B8F800C099F9000000EA0C0078
:10DB700021F8020B2069DBF804E0DAF804C0013276
:10DB80008242F144E044EDD3DBF8002000FB1E228A
:10DB90009144DAF8002000FB1C229044E268013333
:10DBA0009342DED3E1E600BF7AFA0700C3F907002B
:10DBB000482B57D10A79482A27D1394646F049FBE4
:10DBC000C169044600230022B8F800C0B9F800007B
:10DBD00000EA0C0021F8020B2069DBF804E0DAF817
:10DBE00004C001328242F144E044EDD3DBF800206E
:10DBF00000FB1E229144DAF8002000FB1C22904416
:10DC0000E26801339342DED3AFE6682A0B46214631
:10DC10007FF4B8AE394646F01CFBC16904460023C8
:10DC20000022B8F800C0B9F8000000EA0C0021F8A2
:10DC3000020B2069DBF804E0DAF804C0013282420A
:10DC4000F144E044EDD3DBF8002000FB1E229144B8
:10DC5000DAF8002000FB1C229044E2680133934272
:10DC6000DED382E6682B41F023810A79682A0B46CD
:10DC700021467FF487AE394646F0EBFAC169044687
:10DC800000230022B8F800C0B9F8000000EA0C0038
:10DC900021F8020B2069DBF804E0DAF804C0013255
:10DCA0008242F144E044EDD3DBF8002000FB1E2269
:10DCB0009144DAF8002000FB1C229044E268013312
:10DCC0009342DED351E6AA46B3462379D4F81C909A
:10DCD000D1F81C80422B40F0B5800A79422A31D11C
:10DCE000394646F0B6FAC26904460020134698F851
:10DCF00000C099F8001041EA0C0103F8011BDAF8A2
:10DD00000410D4F810C0DBF804E003918844991A99
:10DD10006145F144EBD3DBF80010DAF800200CFB8E
:10DD20001E11894403990CFB11229044E2680130D2
:10DD30009042BFF41AAE1A46D8E75A461C46D3465C
:10DD40009246C2E7622A28D13946682246F081FA13
:10DD5000C16904460023002298F900C099F8000028
:10DD600040EA0C0021F8020B2069DBF804E0DAF845
:10DD700004C001328242F144E044EDD3DBF80020DC
:10DD800000FB1E229144DAF8002000FB1C22904484
:10DD9000E26801339342DED3E7E5482A27D13946CA
:10DDA00046F057FAC169044600230022B8F800C0C3
:10DDB00099F8000040EA0C0021F8020B2069DBF81A
:10DDC00004E0DAF804C001328242F144E044EDD3C9
:10DDD000DBF8002000FB1E229144DAF8002000FB53
:10DDE0001C229044E26801339342DED3BDE5682AE9
:10DDF00041F05E80394646F02CFAC16904460023A2
:10DE00000022B8F800C099F8000040EA0C0021F8A0
:10DE1000020B2069DBF804E0DAF804C00132824228
:10DE2000F144E044EDD3DBF8002000FB1E229144D6
:10DE3000DAF8002000FB1C229044E2680133934290
:10DE4000DED392E5622B40F087800A79622A2CD1DA
:10DE5000394646F0FEF9C26904460020134698F898
:10DE600000C099F8001041EA0C0103F8011BDAF830
:10DE70000410D4F810C0DBF804E003918844991A28
:10DE80006145F144EBD3DBF80010DAF800200CFB1D
:10DE90001E11894403990CFB11229044E268013061
:10DEA0009042BFF462AD1A46D8E7482A27D13946D6
:10DEB00046F0CFF9C169044600230022B8F800C03B
:10DEC00099F9000040EA0C0021F8020B2069DBF808
:10DED00004E0DAF804C001328242F144E044EDD3B8
:10DEE000DBF8002000FB1E229144DAF8002000FB42
:10DEF0001C229044E26801339342DED335E5682A60
:10DF00000B4621467FF419AF394646F0A2F9C169A4
:10DF1000044600230022B8F800C099F9000040EA46
:10DF20000C0021F8020B2069DBF804E0DAF804C0E9
:10DF300001328242F144E044EDD3DBF8002000FBE3
:10DF40001E229144DAF8002000FB1C229044E26873
:10DF500001339342DED308E5482B57D10A79482A8A
:10DF600027D1394646F075F9C169044600230022DD
:10DF7000B8F800C0B9F8000040EA0C0021F8020B24
:10DF80002069DBF804E0DAF804C001328242F1448F
:10DF9000E044EDD3DBF8002000FB1E229144DAF8C8
:10DFA000002000FB1C229044E26801339342DED340
:10DFB000DBE4682A0B4621467FF4BFAE394646F0C3
:10DFC00048F9C169044600230022B8F800C0B9F836
:10DFD000000040EA0C0021F8020B2069DBF804E0A5
:10DFE000DAF804C001328242F144E044EDD3DBF8B8
:10DFF000002000FB1E229144DAF8002000FB1C22C6
:10E000009044E26801339342DED3AEE4682B40F0E3
:10E010004F870A79682A0B4621467FF48EAE39462F
:10E0200046F017F9C169044600230022B8F800C081
:10E03000B9F8000040EA0C0021F8020B2069DBF877
:10E0400004E0DAF804C001328242F144E044EDD346
:10E05000DBF8002000FB1E229144DAF8002000FBD0
:10E060001C229044E26801339342DED37DE4AA4649
:10E07000B3462379D4F81C90D1F81C80422B40F091
:10E08000B7800A79422A31D1394646F0E2F8C269AE
:10E0900004460020134698F800C099F8001081EA61
:10E0A0000C0103F8011BDAF80410D4F810C0DBF8F7
:10E0B00004E003918844991A6145F144EBD3DBF8FD
:10E0C0000010DAF800200CFB1E11894403990CFBA8
:10E0D00011229044E26801309042BFF446AC1A46E7
:10E0E000D8E75A461C46D3469246C2E7622A28D150
:10E0F0003946682246F0ADF8C16904460023002283
:10E1000098F900C099F8000080EA0C0021F8020B91
:10E110002069DBF804E0DAF804C001328242F144FD
:10E12000E044EDD3DBF8002000FB1E229144DAF836
:10E13000002000FB1C229044E26801339342DED3AE
:10E1400013E4482A28D1394646F083F8C1690446C9
:10E1500000230022B8F800C099F8000080EA0C0003
:10E1600021F8020B2069DBF804E0DAF804C0013280
:10E170008242F144E044EDD3DBF8002000FB1E2294
:10E180009144DAF8002000FB1C229044E26801333D
:10E190009342DED3FFF7E9BB682A40F0898639460F
:10E1A00046F057F8C169044600230022B8F800C0C1
:10E1B00099F8000080EA0C0021F8020B2069DBF8D6
:10E1C00004E0DAF804C001328242F144E044EDD3C5
:10E1D000DBF8002000FB1E229144DAF8002000FB4F
:10E1E0001C229044E26801339342DED3FFF7BDBBAB
:10E1F000622B40F089800A79622A2CD1394646F098
:10E2000028F8C26904460020134698F800C099F81F
:10E21000001081EA0C0103F8011BDAF80410D4F8AD
:10E2200010C0DBF804E003918844991A6145F14479
:10E23000EBD3DBF80010DAF800200CFB1E11894448
:10E2400003990CFB11229044E26801309042BFF424
:10E250008CAB1A46D8E7482A28D1394645F0F9FF51
:10E26000C169044600230022B8F800C099F90000F3
:10E2700080EA0C0021F8020B2069DBF804E0DAF8F0
:10E2800004C001328242F144E044EDD3DBF80020C7
:10E2900000FB1E229144DAF8002000FB1C2290446F
:10E2A000E26801339342DED3FFF75FBB682A0B4677
:10E2B00021467FF416AF394645F0CBFFC1690446CD
:10E2C00000230022B8F800C099F9000080EA0C0091
:10E2D00021F8020B2069DBF804E0DAF804C001320F
:10E2E0008242F144E044EDD3DBF8002000FB1E2223
:10E2F0009144DAF8002000FB1C229044E2680133CC
:10E300009342DED3FFF731BB482B59D10A79482A13
:10E3100028D1394645F09DFFC169044600230022FB
:10E32000B8F800C0B9F8000080EA0C0021F8020B30
:10E330002069DBF804E0DAF804C001328242F144DB
:10E34000E044EDD3DBF8002000FB1E229144DAF814
:10E35000002000FB1C229044E26801339342DED38C
:10E36000FFF703BB682A0B4621467FF4BAAE394655
:10E3700045F06FFFC169044600230022B8F800C0D1
:10E38000B9F8000080EA0C0021F8020B2069DBF8E4
:10E3900004E0DAF804C001328242F144E044EDD3F3
:10E3A000DBF8002000FB1E229144DAF8002000FB7D
:10E3B0001C229044E26801339342DED3FFF7D5BAC2
:10E3C000682B40F075850A79682A0B4621467FF450
:10E3D00088AE394645F03DFFC1690446002300225E
:10E3E000B8F800C0B9F8000080EA0C0021F8020B70
:10E3F0002069DBF804E0DAF804C001328242F1441B
:10E40000E044EDD3DBF8002000FB1E229144DAF853
:10E41000002000FB1C229044E26801339342DED3CB
:10E42000FFF7A3BA422A40F0A8800B79422B28D1EB
:10E43000394645F00EFFC26904460020134698F89D
:10E4400000C099F8001001FA0CF103F8011BD4F890
:10E4500010C0D6F804A0D5F804E0991A6145D1445B
:10E46000F044ECD32A6831680CFB1E229044E26829
:10E4700001300CFB1A1190428944BFF476AA1A4667
:10E48000DCE7622B27D16822394645F0E2FE0446DC
:10E49000C0690023002298F900C099F8001001FA21
:10E4A0000CF120F8021B2169D6F804E0D5F804C06D
:10E4B00001328A42F144E044EDD3326801FB1E226E
:10E4C00091442A6801FB1C229044E2680133934284
:10E4D000E0D3FFF74ABA482B27D11A46394645F010
:10E4E000B8FE0446C06900230022B8F800C099F8BD
:10E4F000001001FA0CF120F8021B2169D6F804E0A3
:10E50000D5F804C001328A42F144E044EDD33268C8
:10E5100001FB1E2291442A6801FB1C229044E26800
:10E5200001339342E0D3FFF720BA6822394645F021
:10E5300090FE0446C06900230022B8F900C099F893
:10E54000001001FA0CF120F8021B2169D6F804E052
:10E55000D5F804C001328A42F144E044EDD3326878
:10E5600001FB1E2291442A6801FB1C229044E268B0
:10E5700001339342E0D3FFF7F8B9622A40F0A88054
:10E580000B79422B27D16822394645F062FE0446BA
:10E59000C0690023002298F800C099F9001001FA20
:10E5A0000CF120F8021B2169D6F804E0D5F804C06C
:10E5B00001328A42F144E044EDD3326801FB1E226D
:10E5C00091442A6801FB1C229044E2680133934283
:10E5D000E0D3FFF7CAB9622B28D1394645F039FE9E
:10E5E000C26904460020134698F900C099F900104A
:10E5F00001FA0CF103F8011BD4F810C0D6F804A0FE
:10E60000D5F804E0991A6145D144F044ECD32A6866
:10E6100031680CFB1E229044E26801300CFB1A1199
:10E6200090428944BFF4A1A91A46DCE7482B27D1C0
:10E630001A46394645F00DFE0446C0690023002203
:10E64000B8F800C099F9001001FA0CF120F8021B8B
:10E650002169D6F804E0D5F804C001328A42F144B9
:10E66000E044EDD3326801FB1E2291442A6801FB8D
:10E670001C229044E26801339342E0D3FFF775B95E
:10E680006822394645F0E5FD0446C06900230022B2
:10E69000B8F900C099F9001001FA0CF120F8021B3A
:10E6A0002169D6F804E0D5F804C001328A42F14469
:10E6B000E044EDD3326801FB1E2291442A6801FB3D
:10E6C0001C229044E26801339342E0D3FFF74DB936
:10E6D000482A40F0A7800B79422B26D1394645F0D5
:10E6E000B8FD0446C0690023002298F800C0B9F8BC
:10E6F000001001FA0CF120F8021B2169D6F804E0A1
:10E70000D5F804C001328A42F144E044EDD33268C6
:10E7100001FB1E2291442A6801FB1C229044E268FE
:10E7200001339342E0D3FFF720B9622B29D11A4677
:10E73000394645F08EFDC26904460020134698F91B
:10E7400000C099F9001001FA0CF103F8011BD4F88C
:10E7500010C0D6F804A0D5F804E0991A6145D14458
:10E76000F044ECD32A6831680CFB1E229044E26826
:10E7700001300CFB1A1190428944BFF4F6A81A46E6
:10E78000DCE7482B26D1394645F063FD0446C069D5
:10E7900000230022B8F800C0B9F8001001FA0CF10B
:10E7A00020F8021B2169D6F804E0D5F804C0013234
:10E7B0008A42F144E044EDD3326801FB1E229144C9
:10E7C0002A6801FB1C229044E26801339342E0D3A3
:10E7D000FFF7CBB86822394645F03BFD0446C069D7
:10E7E00000230022B8F900C0B9F8001001FA0CF1BA
:10E7F00020F8021B2169D6F804E0D5F804C00132E4
:10E800008A42F144E044EDD3326801FB1E22914478
:10E810002A6801FB1C229044E26801339342E0D352
:10E82000FFF7A3B8682A40F043830B79422B39469F
:10E8300025D145F00EFD0446C0690023002298F85A
:10E8400000C0B9F9001001FA0CF120F8021B21698F
:10E85000D6F804E0D5F804C001328A42F144E0441D
:10E86000EDD3326801FB1E2291442A6801FB1C2271
:10E870009044E26801339342E0D3FFF776B8622B0D
:10E8800025D145F0E6FC0446C0690023002298F932
:10E8900000C0B9F9001001FA0CF120F8021B21693F
:10E8A000D6F804E0D5F804C001328A42F144E044CD
:10E8B000EDD3326801FB1E2291442A6801FB1C2221
:10E8C0009044E26801339342E0D3FFF74EB8482BFF
:10E8D00025D145F0BEFC0446C06900230022B8F9EA
:10E8E00000C0B9F8001001FA0CF120F8021B2169F0
:10E8F000D6F804E0D5F804C001328A42F144E0447D
:10E90000EDD3326801FB1E2291442A6801FB1C22D0
:10E910009044E26801339342E0D3FFF726B845F014
:10E9200098FC0446C06900230022B8F900C0B9F978
:10E93000001001FA0CF120F8021B2169D6F804E05E
:10E94000D5F804C001328A42F144E044EDD3326884
:10E9500001FB1E2291442A6801FB1C229044E268BC
:10E9600001339342E0D3FFF700B8422A40F0A88079
:10E970000B79422B28D1394645F06BFCC26904461D
:10E980000020134698F800C099F8001041FA0CF1E5
:10E9900003F8011BD4F810C0D6F804A0D5F804E0A1
:10E9A000991A8C45D144F044ECD82A6831680CFBA4
:10E9B0001E229044E26801300CFB1A1190428944F7
:10E9C000BEF4D3AF1A46DCE7622B27D16822394662
:10E9D00045F03FFC0446C0690023002298F900C0BE
:10E9E00099F8001041FA0CF120F8021B2169D6F8C1
:10E9F00004E0D5F804C001328A42F144E044EDD38A
:10EA0000326801FB1E2291442A6801FB1C229044BB
:10EA1000E26801339342E0D3FEF7A7BF482B27D12A
:10EA20001A46394645F015FC0446C0690023002209
:10EA3000B8F800C099F8001041FA0CF120F8021B58
:10EA40002169D6F804E0D5F804C001328A42F144C5
:10EA5000E044EDD3326801FB1E2291442A6801FB99
:10EA60001C229044E26801339342E0D3FEF77DBF5D
:10EA70006822394645F0EDFB0446C06900230022B8
:10EA8000B8F900C099F8001041FA0CF120F8021B07
:10EA90002169D6F804E0D5F804C001328A42F14475
:10EAA000E044EDD3326801FB1E2291442A6801FB49
:10EAB0001C229044E26801339342E0D3FEF755BF35
:10EAC000622A40F0A8800B79422B27D16822394670
:10EAD00045F0BFFB0446C0690023002298F800C03F
:10EAE00099F9001041FA0CF120F8021B2169D6F8BF
:10EAF00004E0D5F804C001328A42F144E044EDD389
:10EB0000326801FB1E2291442A6801FB1C229044BA
:10EB1000E26801339342E0D3FEF727BF622B28D18E
:10EB2000394645F096FBC26904460020134698F921
:10EB300000C099F9001041FA0CF103F8011BD4F858
:10EB400010C0D6F804A0D5F804E0991A8C45D14439
:10EB5000F044ECD82A6831680CFB1E229044E2682D
:10EB600001300CFB1A1190428944BEF4FEAE1A46E5
:10EB7000DCE7482B27D11A46394645F06AFB0446A4
:10EB8000C06900230022B8F800C099F9001041FACA
:10EB90000CF120F8021B2169D6F804E0D5F804C076
:10EBA00001328A42F144E044EDD3326801FB1E2277
:10EBB00091442A6801FB1C229044E268013393428D
:10EBC000E0D3FEF7D2BE6822394645F042FB044648
:10EBD000C06900230022B8F900C099F9001041FA79
:10EBE0000CF120F8021B2169D6F804E0D5F804C026
:10EBF00001328A42F144E044EDD3326801FB1E2227
:10EC000091442A6801FB1C229044E268013393423C
:10EC1000E0D3FEF7AABE482A40F0A7800B79422B2A
:10EC200026D1394645F015FB0446C0690023002271
:10EC300098F800C0B9F8001041FA0CF120F8021B56
:10EC40002169D6F804E0D5F804C001328A42F144C3
:10EC5000E044EDD3326801FB1E2291442A6801FB97
:10EC60001C229044E26801339342E0D3FEF77DBE5C
:10EC7000622B29D11A46394645F0EBFAC26904469F
:10EC80000020134698F900C099F9001041FA0CF1E0
:10EC900003F8011BD4F810C0D6F804A0D5F804E09E
:10ECA000991A8C45D144F044ECD82A6831680CFBA1
:10ECB0001E229044E26801300CFB1A1190428944F4
:10ECC000BEF453AE1A46DCE7482B26D1394645F050
:10ECD000C0FA0446C06900230022B8F800C0B9F8A1
:10ECE000001041FA0CF120F8021B2169D6F804E06B
:10ECF000D5F804C001328A42F144E044EDD33268D1
:10ED000001FB1E2291442A6801FB1C229044E26808
:10ED100001339342E0D3FEF728BE6822394645F01E
:10ED200098FA0446C06900230022B8F900C0B9F877
:10ED3000001041FA0CF120F8021B2169D6F804E01A
:10ED4000D5F804C001328A42F144E044EDD3326880
:10ED500001FB1E2291442A6801FB1C229044E268B8
:10ED600001339342E0D3FEF700BE682A40F0A08052
:10ED70000B79422B394625D145F06BFA0446C06920
:10ED80000023002298F800C0B9F9001041FA0CF1F4
:10ED900020F8021B2169D6F804E0D5F804C001323E
:10EDA0008A42F144E044EDD3326801FB1E229144D3
:10EDB0002A6801FB1C229044E26801339342E0D3AD
:10EDC000FEF7D3BD622B25D145F043FA0446C06956
:10EDD0000023002298F900C0B9F9001041FA0CF1A3
:10EDE00020F8021B2169D6F804E0D5F804C00132EE
:10EDF0008A42F144E044EDD3326801FB1E22914483
:10EE00002A6801FB1C229044E26801339342E0D35C
:10EE1000FEF7ABBD482B25D145F01BFA0446C0696F
:10EE200000230022B8F900C0B9F8001041FA0CF133
:10EE300020F8021B2169D6F804E0D5F804C001329D
:10EE40008A42F144E044EDD3326801FB1E22914432
:10EE50002A6801FB1C229044E26801339342E0D30C
:10EE6000FEF783BD45F0F5F90446C0690023002292
:10EE7000B8F900C0B9F9001041FA0CF120F8021BF2
:10EE80002169D6F804E0D5F804C001328A42F14481
:10EE9000E044EDD3326801FB1E2291442A6801FB55
:10EEA0001C229044E26801339342E0D3FEF75DBD3B
:10EEB0000024FEF75ABD00BF10B50C4C0C4B227855
:10EEC00012B19A7AFF2A0FD10A4A0B481A60F7F753
:10EED00047F80A48F7F744F8094B084A0649044836
:10EEE00002F042FB01232370014810BDB8770020D7
:10EEF000F0690020986008004C6108004461080037
:10EF0000A0860100032A05D11E2914BF0449054922
:10EF10003FF09ABF1E2914BF03490449F8E700BF18
:10EF20007E90070083900700E5900700DA900700C5
:10EF3000054A0648002303F5C0710133082B42F847
:10EF40002100F8D1704700BF000001403546526EE5
:10EF500030B587B00C460592D1E9012317490493D7
:10EF60005528CDE90212236809D054F8042C02A9CF
:10EF700018461CF017F9A4F1080007B030BD184678
:10EF8000009319F025FE827B009B82B100EB82008A
:10EF900002A90569019318460422A8470090F6F7D4
:10EFA000D1FFDDE9000310B120602046E5E71846F7
:10EFB0003FF0FEF90146024831F07CFFA818080036
:10EFC000530A080070B586B0084611461A4602ABCF
:10EFD00001930F4B009304233EF0B3F902984FF4D2
:10EFE0008F6149F018FB40F279410546039849F0DA
:10EFF00012FB084906460C203FF007FD049B3246F1
:10F000002946044602F0B0FA204606B070BD00BFA3
:10F01000642A090098600800F0B50C468DB054F8D9
:10F02000045B0646A87A174639F0AFF8284639F04F
:10F03000DDF808AB01931D4B009321460423701E9D
:10F040003A4613F02FFE062205A9099817F080FB17
:10F050009DF81C100022402013F050FF069B0B99D6
:10F06000B3FBF0F30446049304AA0A9B039303A89A
:10F0700045F0F6F9049E40F27322012130463EF03D
:10F080009FF9039A06FB04F362430392049353B17E
:10F09000059928460A44BDF8201002F08BFB10B1F8
:10F0A000404231F0D7FE0E200DB0F0BD442A0900D9
:10F0B000F0B50C468DB054F8045B0646A87A1746A6
:10F0C00039F063F8284639F091F808AB01931F4BEB
:10F0D0000093214604233A46701E13F0E3FD0522F7
:10F0E00005A9099817F034FB9DF81C100022402058
:10F0F00013F004FF069B0B99B3FBF0F30446049353
:10F1000004AA0A9B039303A845F0AAF9039A049B57
:10F11000624363430392049353B99DF82010284639
:10F1200002F002FB78B96FF01200404231F092FE1B
:10F13000012000900598BDF8201002442846F5F7FC
:10F1400009F80028F1D10E200DB0F0BD242A0900E5
:10F150002DE9F0410C4694B054F8046B0546B07AA2
:10F16000174639F012F8304639F040F80DAB0193EC
:10F17000374B00933A4607232146681E13F092FD51
:10F1800005220AA90E9817F0E3FA9DF83010002224
:10F19000402013F0B3FE0B9B1199B3FBF0F305462F
:10F1A000069306AA109B059305A845F059F9062277
:10F1B00007A90F9817F0CCFA9DF8241000224020E0
:10F1C00013F09CFE089B1399B3FBF0F304460493E1
:10F1D00004AA129B039303A845F042F9049F40F24E
:10F1E0005232384601213EF0EBF8059A069BDDF8D5
:10F1F0001C806A436B43039D059265437C430693E1
:10F20000BDF834700395049493B99DF834103046DA
:10F2100002F08AFAC8B13CB1234608EB0502394630
:10F22000304602F0C7FA68B90E2014B0BDE8F0818C
:10F23000002100910A9930460A443946F4F78AFFC2
:10F240000028E8D0404231F005FE6FF01200F9E7E7
:10F25000EC290900F0B50C4687B054F8045B06466B
:10F26000687A174638F08BFF284638F0BFFF02ABAC
:10F270000193214B00932146701E04233A4613F05C
:10F2800011FD40F203430122002103983EF08CF867
:10F2900040F2F73301220021064604983EF084F83C
:10F2A00040F2652304460922059808213EF07CF8C7
:10F2B000C0B2082802D0052031F0CCFD6B6802985E
:10F2C0001F689B68984228BF1846FDF7D1FEF6B22A
:10F2D000E4B2C7F824055EB1002C0CBF0221032163
:10F2E0006B680022186845F0E8F80E2007B0F0BD02
:10F2F000A11B18BF0121F3E7542B09002DE9F04FA2
:10F3000089B0084611461A4604AB0193774B009327
:10F3100004233EF016F84FF42371049849F07BF96A
:10F3200040F2BD310746059849F07DF94FF46C7104
:10F330000446069849F077F9064618B914B96C489E
:10F3400031F0C4FD6B490C203FF05FFB9DF81C3091
:10F35000FF220546427223B1674840F2433131F043
:10F360006DFD4360654B1B782BB9654BD3F80035B9
:10F3700013F00F0305D0634BD3F800351B0711D1F1
:10F380000123614A02EB03136B6097F80480D3F802
:10F3900008A085F80980404601F0E2FC24B9FF246A
:10F3A000AC7206E05948CBE72479AC72204601F0F4
:10F3B000D7FC26B33679EE72304601F0D1FCD5F891
:10F3C00004B0534F9BF80490242303FB09731B7F65
:10F3D00063B95046FDF74CFE0290B9F1000F11D110
:10F3E000B0F1206F02D0B0F1A05F0ED16B7AFF2B8D
:10F3F00002D0284602F022FA052031F02BFDFF262C
:10F40000EE72DCE7B9F1010FF0D1242202FB09F220
:10F41000B8180021DBF800A041604046B95023F045
:10F4200005FDB8F11F0F8BBF08F01F024246394996
:10F430004FF0A04102F5E0720120FF2C41F82200BC
:10F440004AD0204623F0F2FC204623F0CBFCFF2ECE
:10F4500045D000213046039623F0B4FC039A2421C2
:10F4600001FB09F3F918039381F82160FF2681F865
:10F4700020600221CAF86015029BCAF80885CAF804
:10F480000C45CAF8102500221146CAF8243550460A
:10F4900045F013F8039BCAF8C065FA5807210AB370
:10F4A0004022CAF80423CAF80015DBF8000040F334
:10F4B0000730F3F7F1FCDBF8000040F3073036F0DB
:10F4C00036FF242303FB097700237B77284601239B
:10F4D0003B7709B0BDE8F08F4FF0FF34B7E74FF04E
:10F4E000FF32BCE7CAF80015EBE700BF942B090018
:10F4F000510608007C600800B70B0800D577002093
:10F5000000F0024000300240742B0900A9090800F5
:10F510006C6A00200003005010B50446407A38F0B1
:10F520002EFE63681B68D3F82435B3F1805F23D0C7
:10F5300013D8B3F1006F21D00BD8B3F1007F1FD0E7
:10F540001248B3F1806F18BF0020400040F0010066
:10F5500010BD0F48B3F1206FF5E7B3F1804F11D024
:10F5600006D8B3F1A05F0FD00A48B3F1005FEAE715
:10F570000948B3F1004FE6E70848E6E70848E4E742
:10F580000848E2E70848E0E70848DEE790D00300D3
:10F590000024F40080841E0000127A0040420F0014
:10F5A00020A1070048E8010000093D000048E801EB
:10F5B000F0B50C468DB054F8045B0646687A1746E1
:10F5C00038F0DDFD284638F011FE08AB01931A4BE8
:10F5D0000093214604233A46701E13F063FB062273
:10F5E00005A9089817F0B4F89DF81C1000224020D7
:10F5F00013F084FC099B0A9904930446069BB3FB11
:10F60000F0F303AA04A8039344F02AFF0499039B90
:10F61000614303FB04F20491039252B105989DF8F3
:10F620002C300144284639F0ADF810B9052031F0EE
:10F6300011FC0E200DB0F0BD1C2B0900F0B50C46DE
:10F640008BB054F8045B0646687A174638F097FD8D
:10F65000284638F0CBFD07AB0193194B00932146A8
:10F6600003233A46701E13F01DFB052204A90798D8
:10F6700017F06EF89DF818100022402013F03EFCA1
:10F68000089B03930446059B0999B3FBF0F302AA78
:10F6900003A8029344F0E4FE039B029A634362438F
:10F6A0000393029242B104992846194402F04EF99C
:10F6B00010B9052031F0CEFB0E200BB0F0BD00BF1D
:10F6C0003C2B0900F0B50C4693B054F8046B05468A
:10F6D000707A174638F053FD304638F087FD0CAB92
:10F6E00001932B4B009321460623681E3A4613F0E4
:10F6F000D9FA052209A90C9817F02AF89DF82C10C0
:10F700000022402013F0FAFB0E9B0F99059304464C
:10F710000A9BB3FBF0F304AA05A8049344F0A0FEEF
:10F72000062206A90D9817F013F89DF82010002264
:10F73000402013F0E3FB109B119903930546079BB0
:10F74000B3FBF0F302AA03A8029344F089FE049BE2
:10F75000039A0298059963436A4345436143AB4268
:10F76000059104930392029502D00A4831F0AEFB52
:10F7700053B10698024409980144304602F0AEF8AD
:10F7800010B9052031F066FB0E2013B0F0BD00BFAC
:10F79000EC2A0900810108002DE9F04F2DED028BC4
:10F7A00099B0084611461A460CAB0193594B009389
:10F7B0000C233DF0C6FD40F26D410D9848F033FF3B
:10F7C00040F2EE4181460C9848F02DFF40F269412D
:10F7D0008246149848F027FF4FF42C718046159804
:10F7E00048F021FF40F265410746169848F01BFF9C
:10F7F0000546BAF1000F05D1B9F1000F0DD1464809
:10F8000031F064FBD14518D0C24516D0BA4514D0AA
:10F81000824512D0B9F1000F05D0C1450DD0B945D0
:10F820000BD0A94509D0B8F1000F03D0B84504D0DA
:10F83000A84502D02FB1AF4203D140F2FE3013F001
:10F8400023FA40F26523092205210F983DF0ACFD13
:10F8500040F233434FF6FF720646012113983DF004
:10F86000A3FD109B2D4A0490934227D02C4A981A4E
:10F87000434243415B0002220121119803939623E6
:10F880003DF092FD8346129819F018F9B0EE408AC7
:10F8900048F0E9FE9DF85C30224905932C203FF0AA
:10F8A000B4F8F6B20E9B0993082E059B044607D0C8
:10F8B0001D48082240F2652131F010FB0123DAE7F0
:10F8C00005B913B1194831F0B1FA4560184D2B68EC
:10F8D000D3F8003513F00F0305D0AB68D3F800352B
:10F8E000190714D10123DE0005EBC3036360059300
:10F8F000BDF810300893184640F2334201213DF024
:10F900004BFD039B022B059B18D10A4878E70A4858
:10F9100076E700BFB42B09006BF7070064230800EB
:10F920006823080058600800400B080029050800FB
:10F9300028210020A70508009F090800BAF1000F40
:10F9400000F0F0809AF804200492B9F1000F00F062
:10F95000EC8099F804200692002F00F0E9803A79B3
:10F960000792B8F1000F00F0E68098F804200592A5
:10F97000039A1B790A93002A18BF0E220A99039250
:10F98000824A242303FB012393F82030002B40F00C
:10F99000D58047EA08035FFA8BFB09980B930DF0BB
:10F9A00093F9ABF1020C049B0B90DCF1000B4BEBD9
:10F9B0000C0B5A1C4FEA0B1B05D0184623F064FAB7
:10F9C000049823F00FFA069B581C03D00021184618
:10F9D00023F0F8F9AB590B9AC3F8242547EA08033A
:10F9E000002B18BF4BF0010B039BAA5943EA0B03F2
:10F9F000DBB2C2F86C35AB59049AC3F80C25069AF1
:10FA0000C3F8142547EA0803B3B1079B591C03D078
:10FA10000021184623F0D6F9059B5A1C05D018463C
:10FA200023F032FA059823F0DDF9AB59059AC3F8B3
:10FA30000825079AC3F810250A9A5449A85924237F
:10FA4000534301EB030B524ACC504FF48871CBF86F
:10FA5000042044F01BFDA8594FF4907144F016FDAA
:10FA6000A8594FF4927144F011FDA8594FF4A271B6
:10FA700044F00CFDA8594FF4AC7144F007FDAB59AC
:10FA8000444AC3F80423A859032140F30730F3F78D
:10FA900003FAA85940F3073036F049FCAB59082265
:10FAA000C3F8002500250123CBE90655CBF81450F7
:10FAB0008BF82030B9F1000F45D1BAF1000F59D0C1
:10FAC0009AF8040084F8260001F04AF9B8F1000F12
:10FAD00054D098F8040084F8290001F041F9002F6F
:10FAE00050D0387984F8280001F03AF9DFED2A7A0D
:10FAF000099BA36028EE278A0023BCEEC88A84F8FD
:10FB00002530606884ED038A04F1240123F000FDB0
:10FB1000224B9842024612D1204619B0BDEC028B0E
:10FB2000BDE8F08F4FF0FF320EE74FF0FF3212E7E3
:10FB30004FF0FF3214E74FF0FF3218E7184A194927
:10FB4000194848F0DBFB08983DF063F9089B2061F9
:10FB5000C4E90535C4E9075528B9606823F05EFD9E
:10FB6000089831F039F999F8040084F8270001F079
:10FB7000F7F8A2E7FF2384F82630A7E7FF2384F8ED
:10FB80002930ACE7FF2384F82830AFE7346B00203E
:10FB9000898007001003420000007A440000AD0B8A
:10FBA0000500AD0B0DFF0700EC0B080010B51EF0B3
:10FBB00031F990F82730FF2B044628D0406823F015
:10FBC0002DFD94F8260029F04FFF94F8270029F026
:10FBD0004BFF94F8290029F047FF94F8280029F0FA
:10FBE00043FF61680B4A4FF6FF73E384238591421C
:10FBF0004FF00003C4E90433C4E90733A36103D021
:10FC00000832914203D10123034A0021D1540E202E
:10FC100010BD00BF28210020C677002010B51EF0BF
:10FC2000F9F8044690F8270038F0A3FA94ED030A97
:10FC3000DFED047AB8EE400ABDE8104080EE270AF6
:10FC40001AF056B800007A4410B51EF0E3F80446E6
:10FC500090F8270038F08DFA6368186840F3073091
:10FC6000002801DBF3F708F90023C4E90733A36197
:10FC700063681B6843F30733002B08DB5909012233
:10FC800003F01F0302FA03F3024A42F821300E2068
:10FC900010BD00BF00E100E038B52DED028B0D4630
:10FCA0001EF0B8F8044690F8270038F062FA2846AB
:10FCB00018F004FFB0EE408A48F0D5FCDFED057A7D
:10FCC00028EE278A0E20BCEEC88A84ED038ABDEC9C
:10FCD000028B38BD00007A4413B50A4C40F2811201
:10FCE00040F22B13A14218BF1346019340F2C513F3
:10FCF000009305494FF4FE7340F276223FF0B3F8CB
:10FD000002B010BD64230800BAE507002DE9F047F2
:10FD100015460E461F461EF07DF8044690F8270053
:10FD200038F027FA1DB900252846BDE8F08763683A
:10FD30001B68D3F81435013304D12E4840F26D41CD
:10FD400031F0CCF847F0A4F8DFF8B0A0804689463F
:10FD5000A3699D4238D86368186840F307300028CB
:10FD600044DA2A46314604F1100045F0EBFC94F8E1
:10FD70002530054693B1012204F1240104F110005D
:10FD800045F007FD04F12401606823F0C1FB94F8FD
:10FD9000290023F04BF8002384F8253063681B68A2
:10FDA00043F30733002B08DB5909012203F01F033B
:10FDB00002FA03F3104A42F82130002DB4D10B238C
:10FDC0003B604FF0FF35AFE747F062F8E368B0EB18
:10FDD000080061EB0901984271F10001BBD2FDF707
:10FDE00005F9DAF82830002BB2D09CE7F3F744F895
:10FDF000B7E700BF3206080000E100E0946B002086
:10FE000038B50C462046114606221D4612F012FF58
:10FE10002CB92146BDE838400120F5F75BBE2968C2
:10FE2000CB0706D411F003030DD108680F4A9042A6
:10FE300009D1012C02D00E4831F034F808463EF0CA
:10FE4000ABFA0146E6E70B4A0A40062A04D03BB962
:10FE50000A68094B9A4203D1012C01D10748EBE70C
:10FE6000BDE838400120F5F795BD00BF08F6070052
:10FE70007AF607000F0080FF7CF4070013F80700F4
:10FE8000012807B50B4606D10B68009340F61623F0
:10FE9000019302206B460146002202481BF074F8D1
:10FEA00003B000BD7CF407000146014817F03EBED8
:10FEB000780E0800014A17F07FBE00BF780E0800D8
:10FEC000014A17F079BE00BF7CF4070008B5084668
:10FED0000AB112F0E1FE21B11946BDE8084000F078
:10FEE00005B8014808BD00BF0810080070B50646F7
:10FEF000086810F003038EB00D4603D101684A4A2A
:10FF000091423DD0494C00EA0402062A05D0002B5C
:10FF100038D10268464B9A4234D1023E012E02D9B2
:10FF2000444830F0BFFF0AA91AF0EAFF06462868E5
:10FF300000EA0403062B1AD1000945F0E6F804464E
:10FF400024B90A99304645F0B7F8044668681AF0B3
:10FF5000E5FF26F0F5F801280A9D0AD131462A4628
:10FF600048F09CF9014620B9334848F0BCF9446890
:10FF7000E6E72D4910203EF041FDC0E902564460FD
:10FF80000EB070BD012E01D02C48CAE710F001045C
:10FF90000BD0411002D5002030F098FF0AA848F09D
:10FFA00067FC0AA819F0EAFDEAE701AA40F213216A
:10FFB00017F07CFA019B2BB101AA214620463DF0A7
:10FFC0001DFBDDE72868324603A916F0C1FB20B10E
:10FFD000DDE9030119F0CAFDD2E7286819F048FDF0
:10FFE0000446B8B91020CDE90A043CF012FF8DF8A0
:10FFF00034400C90286806A916F016FC04462046EA
:020000023000CC
:1000000016F0D6FD0028CCD03EF0C6F9FF2806D960
:100010000B48C1E741100AA848F01CFCEAE7C1B24E
:100020000AA848F063FBEAE7780E08000F0080FF9B
:100030007CF4070013F80700EC1308007AF60700B9
:1000400061010800F0B585B0054617460C4618F06A
:10005000BFFD6946064628461AF052FF042F0546A2
:1000600022D1A307009814D12268104B9A4210D1D4
:1000700001AA21463FF047F810B90D4830F0D6FEEE
:10008000DDE901123046521A294419F0A3FF05B0E8
:10009000F0BD014600232246304616F077FB285C6F
:1000A000400040F00100F2E70020F0E7A818080047
:1000B000DEF907002DE9F14F8F0705460C4616467D
:1000C00013D001F00F03022B19D102F0FD06012E0F
:1000D0004FEA111104D001B0BDE8F04F05F0B6B9F8
:1000E00001B0BDE8F04F04F0BFBE4968CBB22D2B84
:1000F00000F087800BD8062B0ED02C2B13D0554A3E
:100100002146284601B0BDE8F04F05F0ADB92E2BD1
:1001100000F08C809D2BF2D1002EF0D104F108026A
:10012000090A284687E0022A02D0A16804F0F2FEFC
:10013000E768002FE3D017F00309E0D17B68DAB25B
:100140008E2AB8460DD1022E4FEA132805D007F1AA
:10015000040A08F1FF3BD94515DB08F1010857F8FF
:10016000288098F80430312B2BD1022E13D1686AE5
:100170003DF0D8FB686A56226FF0020101B0BDE87D
:10018000F04F3AF01CBB5AF8041F284604F0C2FE98
:1001900009F10109DFE72846D8F8081004F0BAFE93
:1001A000012E686A09D1582202213AF008FB686AD8
:1001B00001B0BDE8F04F3DF0DFBB56226FF0020109
:1001C000DCE7322B9BD1012E686A0AD13DF0F8FAA8
:1001D000D8F80810686A090901B0BDE8F04F3DF091
:1001E000A0BA022E01D13DF0A1FBD8F80830686A10
:1001F0001B0918226FF0010101B0BDE8F04F3AF081
:100200005EBBA268002A3FF47AAF002E7FF477AF7E
:100210005168090A022907D1D3682BB1980703D185
:100220001B79AC2B3FF46BAF08327AE7002A7FF4DE
:1002300066AFA16821B901B0BDE8F04F00F00CB87D
:100240008E0703D10B79922B0A46E1D004F1080204
:10025000012166E7370108002DE9F04701F1FF3A77
:100260000546884691464FEA0A2700244FF0FF369C
:1002700017F5807F0CD1731C05D1686A4346302284
:10028000514607F065FE002444451DD1BDE8F087C6
:1002900059F8241071B18A070CD10A79222A09D1A0
:1002A00001360BD1686A47EA04033122514607F050
:1002B0004FFE26460134A7F58077D9E72846084A3D
:1002C000BDE8F04705F0D0B859F82410A64208BFA1
:1002D000896800222846FFF7EDFE0134D4E700BF0D
:1002E00036FB070001F00F03022B2DE9F04707460C
:1002F0000C4604D1BDE8F047090904F053BC0029BD
:100300005BD011F0030558D10B792C2B3FD18968B4
:1003100004F000FEE568002D4FD015F003084CD125
:100320006E68F2B28E2A2B4609D1360A05F104090D
:1003300006F1FF3AC24518DC013655F826301A7925
:10034000312A1AD19968384604F0E4FD7C6A2046C7
:100350003DF0C2FA20463DF0E5FA20465622BDE8BF
:10036000F0476FF002013AF02ABA59F8041F3846F4
:1003700004F0D0FD08F10108DCE7322A1DD19968AC
:10038000786A0222BDE8F04709093DF0B2B92D2B89
:1003900013D18C688CB163681B0A022B01D1E3680E
:1003A00033B9261D6368B5EB132F0DD3BDE8F08775
:1003B0009A07F6D11B79AC2BF3D121463846064A71
:1003C000BDE8F04705F050B856F8041F3846FFF76F
:1003D00089FF0135E6E700BFD500080070B5137846
:1003E00003F06003202B59D12D4B90885C78844218
:1003F0000ED093F83D48844250D103F63C000125CD
:100400005478203C032C49D8DFE804F005050D3072
:1004100018460025F4E7012903D1072104302FF005
:10042000D3FF012070BD012902D12FF0BDFFF8E7F5
:100430000329F6D15188847FC17001F0010282F056
:1004400001018C4218BF81776AB95B68B3F5966F7A
:10045000E7D14FF08043B322C3F81C257E22C3F8B6
:10046000202529F0D7FA2DF077FEDAE70129DCD034
:100470000329D6D10B4B1B78002BD2D00A4B1B681B
:100480000133CED0002DCCD15388002BC9D0074BDF
:10049000074A9A6603F160029A62C2E70020C1E748
:1004A000542A0020EF79002008210020946B0020BE
:1004B000402208002DE9F04741F27802002121484E
:1004C0003CF0DBFD1F4B204800211F464FF0FF0989
:1004D0004FF4E1380A464FF0080E4FF4806540F6BD
:1004E0003C0C012603F23C441C630CFB01744FF0EE
:1004F000000A83F80B90C3F804801A725A7283F8CA
:100500000AE083F825209D8683F8362062872287BB
:1005100083F80DA003F13C0AD862C3F818A09D83AC
:100520009E776284228400F140045C614C1C022CA2
:1005300003F63C0300F180004FF00101D2D1BDE889
:10054000F08700BF542A0020542900202DE9F84FDD
:100550004B79022B81468A4615D18B79022B12D119
:100560004D4F97F8266096B1BE7B86B197F86238FA
:1005700063B197F84A384BB14FF0E023D3F8F03D20
:10058000DB0700D500BE0020BDE8F88F012640F64D
:100590003C037343F91807F803909AF802304B7044
:1005A0009AF800400AEB020854444445627805D2A8
:1005B00023782344984501D3242A18D0052A0CD146
:1005C000204632F02DFB0028D6D040F63C0303FB3A
:1005D0000673A2789A7023781C446378042B38D170
:1005E00063790A2B35D123464FF0000B2AE01C46D5
:1005F000DBE743452CD29D18A84529D36B78052B02
:10060000BAD1EB7803F00303022BB5D1284632F0C0
:1006100007FB0028B0D0AB78DB091ED040F63C03C6
:1006200003FB067383F80C90AA789A73AA88C2F326
:100630000A021A8240225A8200225A841A840BF13A
:10064000010B2B4621795FFA8BF291421A78D0D8B0
:100650009C18A4EB0A0080B296E740F63C0C0CFB19
:100660000673AA8883F82490A97883F8261070422C
:10067000A98800EA0C00C2F30A022430C1F30A017F
:100680005A85384400225A8719851A8747F0EDFAAF
:100690000028D4D170E700BF542A002000220A4B62
:1006A00030B5114614460125987F1C6000B99D772E
:1006B000501C022883F8261099734FF0010203F6AC
:1006C0003C03F1D130BD00BF542A00202DE9F04792
:1006D0006F4C984694F8263099420F467AD0A27B08
:1006E0008A421BD0A2788A4200D1B9B994F8623804
:1006F0009F4272D094F84A28BA4269D094F83E28B2
:10070000BA4201D1002F63D14FF0E023D3F8F03D7E
:10071000DB0700D500BE0020BDE8F08700256E4253
:1007200026F4F86626F0030636059F424FEA165671
:100730003CD140F63C0303FB054306F12409D96A8A
:10074000A14431B106F130001FFA88F2204447F08D
:10075000B0FB40F63C0101FB0541C87AFF281ED0E2
:100760000A8F4B8FB1F834E092B29BB29A42B6BF77
:10077000C3EB4E0AA2EB030A92441FFA8AFAD6454B
:100780000AD2724540F63C012BD3A2EB0E0301FBCB
:1007900005419BB24B87F246BAF1000F46D148465D
:1007A000B9F81430B9F8163047F05FFA40F63C0358
:1007B00003FB0545AB7BBB4208D10C36A01947F0C3
:1007C000D0FA18B94146A01947F00DFB0120A3E764
:1007D0000125A4E700263546ABE740F63C06012597
:1007E000A7E702EB0E0301FB05419BB24B87F246E4
:1007F0009E451ED940F63C0101FB05419A42096B1A
:1008000001EB030C19D8AEEB0302AAEB0E0E7344F6
:100810009BB292B29BB1013B0B44002BBFD04FF077
:10082000000E013A14E0A2EB0E0292B29645FAD9FC
:10083000DEE7A3EB0E039BB2DAE752460021531E1C
:100840006344EAE78B421ED10CEB02030EF1010E6A
:10085000C645A4D093F800A08245F3D10D4B1B6888
:1008600098429CD140F63C0303FB054300224846D6
:100870005A871A8747F0F9F9074B084A9A6603F135
:1008800060029A628BE7634589D0013BDEE700BFD7
:10089000542A002008210020946B002040220800E8
:1008A00010EE103AC3F3C7517F39162982B013DC1A
:1008B000002913DB124A0A4113420DD0DFED117AF1
:1008C00030EE270A002B8DED000AA8BF9B18009977
:1008D00023EA020300EE103A02B07047DFED097A16
:1008E00030EE270A002B8DED010A019A04DB5B0034
:1008F00018BF4FF07E53EDE74FF00043EAE700BF2B
:10090000FFFF7F000000807B054B4FF0FF32072880
:1009100043F8202084BF1B1883F85020704700BF85
:10092000086A0020014608B5014830F0D7FA00BF38
:10093000C80A080042F21623984273B50E4619D031
:1009400042F27613984215D08B070FD00B4D00243E
:100950003046297801236A4616F0F8FD009848B918
:100960000134032C05F10105F2D104E00A68044BBF
:100970009A42EBD1012002B070BD00BF9B7F0800FE
:100980004019080038B50023C3714FF0FF33C3642A
:1009900005463CF0C8FB044640BBB5F87E224AF64B
:1009A00055239A4224D115490B2205F180003CF0D1
:1009B0000FFBF8B195F8802002F11803DBB2012B90
:1009C00001D9EB2A18D10E49032205F1B6003CF0FB
:1009D000FFFA48B10B49052205F1D2003CF0F8FAC4
:1009E000041E18BF01246400204638BD0424FBE720
:1009F0000324F9E70124F7E70224F5E72DE60700D1
:100A000039E607003DE6070008B5014830F038FA3E
:100A10005E07080008B5074B0340062B05D0830787
:100A200006D10268044B9A4202D1044830F03AFAE7
:100A300008BD00BF0F0080FF7CF40700940208008F
:100A400037B501236A4604460D4616F07FFD009B2C
:100A500023B903482A46214630F02CFA03B030BDB2
:100A6000E70A080037B501236A4604460D4616F02A
:100A70006DFD009B23B903482A46214630F01AFA3F
:100A800003B030BDDC0A0800012808B504D10348D2
:100A900040F2C71130F022FA08BD00BF710B080008
:100AA00008B510B9014830F011FA08BD1607080062
:100AB0002DE9F04104460D4617461E4659B1186807
:100AC00018F086F86168814205D0C388CA88064854
:100AD000892130F0EFF9A06833463A462946BDE84F
:100AE000F04113F0A1BC00BFEF0A08002DE9F04F60
:100AF0002DED028B83078BB004460D4609D10368A8
:100B0000754A934205D111F0030802D10A689A424E
:100B100002D0724830F0C6F943F05AFB18B12846AB
:100B200043F056FB08B96E48F4E7277938461FF0C2
:100B300085FE019028791FF081FE0690384621F04D
:100B4000CBFED4E9036304903A46E079009308A908
:100B5000CDE9083643F07DFBC3690393D4F81CB09C
:100B6000EB69DDF80CA002930746D946B0454BD19E
:100B7000662205F10C01E87943F06BFB6622C3693C
:100B8000049005F10C01E879059343F062FBD0F87D
:100B90001C804FF00009B14561D1009A039B7C692C
:100BA00004FB0234059B08EB860503EB8609A6EBE4
:100BB000020B9046009B08F1FF3A534500F28780F4
:100BC00004980BB0BDEC028BBDE8F08F484605934E
:100BD000019B9847049B504698477A69059B92442D
:100BE000A26901339144009A9342EFD1D7E90523DA
:100BF000009902FB11339A44D4E9053202FB113308
:100C0000994408F10108B1E70023ECE7079358463F
:100C1000019B9847079BA269F3EC017AA0EE278A13
:100C200093440AF1010AD145F0D10298069B9847F6
:100C3000019B584630EE488A9847C8EE007A08EB88
:100C4000890ACAED007AD4E9053202FB19339B44C4
:100C5000029AAB691A44029209F101099BE79FEDE0
:100C6000218A43464FF0000ADDE7019B2046CDE98B
:100C7000022198470399BB69F1EC017A029AE0EEF0
:100C8000278A1C440132B242EFD346454FEA8B0318
:100C90002EBFD84600234FF000084B4408F101084E
:100CA000A3EB8809BB6935ED018A03FB1848404670
:100CB000019B984738EE688A0BF1010BC8EE007A69
:100CC000C9ED007A7C69A8EB0404D04672E7DFED39
:100CD000058A49464246D6E74857080080FE070085
:100CE000C2FC070000000000D0ED077ADFED0F6ABC
:100CF000427BB4EEE70AF1EE10FAD8BFB0EE670A15
:100D0000D0ED017A80ED060AB8EE677AC7EE267A52
:100D100067EE807AFCEEE77A17EE903A53435B0079
:100D2000C26C934294BF83648264704700007A442B
:100D30000E2810B5044610D0084BD3F8A8313BB1AB
:100D40000BF026FC20B12046BDE810400BF068BA3D
:100D50002046BDE8104025F085BF10BD946B0020F3
:100D60004109054A00F01F000123834052F8210089
:100D7000034342F8213070476C6100202DE9F04FA9
:100D800004288BB004462CD07D4D286818B125F07E
:100D900069FF00232B6024B37A4B9C4221D001AB26
:100DA00002932146784B039302A8002601963DF05A
:100DB0000CFF0198013026F025F9286088B1019BCD
:100DC0000890CDE9063601238DF8243006AB049354
:100DD00021466E4B059304A83DF0F7FE2A68019B5F
:100DE000D6546B4C6B4D20680BF01AFA00236A4AFC
:100DF0002360D5F8E8401360002C35D1674E337876
:100E000023B16748047200F053FC347028F052FE9E
:100E100027F0D4FC09F0BAFE624BD5F8FC40002262
:100E20001A70002C55D020460BF0B2FB002800F0C1
:100E30008B80A7685C4B3B40062B06D017F003065F
:100E40001BD13A68594B9A4204D106A938461AF088
:100E500039F80646D5F8FC30DDF81890DFF86C81DB
:100E60006BB916202FF0F6FF94F82530666813B999
:100E700020460DF071FF3446BEE70026EAE7D8F8B9
:100E8000004046B163684B4505D121684A4630466B
:100E90003CF09EF810B1A3689F4251D1E368C8F8B6
:100EA0000030D5F8F830A34202D10023C5F8F8305D
:100EB000002320461A4640F2FD413EF038FBD5F8AB
:100EC000FC40002CAFD1D5F8FC301C46DB68002B71
:100ED000FBD1374FC5F8F8400026069600F0D2FE49
:100EE0003C680DF11808B146002C2FD1069B3B60E1
:100EF000304B1E60304B1C6000F0DAFE30F074F9AD
:100F00002E4B6B63AB8AC5F8044143F00103AB82FF
:100F1000C5F8C0412A4D0AF0BFFF242221462948C6
:100F20003CF0ABF8286825F09DFE2C60264D286823
:100F300025F098FE2C600BB0BDE8F04F28F03EBDC8
:100F4000E36804F10C088BE7E468BAE7D4F808A07A
:100F5000C4F8089020460BF01BFB834660B960681C
:100F60000BF016FB50B9C8F80040304604F10808F1
:100F70002646E0605446B7E70020FAE75846F8E70F
:100F8000986F00200C6C0020079D0600B7870700B3
:100F90005C610020946B002064610020B877002021
:100FA000F0690020AB7700200F0080FF7CF4070081
:100FB000606100206861002054610020040F090076
:100FC000444D0020286D0020F4600020906C00202B
:100FD00038B5084D084C287821F056FF20683BF0C2
:100FE00075FA287821F022FF2068BDE838403BF0F0
:100FF0006DBA00BFF86100203821002008B5064A0C
:10100000034650782BB121F03FFFBDE80840FFF7C1
:10101000DFBF21F00BFFF8E7F861002013B540F2C5
:10102000ED416A4616F01EFA00216A4608463CF079
:10103000E5FA084C3DF060FC08B102B010BDFBF7CA
:10104000D5FFA16A0029F8D16A4608463CF0D6FAD5
:10105000F0E700BF946B00202DE9F3470C461E46D5
:1010600090461CF0CBFEDDE90A57837C5B423B7067
:10107000E307814612D414F0030A03D12268394BE6
:101080009A4207D020463DF02BFC002831D0BAF11F
:10109000000F26D12268334B9A4222D1204617F006
:1010A00085FD031488F8003003123370287099F816
:1010B0001230002B4ED199F80C20042A4AD199F80D
:1010C0001120002A46D098F800203178914241D171
:1010D0002A788A4201BF3A7088F8003033702B704A
:1010E00038E0204617F0EAFCFDEEC07A17EE900AD1
:1010F000D7E76A4601A9204617F076FC04220321AF
:10110000019840F2932311F08DFE009B1868F3F7CD
:101110008DFA009B88F800005868F3F787FA009B67
:1011200030709868F3F782FA019B2870032BBED9C0
:10113000009BDC6820463DF0D3FB70B1204617F0E1
:10114000BDFCDFED097A20EE270AFCEEC07A17EE2F
:10115000900A387002B0BDE8F087204617F026FDEF
:10116000F7E700BF08F6070000007F4370B52DEDDC
:10117000028B0646B0EE408A1CF040FEDFED1F7A7F
:1011800080ED068A28EE278A4289BCEEC88A04468A
:1011900018EE103A9BB29A4209D042680589438101
:1011A000B3F5807F02FB05F5426A03D15AB9BDEC65
:1011B000028B70BD3AB928463BF048FE216A606256
:1011C0002A463BF019FF0023AB420AD194F828309D
:1011D000002BECD0BDEC028B3046BDE8704037F000
:1011E00020BAA27C0AB19A0706D0D4E90812608915
:1011F000D25C42431212CA540133E5E70000804337
:10120000084AD2F8083143B190F8263023F004039D
:1012100080F826300023C2F8083190F82600C0F389
:10122000800070470050024010B50446084617F091
:1012300045FCD4ED067ADFED186A637BA26DB4EE4F
:10124000E70AF1EE10FAD8BFB0EE670AD4ED017AE2
:1012500084ED050AB8EE677A0021C7EE267A67EEBC
:10126000807AFCEEE77A17EE900A5843236C400030
:10127000984238BF18469042236D28BF10466065DB
:10128000121A18443BF0F9FE236B23B12046BDE847
:10129000104044F0FEB810BD00007A442DE9F04F34
:1012A0002DED028B85B00E290446039100F08A8053
:1012B000084617F08DFCC37B3BB9C388584840F201
:1012C000713240F2CF412FF0F5FD03AB0022012136
:1012D00054481AF017F88046039058F8047F0646E1
:1012E0006622012138463CF06BF84FF0000ABA45FF
:1012F00022D10836B900606ADFF82C913BF0A9FDD5
:10130000B9006062A06A3BF0A4FDB900A062E06A87
:101310003BF09FFDC4E90B074FF0000AB7EE008ACF
:10132000BA4552D1236B13B1204644F0B2F805B050
:10133000BDEC028BBDE8F08F58F8045F284617F02B
:1013400047FCC37B81461BB300EB8303364A1B6912
:1013500093421DD1AB4666225BF8045F022128460A
:1013600011F044FD4FF00009A94540F2094202D1B5
:101370000AF1010ABBE7B9F1000F5BF8040F0CBFDB
:1013800011464FF4617147F05AF909F10109EBE791
:1013900028463DF0A5FA08B9EB0705D540F209410A
:1013A000284647F04CF9E3E7B9F80630019340F2DC
:1013B000173300931D4840F2713340F2CF4275213C
:1013C0002FF078FD0026374694E756F82AB05846A5
:1013D00017F0FEFB656AC37B4FEA8A084544ABB150
:1013E00000EB830003694B4510D1DBF808003BF0AC
:1013F0005FF885ED000AA36ADBF80C0098443BF027
:1014000057F888ED000A0AF1010A89E758463BF0CF
:101410004FF885ED000AA36A434483ED008AF2E7A2
:10142000EF0A080044EC0700E9B204007E0B080054
:10143000F8B504460D46FBF7CBFD04F148022846FB
:10144000256440F28D41002516F030F80121204638
:10145000C4E90B5584F8455084F8465045F0E8FA45
:10146000FF2384F85430012120463BF05AFF01212C
:1014700020463BF074FE4FF490522946606B3BF0DF
:10148000FCFD4FF490522946A06B3BF0F6FD266917
:101490003822294630683BF0F0FD4FF4A47229460B
:1014A00070683BF0EAFD4FF48E722946B0683BF05D
:1014B000E4FD41F210222946F0683BF0DEFD4FF4D6
:1014C0005272294630693BF0D8FD4FF4D952294673
:1014D00070693BF0D2FDB06942F2042229463BF02C
:1014E000CCFD256945B3616AE36A2846194434F0A6
:1014F000D7F9013020D0D5F8D037032B1CD195F87F
:10150000D427164BD5F8BC67D5F8C077062101FB68
:101510000233B3F90450FBF74DFD102375432373D9
:101520000123E38105FA03F3A360AD0000236760A4
:101530006673E563A365F8BDE36A0133E3620121E5
:1015400020463BF00CFE94F84530002BC9D0FBF749
:1015500031FD0349034846F0C6FE00BF0C350900C3
:1015600090070800EC0B08002DE9F0470E46FF211C
:101570008172117904463079884203D140F2FE30FD
:1015800011F082FB434800216160057A1DB1017EA4
:1015900000297BD10125404900EB051060608B429A
:1015A00096F8048092F8049023D83C4FBB428CBF3D
:1015B0004FF080674FF0CC7784F809801079A072E3
:1015C000FFF7CEFB3079364DFFF7CAFB6368012287
:1015D0001A72666896F804A0342101FB0AF16A18B1
:1015E00092F82D3043B1204600F062F805202FF02C
:1015F00031FC4FF0C867DFE7B8F11F0F936082F846
:10160000303082F82F3082F832308CBF08F01F0360
:101610004346566003F5E07388BF224A224868506B
:1016200098BF4FF0A04240F20C61B9F11F0F42F891
:1016300023108CBF09F01F034B4603F5E0738CBFEA
:10164000184A4FF0A04240F20C6142F82310336870
:10165000C3F80885C3F80C95C3F82475342303FB3D
:101660000AF3EB5853B13068072140F30730F1F724
:1016700013FC306840F3073034F059FE342303FB89
:101680000A55012385F82D30BDE8F08707482FF073
:101690001DFC00BF4C2100207F1A06008FD00300E4
:1016A000CC6A0020000300507F800700B4090800C6
:1016B000F8B5837AFF2B044633D04668194D377945
:1016C00034237B43EA1892F82D20FAB1EB5823B16A
:1016D000306840F30730F1F7BDFB304621F0FCFEE7
:1016E000342303FB075393F832304BB93368D3F8F4
:1016F000080521F057FB3368D3F80C0521F052FBA5
:10170000342303FB0755002385F82D30A07A28F0F9
:10171000ABF9607A28F0A8F9636800221A72FF23F7
:10172000A372F8BDCC6A002038B543681C681A79EA
:101730000623C4F800351E4B0546342000FB023357
:10174000022283F82D200023C4F88815C4F84435FC
:10175000C4F8483501232362A360D4F850311BB983
:10176000D4F82431002BF8D04FF4A871204642F071
:101770008DFE01236361D4F80431002BFBD04FF4BC
:101780008271204642F082FED4F8243173B12046A3
:101790004FF4927142F07AFED4F8C434C4F8C434E1
:1017A0000024686821F098FE204638BD0124F8E73F
:1017B000CC6A00202DE9F04F1C46436816461A7982
:1017C0001B688B46062187B0C3F80015194B3421DE
:1017D00001FB02330222074683F82D204FF0010A55
:1017E0004FF000094CB9144D786821F075FE284679
:1017F00007B0BDE8F04F2EF067BFB4F5806FA0468C
:101800004FF0000228BF4FF4806801A93846CDE9A7
:101810000289CDE904698DF804A08DF805B0F3F7CD
:1018200071F8054B98420546DED1A4EB0804464406
:10183000D8E700BFCC6A00200000AD0BF8B54568C2
:10184000234C2F7924237B43E2180646127F002A7B
:1018500032D0E35823B1286840F30730F1F7FAFAA1
:1018600024237B43E218E3582D687BB1194BC5F85C
:101870000833537F53B101236B61D5F80431002B3A
:10188000FBD0242303FB074300225A77242303FBC6
:10189000074393F82100FF2801D021F083FA0023A9
:1018A000C5F800350C4B9D4204BF01236B60242317
:1018B00003FB074400232377707A28F0D5F8B07A29
:1018C00028F0D2F8F07A28F0CFF8FF237372F8BD31
:1018D0006C6A00205201080000F002402DE9F04F30
:1018E0009B464368DFF85C90D3F80080DFF858A08F
:1018F00085B007460D461646BBF1000F01D1012009
:1019000017E07B68DC685C4528BF5C46C84505D1AC
:10191000224629464FF000503BF06EFB786869463E
:10192000CDE90054CDE9026421F0EEFC504503D02E
:10193000002005B0BDE8F08F25442644ABEB040B36
:10194000DAE700BF00F002400000AD0B2DE9F04FD8
:101950004368DFF864A0D3F80090DFF860B085B08A
:1019600080460E461546D8F80430DB68AB4228BFE7
:101970002B46D1451F4617D11A4631464FF000502D
:101980003BF03AFB4FF00053D8F8040000246946BE
:10199000CDE90037CDE9024421F0B6FC584505D029
:1019A000204605B0BDE8F08F3346EDE7ED1B3E4421
:1019B000D9D10120F5E700BF00F002400000AD0BD7
:1019C0002DE9F04F83B0994643681B68D3F80C3576
:1019D000013300AF80460D46144604D14F4840F213
:1019E000EE412FF07BFA002A00F08F8001F0604B6F
:1019F000BBF1005F0FD0802A1FD9494BD3F8A83123
:101A0000DBB110463BF022FA03462946224618462F
:101A10003BF0F2FA0546D8F80430187921F0F2FDCF
:101A200090B905F06043B3F1005F10D03D4AC9F8AA
:101A300000203D493D4846F061FCE31D23F00703CB
:101A4000ADEB030D6B46E0E7FBF7D0FAE3E7D8F820
:101A5000046096F804A0504621F0D4FD08B1344A41
:101A6000E5E7344A242303FB0A234FF490715C61B9
:101A70009D6030687B6042F009FD30684FF4AC71C6
:101A800042F004FD7B68316858699A68C1F84425C2
:101A9000C1F848053168012088605B68F3B9336894
:101AA000244AD3F82001D3F858110843F9D099B942
:101AB0000121D9603168D1F85831002BFBD01E4B81
:101AC000242101FB0A22002151611B4AC9F8003080
:101AD000934203D00832ACE7184BF1E70023C9F872
:101AE0000030D8F80430187921F08CFD90B9BBF1A2
:101AF000005F0AD00A4BD3F8A83133B128460AF068
:101B000047FD10B128460AF08BFB20460C37BD4636
:101B1000BDE8F08FFBF76AFAE3E700BF3206080082
:101B2000946B00200A00AD0B0DFF0700EC0B0800C2
:101B30000B00AD0B346B00200000AD0B0800AD0BAB
:101B400003791F2B86BF03F01F03074A4FF0A04203
:101B500003F5E07352F82300C0F302200638012891
:101B60008CBF0020012070470003005008B5436877
:101B700018791F2887BF0D4900F01F0202464FF059
:101B8000A04121F061F9012802D109482FF03AF96A
:101B900002F5E07251F82200C0F38100012803D061
:101BA000C31E5842584108BD0220FCE70003005004
:101BB0009608080008B543680246187921F044F9F0
:101BC00053681A7928B9104621F04EF900F0010047
:101BD00008BD1F2A8ABF054B4FF0A04302F01F0229
:101BE000D3F80405D04000F00100EFE700030050F7
:101BF0000379012914BF032207221F2B86BF03F09C
:101C00001F0306494FF0A04103F5E073120242F0B2
:101C1000030241F823200020704700BF000300505A
:101C200013B50E4B1B78044613B9002002B010BD4B
:101C300008236A460021184643F0C0FF0028F4D06C
:101C4000204627F07BF90028EFD0054BD4F8D420AC
:101C50001A60044B94F8C4201A70E7E7DA79002080
:101C6000E46F0020D7770020C0B240F0007000F190
:101C70007E40033810289ABF014B185C0020704743
:101C8000942C0900084B1A683AB9EFF310820749FF
:101C9000003A18BF01220A7072B6BFF35F8F1A684C
:101CA00001321A60704700BF786F0020B9770020BA
:101CB00008B5094B1A6812B9052027F0BFFE1A684B
:101CC000013A1A601B682BB9BFF35F8F034B1B7877
:101CD00003B962B608BD00BF786F0020B977002055
:101CE0000A4B186880B1C10709D4820709D4430799
:101CF00009D410F4D81F14BF032006207047042015
:101D00007047052070470220704700BFA06F002079
:101D10002DE9F04F9E4B160181468A4617460FCBA0
:101D2000ADF2AC4D09AD85E80F0004362A4600231C
:101D30001468D4F8001581B9D4F8600588420CDA2B
:101D4000D4F86405884208DAD4F86805884204DAD1
:101D5000D4F86C058842C0F2BC800133042B02F138
:101D60000402E5D100242546CEE003F108011AF86B
:101D700002B089B280201BEA000F48F2050E18BF9E
:101D8000E64625F813E001339BB28B424FEA500040
:101D9000F1D1013292B2D300BA429BB2E5D34FF4F3
:101DA000004225F8132001339BB2760825F8132052
:101DB000B6B200231422C4F80C35C4F80435C4F8B4
:101DC0000825C4F81435C4F81035C4F82055C4F8F3
:101DD0002465C4F82835C4F82C35D9F804201279C4
:101DE00001924FF0FF32CDE90222049201AA03F5DD
:101DF000AC71013352F8040B44F82100042BF6D1E6
:101E00000125C4F800554FF48871204642F03EFB8E
:101E1000A560D4F8103133B34FF48871204642F0F6
:101E200035FB5C4B0FCB002605AD85E80F00C4F8F1
:101E30000065334603F5AC72013355F8041B44F8D2
:101E40002210042BF6D1002025F040F8043041F197
:101E50000001C8E900010DF2AC4DBDE8F08F002291
:101E600048F20C0C97E7FBF7C1F8D2E71AF802B07A
:101E700008214FF0800CD4F804E0AEEB030EBEF165
:101E8000460FF8D96368D5F808E51BEA0C0F4EEA4F
:101E9000060EC5F808E512D0D4F804E0AEEB030E48
:101EA000BEF1280FF8D9D5F80CE501394EEA060E37
:101EB000C5F80CE54FEA5C0CDDD1013255E0D4F8F1
:101EC00004E0AEEB030EBEF1110FF8D9EBE762B6FA
:101ED000B9E740F284439E4216D9DFF8D0802E4DF8
:101EE000D8F80030B3420DD2D5F8000108B1C8F8D7
:101EF0000010012231460AF05BFBC5F8000108B171
:101F0000C8F80060D5F80051DFF8A480002024F064
:101F1000DDFFD8E9002390429941F7D30DB1002CA1
:101F20009DD172B6D9F804301C4A1B791C4C1F2B6A
:101F300088BF03F01F034FF0010606FA03F6D2F83C
:101F4000FC3088BF174D43F08073C2F8FC30236823
:101F50004FF4307943F0010398BF4FF0A045236060
:101F600009FB07F900226068134691B28F423FF6E1
:101F70007DAF6268D21A462AFBD963681B1A4B45AB
:101F8000A5D3094B4FF4964043F001039847E9E786
:101F9000188E0700288E0700946B002000ED00E0EB
:101FA000001000E000030050C0200900906F0020E6
:101FB0004829002037B500F03BF8124C6946C4F8B8
:101FC000B4003AF0F3FEC4F8F800B0B9D4F8FC401D
:101FD0000CB903B030BD6568012D0CD129460A4803
:101FE00017F0B2FF01AB01902A464FF42171204651
:101FF0003DF0BAFAEDE7E468EAE76B4601224FF4F8
:102000002171F5E7946B00206C93070010B5074B26
:10201000D3F8B44044B1204644F05BFE014620466C
:10202000BDE8104017F090BF662010BD946B0020F3
:10203000F8B503782F2B00AF06466BD0514CD4F87F
:10204000B45045B902203AF001FF4F49054644F02B
:102050008EFBC4F8B450284644F03BFE044630469C
:1020600044F037FE204402303AF0F0FE04462846A1
:1020700044F02FFE2946024620463AF0BDFF28468E
:1020800044F027FE054638B1231813F8012C2F2AF7
:102090001EBF2F2201351A70304644F01AFE314619
:1020A000421C60193AF0A8FF204644F012FE0022BC
:1020B00021461346154690422ED145B39B00073367
:1020C00023F00703ADEB030D204644F002FE00238E
:1020D0006E46651E204419461A4615F801EF04F8AD
:1020E00001E0BEF12F0F01F1010C02D0BEF1000F93
:1020F00045D1012B2FD115F8013C2E2B3AD1531E7F
:1021000056F823100023A842E7D100236354204649
:10211000BD46F8BD1D4D9EE711F8016B02F1020EA0
:102120002F2E08BF0133704502F1010C0FD92F2E5D
:102130000DD10E782E2E0AD14E782E2E07D10332D5
:10214000904206D08A782F2A08BF45F001056246E2
:10215000B1E70125FBE7022B0CD115F8013C2E2B32
:1021600008D115F8023C2E2B04D1012A88BF02F1B8
:10217000FF32C4E746F822C061460132C2E70133AC
:102180006146C0E7946B00206C9307009DE3070055
:1021900070B50E4C0E1805464FF48071204642F083
:1021A00075F901232360B54202D10120606070BD42
:1021B000D4F80031002BFBD04FF48071204642F060
:1021C00065F9D4F8083505F8013BECE700D000408C
:1021D0002DE9F74F04469DF830A00F4690469BB17D
:1021E00069494FF00009012247F6FB70B1FBF2F696
:1021F000B6FBF3F6351F854208D909F10109B9F19B
:10220000080F4FEA4202F1D102209FE05F4900250A
:102210008B460A68D2F80005C00740F1A580BAF1E4
:10222000000F40F09A80D2F80805864240F0958071
:10223000D2F80C05814540F09080504600F5AC7C0A
:1022400052F82CC0BCF1FF3F40F0838040B2626086
:102250000125227AE76060F3060222723879019341
:10226000FEF77EFD019B6361237A6AF3C713237235
:10227000E368187920F0B6FD63680022C3F80025F2
:10228000002D51D16368424A934272D002F5A042B8
:10229000934270D002F5805293426ED002F53042E4
:1022A00093426CD103205BF8203000250222C3F852
:1022B0000055C3F80455C3F810254FF4FA42C3F88B
:1022C0001455C3F80C55C3F80825324A844602EB6E
:1022D000C000C3F820054FF4004022F83C00042160
:1022E00002EBCC02C3F824154FF0FF31C3F8285598
:1022F0005080C3F82C559080C3F84055D080C3F867
:102300004455C3F84855C3F84C55C3F86015C3F895
:102310006415C3F86815C3F86C156368C3F80C95A9
:10232000C3F80455C3F80865237A6268397903F065
:102330007F0303F5AC73204642F823106368012243
:10234000C3F80025414636F00FFB002003B0BDE87E
:10235000F08F013004287FF471AF0135042D01F1B5
:1023600004017FF456AF0022626052B1002005469E
:102370006FE7284697E7012095E7022093E7FF20C3
:1023800091E70320E2E700BF0024F400AC2009003D
:1023900000C001406072002070B5C368044618791F
:1023A00020F000FD62681F4B9A4232D003F5A04333
:1023B0009A4230D003F580539A422ED003F5304331
:1023C0009A422CD10323217A174E01F07F01F05C51
:1023D00001258D4020EA050001F5AC71F054002381
:1023E0004FF0FF30636042F8210003F5AC7152F802
:1023F0002110013105D10133042BF6D10023C2F89D
:102400000035E36813B1187927F02EFB0023E36051
:1024100070BD0023D7E70123D5E70223D3E74FF0B0
:10242000FF33D0E700C00140C877002008B503287B
:102430000DD8DFE800F00E02060940F2FB3010F084
:1024400023FC40F22130FAE702482EF019FD024841
:10245000FBE708BD3E0808000707080010B5044662
:10246000002024F033FD064B5A68064B800A40EAF0
:102470008150D31821461844BDE810402DF04CB9C6
:10248000107A002080436D3808B502484FF400717F
:102490002EF024FDFE08080010B5114A134604462C
:1024A00053F8FC1F11B916202EF0D4FC186881686F
:1024B000A14210D1C1681960D2F8F830984202D117
:1024C0000023C2F8F8300023BDE810401A4640F25D
:1024D000FD413DF049B8C16800F10C03E2E700BFDF
:1024E000946B002030B52DED068B044683B0083088
:1024F0002BF028FFAB4BD3ED007A04F10C0020EE5B
:10250000279A2BF01FFF2379032BB0EE408A40F26D
:10251000A18004F110002BF015FFF0EE408A042298
:102520000DEB020104F114008DED019A3AF050FD1B
:10253000002800F0928084ED059A002504220DEB1E
:10254000020104F118008DED018A3AF041FD10B14D
:1025500084ED068A002504220DEB020104F11C0023
:10256000CDED018A3AF034FD002878D0C4ED078A19
:10257000DFED8D7A9FED8D5A2379FFEE006AE9EE4B
:10258000276A052BDFED8A7A26EEA66AB8EE000AE6
:1025900066EE865A26EE257A27EE277A66EE067ACA
:1025A00067EE857A9FED835AE6EE057A9FED826AA3
:1025B00077EE867A9FED816AA5EE867A9FED806A36
:1025C000A6EE867A77EE876A77EEC77A38EE087AD3
:1025D00087EE878AF7EE007A61D0062B00F09F80A5
:1025E000042B47D0022B78EE275A26EE800A37EECE
:1025F000C8AA3AD0032B00F0CE80012B0CBF76EE98
:10260000A79A77EEE69AB6EE008A0ABF29EE888A84
:1026100029EE888AF1EE699AB0EE489AC7EEA58A4B
:1026200020EE280A35F0A3FA2AEE280A206235F0B7
:102630009EFA28EE280A606235F099FA29EEA80A77
:10264000A06235F094FA29EE280AE06235F08FFA9C
:10265000206306E0DFED5B8A61E701256EE7002D70
:1026600086D003B0BDEC068B30BDDFED569AB1EEDF
:10267000489AD3E788EE28AAB0EE677AA8EE887A5F
:1026800026EE800AB0EE679AA8EEC89A7AEE275A2C
:10269000F0EE409A37EECAAAB0EE478ABEE74A4B40
:1026A00018EE902AF6EE005AA3EB520306EE103A0B
:1026B00068EEA55AB7EE087A65EE865A38EEA75A44
:1026C000A6EE657AB0EE459A27EE067A38EEE76A0E
:1026D00027EE287AA6EE669AF0EE469AB0EE45AA64
:1026E000A6EE26AAE5EE669A37EE077A78EEA85AA5
:1026F000F0EE494AA5EE266AA7EE489A69EEA59A39
:10270000F0EE4A5AE7EE084AE7EE085A29EE289A10
:1027100026EE000AA7EE48AA24EEA88A7EE72A4BF6
:1027200018EE902AF6EE005AA3EB520306EE103A8A
:1027300068EEA55AB7EE087A65EE865A38EEA75AC3
:10274000A6EE657AB0EE459A27EE067A38EEE76A8D
:1027500027EE287AA6EE269A37EE077AB0EE45AA3B
:10276000A6EE66AAF0EE469AF0EE494AE5EE269A03
:10277000A7EE489AA5EE666A28EE800AF0EE4A5A5D
:1027800069EE809AE7EE084AE7EE085A29EE289AA1
:1027900036EE060ABEE7F0EE409AB0EE679AB0EE6B
:1027A000678A3BE72470002083F9A23FEA95323C18
:1027B0008964E1BAB3375FBE9503353F6AC9693DA5
:1027C000E42B0EBF00000000DF59375F70B50446F0
:1027D0002DED048B10302BF0B5FD404BD3ED007A7E
:1027E00004F11C0020EE279A2BF0ACFD94ED088A32
:1027F000257B39EE088AF0EE408A38EE008A002DFB
:1028000064D0DFED377AB4EEE79AF1EE10FA59DDD5
:10281000DFED347AB4EEE78AF1EE10FAC8BFB0EE1D
:10282000678AE66A731B07EE903AF8EEE77A78EE6D
:10283000688A27EE888AC4ED088AB0EE480A08F054
:102840007DFEFCEEC07AA16A17EE903A31F91320B2
:1028500008EE902A627BF8EEE88AD2B1F8EE677A49
:102860005A1C964238EE678A03D1002D14BF1A46CF
:10287000002231F9123007EE903AF8EEE77AB7EE1F
:10288000007A37EE487A67EE887AE7EE287AF0EE3B
:10289000678A04F114002BF055FD04F11800B0EE26
:1028A000409A2BF04FFD6FF00E00B0EE408AB0EE74
:1028B000680A0CF0DDFDA0EE098AB0EE480ABDEC16
:1028C000048B70BDADD5F4EEC87AA5E7B0EE480A2A
:1028D00008F034FE38EE408AA3E700BF28700020DD
:1028E0000000000000FE7F3F10B504462DED028B76
:1028F0000C302BF027FD237E0D2BF0EE408A06D105
:10290000B0EEC08AB0EE480ABDEC028B10BD04F1F7
:1029100010002BF017FD04F11400B0EE408A2BF0EC
:1029200011FD237E0C2B00F2D880DFE803F0070CAA
:102930001116363B533E5F7E9BBDCC0038EE888A35
:1029400038EE008ADEE738EE888A38EE408AD9E72A
:1029500028EE888A28EE008AD4E7F0EEC07AF4EEFA
:10296000677AF1EE10FA13D69FED5F7AF4EE477AAC
:10297000F1EE10FA0CDC9FED5D7AF4EEC77AF1EE21
:1029800010FA05DAB5EE400AF1EE10FA00F0A58073
:1029900068EE888A88EE808AB4E7A8EE880AB0EEEE
:1029A000408AAFE738EE888AD4E7B5EEC00AF1EE88
:1029B00010FA06D4F7EE007AB4EEE70AF1EE10FA58
:1029C00011DCDFED4B7AF4EEC07AF1EE10FAC8BFFD
:1029D000B0EE670AF7EE007A77EEC07A20EE088A4A
:1029E000A7EEA88A8EE7B0EE670AF3E7F0EEC87AA2
:1029F000F4EE677AF1EE10FA12D69FED3B7AF4EE20
:102A0000477AF1EE10FA0BDC9FED387AF4EEC77AD4
:102A1000F1EE10FA04DAB5EE408AF1EE10FA5CD06D
:102A2000C8EE887A37EE808A6CE7F0EEC07AF4EE72
:102A3000677AF1EE10FA12D69FED2B7AF4EE477A10
:102A4000F1EE10FA0BDC9FED297AF4EEC77AF1EE85
:102A500010FA04DAB5EE400AF1EE10FA3DD078EE45
:102A6000888A97E7F4EEC88AF1EE10FA0FD5B4EE33
:102A7000C08AF1EE10FA3FF545AFB4EEE80AF1EE88
:102A800010FAD4BFB0EE688AB0EE408A3AE7F4EEAE
:102A9000C08AF1EE10FA23D4B4EEC08AF1EE10FA37
:102AA000D8BFB0EE408A2DE7B4EEC80AF1EE10FAB6
:102AB000D8BFB0EE408AB4EEE88AF1EE10FAC8BF93
:102AC000B0EE688A1EE7B4EEC08AF1EE10FAD8BF05
:102AD000B0EE408AF4EEC88AEFE79FED058A11E771
:102AE000B0EE688A0EE700BFFFFF7F7F0000800026
:102AF000000000007FB50C46E107054617D4A20789
:102B000020D12268234B9A421CD14268E36B9A423F
